:100000000C9433070C9464070C9464070C946407F5
:100010000C9464070C9464070C9464070C946407B4
:100020000C9464070C9464070C9464070C946407A4
:100030000C9464070C9464070C9464070C94D72800
:100040000C9464070C9464070C9464070C94640784
:100050000C9464070C9464070C9464070C947D530F
:100060000C9464070C9442180C9418180C946407B0
:100070000C9464070C9464070C9464070C94640754
:100080000C9464070C9464070C9464070C94640744
:100090000C9499340C9409340C9450340C94A1436E
:1000A0000C9464070C9464070C9464070C94640724
:1000B0000C9464070C9464070C9464070C94640714
:1000C0000C9464070C9464070C9464070C94EE176A
:1000D0000C94C4170C9464070C9464070C94640784
:1000E0000C946407420827082E08420842084E086C
:1000F00057082E0842084208D40AD90ADE0AE80A3C
:10010000F20A6B0BFC0A040B0C0B160B200B2A0BD0
:10011000390B430B6B0B4D0B570B610B070DF10CA0
:10012000F10C070D070D140D160D160D070D070D1B
:10013000F5100511E11023112311231123112311AF
:100140002311231123112311D00E5C106310DA1038
:100150007C107D1E7D1E7D1E7D1E7A1E7A1E811ED8
:10016000811E811E811E811E811E811E811E7A1E9E
:100170007A1E811E811E811E811E811E7F1E7D1E94
:10018000B32EA12EA12EB32EB32EB32EBF2EBF2E73
:10019000B32EB32E1E301A301A301E301E301E30D1
:1001A0002130E72F1E301E30A235A535BD35D435A0
:1001B0001D363036503613521652055209520F5220
:1001C0004D521A521E52245228522C52325236523A
:1001D0003A524D5240524452485207634236B79BFE
:1001E000D8A71A39685618AEBAAB558C1D3CB7CC97
:1001F0005763BD6DEDFD753EF6177231BF0000000F
:10020000803F08000000BE922449123EABAAAA2AF1
:10021000BECDCCCC4C3E00000080BEABAAAAAA3E0C
:1002200000000000BF000000803F00000000000848
:100230004178D3BB4387D1133D190E3CC3BD4282E5
:10024000AD2B3E68EC8276BED98FE1A93E4C80EFA3
:10025000FFBE01C4FF7F3F00000000000C94B84CBB
:100260000C9454210C94430B0C94E80A0C942F2703
:100270000C94E72F0C94D95F0C9424520C941A30F0
:100280000C94A4210C943C4E0C94F10C0C941E2262
:100290000C94040B0C9468450C94A6150C94161938
:1002A0000C940E410C94E1260C948D2A0C94F1458B
:1002B0000C94A4150C94160D0C9461450C944D30BF
:1002C0000C945C100C9450140C94F5100C942C525B
:1002D0000C94A12E0C9493210C940C0B0C94F726E7
:1002E0000C94753B0C944D150C94BD350C942E0854
:1002F0000C9432410C94B7140C946A450C944D0B39
:100300000C943A520C9421300C9422280C94070D32
:100310000C9405520C948C2A0C94E6200C94D12158
:100320000C9463100C9466070C94D00E0C94420845
:100330000C943E470C9433460C94AE270C94C75350
:100340000C9456460C94A24C0C940F410C94F20A57
:100350000C941E520C94DE0A0C9440520C94474D9F
:100360000C944D520C94A5350C94DD530C941652FC
:100370000C94FC0A0C94D40A0C94140D0C94E553C0
:100380000C948F210C94B6200C947F1E0C94902A10
:100390000C94A2350C9462470C94D90A0C947417EF
:1003A0000C941A520C94200B0C94134E0C9444523F
:1003B0000C941E410C9494140C94A3140C94503679
:1003C0000C94B32E0C9403270C94A8150C94E31BE7
:1003D0000C94D8200C94AD460C944D450C941E30D2
:1003E0000C9406460C9423110C947A1E0C9409521A
:1003F0000C949A230C9413520C940F520C94485260
:100400000C94811E0C9411210C94160B0C947446C0
:100410000C945A460C947C100C94F6460C945B2178
:100420000C9451450C941D360C9430270C94BF2E1F
:100430000C94E1100C94B5150C9475450C94D435BE
:100440000C94B1150C9401270C9457080C94C51406
:100450000C9427080C947E450C9406150C940511F9
:100460000C944E080C942A0B0C9432520C94931654
:100470000C94DA100C94FB440C9430360C947352A8
:100480000C94F44D0C946B4F0C94C1210C947D454D
:100490000C94570B0C9418170C94A14C0C942852E4
:1004A0000C9449450C94390B0C94610B0C949920D5
:1004B0000C9436520C942E4D0C946B0B0C942921F9
:1004C0000C947D1E496E76616C6964204D41433AFF
:1004D00020736574206669726D7761726527732079
:1004E0004D414300496E76616C696420636F6D6DA8
:1004F000616E64003E3E2000312D77697265206395
:100500006F756E743A200020416464723A0064652D
:1005100076230020616C69766500204E6F64653A31
:1005200000536561726368696E67004D6F64627540
:100530007320706F6C6C696E67206572726F723DAC
:10054000002056616C3A20004D423A20004D6F6405
:1005500062757320706F6C6C696E67206572726F64
:10056000723D002D002050492056616C203A004D0C
:100570006F6462757320706F6C6C696E6720657252
:10058000726F723D002D0020464D2056616C203A5E
:10059000002F6D79686F6D652F735F6F75742F0015
:1005A00020000A667265653A00202D2D00204F4616
:1005B0004600204F4E00204F46460020636D643AAF
:1005C000002043757274656D703A00205365743A6B
:1005D000002045787069726564003D002F00496E07
:1005E0003A20003A003D3E003D00564323004D6F47
:1005F00064627573206F70206661696C65640020A9
:10060000636D643D003D0056435F6865617423007F
:100610003D0050696E3A003D0050696E3A00573A0D
:10062000002048616C74656400466F7263652057F2
:1006300068697465003D00526573746F7265643A51
:1006400020003A204E6F2073746F726564207661CB
:100650006C756573202D2064656661756C7400523D
:100660006573746F7265642066726F6D3A00204D19
:10067000454D3D00436D643D00526562696E6420E6
:1006800073756363657373004572726F723A20729B
:100690006562696E64206661696C0052656E65779B
:1006A00065642073756363657373004572726F725E
:1006B0003A2072656E65776564206661696C0041F9
:1006C0006363657074696E6720636F6D6D616E64DE
:1006D000732E2E2E002074727920616761696E205E
:1006E000696E2035207365636F6E6473006661699F
:1006F0006C65642C2072633D004177616974696E9A
:100700006720666F722072657461696E656420741B
:100710006F70696373002F6D79686F6D652F696EF7
:100720002F00636F6E6E65637465642061732000D3
:10073000202E2E2E0020757365723A003A00417407
:1007400074656D7074696E67204D51545420636FE9
:100750006E6E656374696F6E20746F200046616908
:100760006C656420746F20636F6E6669677572656F
:100770002045746865726E6574207573696E6720B4
:1007800044484350005374617274696E67206C6111
:100790006E0072657175657374204D515454204319
:1007A0006F6E66696700536176656420746F2045DB
:1007B0004550524F4D00536176696E6720636F6EEE
:1007C00066696720746F20454550524F4D2E2E00AC
:1007D000636F756C64206E6F742070617273653A1C
:1007E000200055706461746564006F6E006F66660A
:1007F00000485454502F312E312025690020485490
:1008000054502F312E310D0A486F73743A202573DE
:100810000D0A4163636570743A202A2F2A0D0A433A
:100820006F6E6E656374696F6E3A20636C6F73658B
:100830000D0A0025730020000D0A004745540020D2
:1008400074727920616761696E20696E203520734A
:1008500065636F6E6473006661696C656420746FB4
:1008600020636F6E6E656374004552524F523A209A
:100870005365727665722072657475726E65642058
:1008800000436F6E6669672070617273696E6720DE
:100890006661696C656400676F7420436F6E66699A
:1008A0006700436F6E666967205552493A20687445
:1008B00074703A2F2F00282B294F57495245002892
:1008C0002B294D4F4442555300282B29444D5800A5
:1008D000282B294453323438322D31303000282B24
:1008E000294672656552616D207072696E74696E19
:1008F0006700435553544F4D5F4649524D5741523F
:10090000455F4D4143004669726D77617265204DC8
:100910004143204164647265737320006C617A798D
:10092000686F6D652E727500436F6E666967207320
:1009300065727665723A00282B2957415443484422
:100940004F470038643865333537000A4C617A798F
:10095000686F6D652E7275204C69676874487562A2
:1009600020636F6E74726F6C6C65722000010210F0
:1009700020200808102040102040800201020108B9
:100980000402010102040810204080804020100869
:1009900004020180040201804020100804020108C2
:1009A0000402010102040810204080010204081022
:1009B00020408000002200250028002B002E00315E
:1009C00000340002010000050108010B01050505C6
:1009D00005070508080808020202020A0A080804B6
:1009E00004040401010101010101010303030303E4
:1009F000030303040707070C0C0C0C0C0C0C0C0273
:100A000002020206060606060606060B0B0B0B0B79
:100A10000B0B0B436F6E6E2E2061626F72746564F8
:100A2000003A3D0041637469766500477270206347
:100A30006865636B3A20005265747279696E67204D
:100A4000434D440053746174757320646566666534
:100A5000726564002D3E005075623A2000556E6B41
:100A60006E6F776E20636D642000536B69707069E0
:100A70006E672E2E004F4F4D21005D20000A5B0057
:100A80002E004D7920495020616464726573733A79
:100A900020003A00436F6E66696775726564204D89
:100AA00041433A00444D58696E204275666665724E
:100AB00020616C6C6F632065727200496E697420EE
:100AC000696E2063683A0009445332343832206535
:100AD00072726F720009526573657420646F6E657F
:100AE0000009436865636B696E6720666F72203129
:100AF0002D5769726520646576696365732E2E2EA5
:100B0000004453323438322D3130302070726573E6
:100B1000656E74004453323438325F3130305F498F
:100B200032435F544F5F31575F425249444745203B
:100B3000696E69740020416464723A0064657623CA
:100B400000312D7769726520006D71747420006D1D
:100B50006F646275732000696E707574732000692C
:100B600074656D732000436F6E66696775726564A6
:100B70003A003D0050696E3A00444D5820696E209D
:100B8000737461727465642E204368616E6E656C67
:100B9000733A00444D58206F7574207374617274F9
:100BA00065642E204368616E6E656C733A20004C5C
:100BB0006F61646564006C6F6164206661696C6577
:100BC00064004E6F2073746F72656420636F6E668D
:100BD0006967006C6F6164696E6720436F6E666958
:100BE0006700005EBCE2613FDD83C29C7E20A3FD06
:100BF0001F419DC3217FFCA2401E5F01E3BD3E60FB
:100C000082DC237D9FC1421CFEA0E1BF5D0380DE2C
:100C10003C62BEE0025CDF81633D7C22C09E1D43DE
:100C2000A1FF4618FAA427799BC584DA3866E5BB8C
:100C30005907DB856739BAE406581947A5FB7826BA
:100C4000C49A653BD987045AB8E6A7F91B45C698EC
:100C50007A24F8A6441A99C7257B3A6486D85B059E
:100C6000E7B98CD2306EEDB3510F4E10F2AC2F714C
:100C700093CD114FADF3702ECC92D38D6F31B2EC7A
:100C80000E50AFF1134DCE90722C6D33D18F0C52AC
:100C9000B0EE326C8ED0530DEFB1F0AE4C1291CF5E
:100CA0002D73CA947628ABF517490856B4EA69370C
:100CB000D58B5709EBB536688AD495CB2977F4AA3A
:100CC0004816E9B7550B88D6346A2B7597C94A146C
:100CD000F6A8742AC896154BA9F7B6E80A54D7891E
:100CE0006B3500002100240027002A002D00300071
:100CF000330001010000040107010A010000200087
:100D00002300260029002C002F00320000010000E3
:100D100003010601090100000A0B02090C0D0E086F
:100D200007030401000000000000000000000000B4
:100D300000000000000000000000000000000000B3
:100D40000000121110000000000000000000000070
:100D50000000000000000000000000002F6D796816
:100D60006F6D652F735F6F75742F004E6F74206603
:100D7000696E64003D005573652074686520636F7B
:100D80006D6D616E64733A202768656C7027202D45
:100D9000207468697320746578740A2773657420F9
:100DA00064653A61643A62653A65663A66653A3006
:100DB00030272073657420616E642073746F7265D0
:100DC000204D41432D6164647265737320696E2008
:100DD000454550524F4D0A277361766527202D20D7
:100DE0007361766520636F6E66696720696E204E59
:100DF0005652414D0A2767657427202D2067657478
:100E000020636F6E6669672066726F6D2070726511
:100E10002D636F6E666967757265642055524C0A62
:100E2000276C6F616427202D206C6F616420636FD5
:100E30006E6669672066726F6D204E5652414D0A8C
:100E4000276B696C6C27202D207465737420776183
:100E5000746368646F67006364696E6F707375783C
:100E6000585B0000D95F11241FBECFEFD1E2DEBF77
:100E7000CDBF00E00CBF15E0A0E0B2E0E8ECFEED75
:100E800000E00BBF02C007900D92A832B107D9F75E
:100E90002BE0A8E2B5E001C01D92A539B207E1F749
:100EA00017E0C3E3D7E000E006C021970109802FD7
:100EB000FE010E941161C233D10780E00807A9F743
:100EC0000E943A550C94626F0C9400003F924F922E
:100ED0005F926F927F928F929F92AF92BF92CF92CA
:100EE000DF92EF92FF920F931F93CF93DF93CDB7D3
:100EF000DEB761970FB6F894DEBF0FBECDBF7C01A1
:100F00006B012A014901702E64E776E081EC96E0DE
:100F10000E94C0154AE050E0B60181EC96E00E94C4
:100F20008C166EE676E081EC96E00E94C0159E017C
:100F30002F5F3F4F590180918B0B90918C0B009745
:100F400011F485E99BE0A501481B590B052E000C07
:100F5000660B770B2AE081EC96E00E94F91581EC94
:100F600096E00E94D9161B861A861D861C861F864F
:100F70001E868114910479F460E070E0C7010E943C
:100F800032508C0133E0C316D104E9F084E0C81676
:100F9000D10491F035C0F401DE011A9680E090E0B2
:100FA000841595054CF78330910531F321913191EA
:100FB0002D933D930196F4CFC7010E94B02F892B4A
:100FC00009F095C088C0D70118968C91873009F434
:100FD000CCC0C7010E945E50853079F46FE576E0A1
:100FE00081EC96E00E94C0154AE050E065E070E0B8
:100FF00081EC96E00E94DD166EC08DEF9FEF91C6EA
:10100000B1E0CB16D10409F466C024F4C114D104B4
:1010100061F0ABC0F2E0CF16D10409F468C025E05E
:10102000C216D10409F47EC0A0C069E0C7010E94C5
:101030004950D70118968C9190E08A309105B8F507
:10104000FC018827EE58FF4F8F4F0C9411618C855F
:101050009D85892B19F48FE7F70180874A855B8589
:101060006C857E85C7010E94FF4F772001F160E209
:10107000C7010E94495064E47AE081EC96E00E9446
:10108000061715C0772051F060E2C7010E94495051
:1010900064E47AE081EC96E00E9406174A855B855D
:1010A000052E000C660B770BC7010E94FF4F0E94B4
:1010B00071536093990570939A0580939B05909363
:1010C0009C05D70112968D919C911397909398054A
:1010D000809397054AC0F7018085813009F064C488
:1010E000C7010E945E50813009F05EC419C5C70176
:1010F0000E945E508530B1F11B861A861D861C86C3
:101100001F861E8662E0C7010E944950772051F178
:1011100020E030E040E050E062E070E0C7010E9473
:101120009E2D20C0C7010E94B02F18161906ECF49E
:101130001B861A861D861C861F861E8665E0C701D3
:101140000E94495020E030E040E050E062E070E072
:10115000C7010E949E2D61E276E081EC96E00E943C
:10116000061703C032E0C32ED12CD70118968C91FC
:10117000843009F457C158F4813009F446C0B0F105
:10118000823009F472C0833009F4A8C10CC48830DD
:1011900009F453C338F4863009F479C1873009F46F
:1011A00052C101C4893009F4BBC28F3709F0FBC3B7
:1011B00060E0C8010E94C32960E0C80101960E9456
:1011C000C32960E0C80102960E94C329AE85BF858D
:1011D0002FEF30E00E94206124E630E040E050E054
:1011E0000E94216F622FC801039619C1AA85BB8591
:1011F0002FEF30E00E94206124E630E040E050E034
:101200000E94216F622FC8010AC12C853D8584E6AA
:1012100090E0821B930B2E853F85829FD001839F98
:10122000B00D929FB00D11242FEF30E00E9420618D
:1012300020E137E240E050E00E94216F622FC801B8
:101240000396288B398B0E94C3296EE176E081ECEE
:1012500096E00E94C0154AE050E02889622F398943
:10126000732F81EC96E00E94DD16AE85BF852FEFCF
:1012700030E00E94206124E6822E912CA12CB12C1A
:10128000A50194010E94216FE22EC22EAC85BD857E
:101290002FEF30E00E942061A50194010E94216F90
:1012A000F22ED22EAA85BB852FEF30E00E9420615E
:1012B0002DE631E040E050E00E94216F522F422F96
:1012C0004F71440F440F842F880F45E5682F649FAA
:1012D000060E60E0611D1124922F9074207257FD5C
:1012E00021C091110BC0211104C0862F8095562F6B
:1012F00011C055E5560F40E06BEA33C021110DC017
:10130000482F5AEA459F040E40E0411D11248BEA04
:10131000841B560F682F40E024C080E0562F509564
:10132000462F0EC0911111C021110CC0482F2AEA7E
:10133000429F040E40E0411D11245BEA541B4B5AAE
:1013400060E00FC0462F40950BC0211104C085E519
:10135000860F4BEA03C08AEA860F90E0461B682F8F
:1013600050E0BFEFDB1609F426C0DD2009F166234B
:1013700029F02F2D629F060E60E0611D552329F094
:101380003F2D539F050E50E0511D442329F02F2D72
:10139000429F040E40E0411D1124F0942F2D229F06
:1013A000020E20E0211D1124620F520F420F03C0D4
:1013B0004FEF5FEF6FEF3FEFC31609F421C020E05E
:1013C0003E2D332321F0339F212D09F02F5F22235F
:1013D000A1F0662321F0629F060E60E0611D552397
:1013E00021F0529F050E50E0511D442321F0429FF1
:1013F000040E40E0411D112403C040E050E060E0D5
:10140000C801498B588B0E94C3295889652FC80190
:1014100001960E94C3294989642FC80102960E943F
:10142000C329C1C2D70114960D911C911597F801DB
:101430008085853009F0B7C2C8010E94631F8330E0
:1014400009F0B1C20FC2D7011496ED91FC91159726
:101450008085853009F0A7C2E680F780E114F104A9
:1014600009F4A1C2F70161857285C5010E94CD50C2
:10147000072D9E01265F3F4FA201B601C5010E94C4
:101480006607D7011296ED90FC901397E7CFE02EF8
:1014900061E0802F0E94FB52FF24F394CA94CD2870
:1014A00009F0F12C6F2D8E2D0E94CB5269E176E070
:1014B00081EC96E00E94C0154AE050E0B80181EC52
:1014C00096E00E948C1667E176E081EC96E00E943F
:1014D000C0156F2D70E04AE050E01DC117FF07C036
:1014E000119501951109EE24E394F12C02C0E12C31
:1014F000F12CD02E61E0802F0E94FB528091A10040
:10150000887F8093A10080919100887F80939100D3
:101510008091A10082608093A100809191008260FF
:1015200080939100AA85BB85EF2899F0CD01BB0F70
:10153000AA0BBB0B9C01AD0124563109410951098D
:10154000AFEFB0E00E94406F2CE93FEF4FEF5FEF4D
:1015500008C02FEF30E00E94206124E630E040E038
:1015600050E00E94216F790161E08D2D0E94FB52B5
:10157000E114F10409F4B3C0EFEFEE16F10409F43D
:10158000B0C0F801FF27EA5EF24FE4914E2F50E021
:10159000FA013197E231F10508F09DC08827E4583F
:1015A000FF4F8F4F0C94116184B5806884BDE7BCF8
:1015B0009CC084B5806284BDE8BC97C080918000E7
:1015C000806880938000F0928900E09288008DC04E
:1015D00080918000806280938000F0928B00E09286
:1015E0008A0083C080918000886080938000F092A0
:1015F0008D00E0928C0079C08091B000806880936B
:10160000B000E092B30071C08091B000806280931E
:10161000B000E092B40069C080919000806880932F
:101620009000F0929900E09298005FC08091900045
:10163000806280939000F0929B00E0929A0055C0E7
:1016400080919000886080939000F0929D00E092DD
:101650009C004BC08091A00080688093A000809186
:10166000A0008F7B8093A000F092A900E092A800D8
:101670003CC08091A00080628093A000F092AB00FB
:10168000E092AA0032C08091A00088608093A00000
:10169000F092AD00E092AC0028C0809120018068FB
:1016A00080932001F0922901E09228011EC08091D0
:1016B0002001806280932001F0922B01E0922A01A8
:1016C00014C080912001886080932001F0922D0148
:1016D000E0922C010AC0F0E8EF16F10414F460E087
:1016E00001C061E08D2D0E94CB5262E176E081EC79
:1016F00096E00E94C0154AE050E0B80181EC96E007
:101700000E948C1660E176E081EC96E00E94C015A4
:101710004AE050E0B70181EC96E00E94DD1643C13B
:101720001A8560E070E0C7010E943250082FB92E80
:101730006AEE75E081EC96E00E94C0154AE050E048
:10174000602F7B2D81EC96E00E948C1668EE75E090
:1017500081EC96E00E94C015612F012E000C770BE2
:101760004AE050E081EC96E00E94DD1680913A0557
:1017700090913B05892B89F06EEE75E081EC96E047
:101780000E9406176C2D6064C7010E944950412FCA
:10179000110F550B660B770BA2C081E090E0909380
:1017A0003B0580933A0526E040E855E260E070E0B2
:1017B00084E296E00E946C180093FD0784E296E0B4
:1017C0009093FC078093FB071092080910920A0976
:1017D0001092090980ED97E0909383088093820826
:1017E0001092850810928408112339F085E090E06A
:1017F000909387088093860804C0109287081092FF
:10180000860886E00E94921C62E370E080E090E02F
:101810000E94375382ED97E090938308809382086B
:10182000109285081092840824E61202A001112467
:101830005093870840938608AFC0D7011496ED9166
:10184000FC91159761857285C5010E94CD50C50137
:101850000E94F24F882309F4A6C08985893009F0D7
:10186000A2C0ADC160E0C8010E94F01BDC01199666
:101870003C901997D32C1A96CC9061E0C8010E9435
:10188000F01BFC01418452846384748462E0C801CB
:101890000E94F01BDC0119960D911C911A97AA85E4
:1018A000BB852FE330E00E94206124E630E040E079
:1018B00050E00E94216F49015A0180913A059091B0
:1018C0003B05892B81F06EEE75E081EC96E00E947D
:1018D000061760E4C7010E944950B501A401C70181
:1018E0000E94FF4F60C081E090E090933B058093A1
:1018F0003A0526E240E855E260E070E084E296E0D6
:101900000E946C183092FD0784E296E09093FC07E9
:101910008093FB071092080910920A091092090996
:10192000012B09F448C1982C882488248A944AE021
:1019300050E06D2D7C2D81EC96E00E948C1665EEBA
:1019400075E081EC96E00E94C015B301A201662704
:10195000772720E181EC96E00E94F91563EE75E0AF
:1019600081EC96E00E94C015A40160E070E020E1E7
:1019700081EC96E00E94F91581EC96E00E94D91660
:101980005092830840928208109285081092840831
:10199000909287088092860886E00E94921C10929E
:1019A0003B0510923A05BDC161E0C7010E94495054
:1019B000C7010E940E50AB01BC0114161506160695
:1019C00017060CF041C0D70118968C9190E08A3030
:1019D000910560F5FC018827E257FF4F8F4F0C946B
:1019E00011614A875B87862F062E000C990B9D8715
:1019F0008C87872F072E000C990B009711F480E538
:101A000090E09F878E87C7010E94FF4F3FC05B8792
:101A10004A8760E2C7010E94495064E47AE081ECA1
:101A200096E00E9406174DC05B874A87772049F0F1
:101A300020E030E040E050E061E070E0C7010E944B
:101A40009E2D20E030E03FC02AE030E081EC96E0BF
:101A50000E94421662E476E081EC96E00E9406174E
:101A6000F7018085853079F060F481508230D8F4B8
:101A700084E690E09B878A871D861C869F878E87D9
:101A800005C0883081F484E190E00FC060E2C701B6
:101A90000E94495064E47AE081EC96E00E940617C7
:101AA00023E030E010C084E690E09B878A879E01A7
:101AB000265F3F4F41E050E060E070E0C7010E94C8
:101AC0009E2D21E030E0CE010A966C01812C912CF4
:101AD00082169306F1F167E376E081EC96E0288BBD
:101AE000398B0E94C0154AE050E0B40181EC96E0C9
:101AF0000E948C1665E376E081EC96E00E94C015AA
:101B0000D6016D917D916D014AE050E081EC96E047
:101B10000E94DD16BFEF8B1A9B0A39892889D8CF1E
:101B20000E9471532091990530919A0540919B052F
:101B300050919C05DC01CB01821B930BA40BB50BD0
:101B4000853F9140A105B10520F0F70180858130E6
:101B500071F0F7018085813031F48C859D85892B6A
:101B600011F48FE78087CC24C394D12CFECA69E29C
:101B700076E081EC96E00E9406178FE7D701189671
:101B80008C931D861C8684E690E09F878E874A850D
:101B90005B8560E074E6C7010E94FF4F7720C9F2C1
:101BA0009E01265F3F4F43E050E060E070E0C701D8
:101BB0000E949E2DCECF992499249A94B8CE1C2DA4
:101BC0009A8460E070E0C5010E943250082FB92E5F
:101BD00067E076E081EC96E00E94C0154AE050E0B4
:101BE000602F7B2D81EC96E00E948C1665E076E0FC
:101BF00081EC96E00E94C015692D092C000C770B32
:101C00004AE050E081EC96E00E948C166FEF75E0A0
:101C100081EC96E00E94C0154AE050E06C2D0C2C3F
:101C2000000C770B81EC96E00E94DD1680913A055E
:101C300090913B05892B89F06EEE75E081EC96E082
:101C40000E9406176C2D6064C7010E944950492DFF
:101C5000990C550B660B770B42CE81E090E0909388
:101C60003B0580933A0526E040E855E260E070E0ED
:101C700084E296E00E946C180093FD0784E296E0EF
:101C80009093FC078093FB071092080910920A09B1
:101C9000109209091230A1F1153091F1692D990CBA
:101CA000770B880B990B0E94576222E538EB42E1D3
:101CB00052E40E943C6120E030E040E251E40E94A6
:101CC0000C632DEE3EE94CE35EE30E94AD616B01D7
:101CD0007C0120E030E0A9010E94076320E030E0B1
:101CE00040E05FE387FD05C0C701B6010E943C618B
:101CF00004C0C701B6010E943B610E941F6202C07E
:101D000060E070E083ED97E0909383088093820811
:101D10001092850810928408709387086093860853
:101D20003BCE61960FB6F894DEBF0FBECDBFDF91FC
:101D3000CF911F910F91FF90EF90DF90CF90BF90C8
:101D4000AF909F908F907F906F905F904F903F905B
:101D500008954F925F926F927F928F929F92AF926F
:101D6000BF92CF92DF92EF92FF920F931F93CF9388
:101D7000DF93CDB7DEB766970FB6F894DEBF0FBE20
:101D8000CDBFE0914005F09141053C96E131F10570
:101D900008F059C28827E856FF4F8F4F0C94116105
:101DA00065E877E081EC96E00E9406170FB6F8949C
:101DB000A895809160008861809360001092600017
:101DC0000FBE8091FB0581112AC01092E30510928D
:101DD000E20588EE93E0A0E0B0E08093E405909304
:101DE000E505A093E605B093E70588E993E09093B5
:101DF000E1058093E00584E693E09093EF058093FE
:101E0000EE051092F0051092F1051092F205109275
:101E1000F30584E08093F80581E08093FB058DE96C
:101E200095E090931706809316066CE271E080E0CF
:101E300090E00E94375361E085E30E94CB5261E05D
:101E400085E30E94FB528CB580618CBD8CB58064AB
:101E50008CBD61E084E30E94FB5261E083E30E9459
:101E6000FB52249A80E590E00E94AB2767E080E077
:101E700090E00E947C4065E58BE190E00E947C4010
:101E800065E58AE190E00E947C400E94AA2780E0FC
:101E900090E49093A10A8093A00A80E090E690934A
:101EA000A90A8093A80A80E098E49093A30A8093FB
:101EB000A20A80E098E69093AB0A8093AA0A80E099
:101EC00090E59093A50A8093A40A80E090E7909310
:101ED000AD0A8093AC0A80E098E59093A70A8093BE
:101EE000A60A80E098E79093AF0A8093AE0A80E557
:101EF00090E00E94AB2746E050E068E275E089E0A0
:101F000090E00E944D4084E693E09A8389831B828F
:101F10001C821D821E82CE0103960E94A3270E946E
:101F2000AA278091160690911706DC0192961D92C1
:101F30001D921D921C929597FC0116A217A210A645
:101F400011A69A961D921D921D921C929D9740EE8D
:101F50005EE260E070E046AB57AB60AF71AF40EA65
:101F60005FE060E070E0DA964D935D936D937C9353
:101F7000DD97189626E0FD01322F11923A95E9F788
:101F8000AC01425F5F4F34E1FA0111923A95E9F7F3
:101F9000E8E2F5E001900D922A95E1F7FC01EE5B95
:101FA000FF4F10820E944B3E8130910509F051C0D5
:101FB00080E590E00E94AB276091160670911706AD
:101FC000625F7F4FCE0101960E94B417CE01039647
:101FD0000E94A32760911606709117066A5E7F4FD4
:101FE000CE0101960E94B41744E050E0BE016D5F3F
:101FF0007F4F81E090E00E944D4060911606709105
:1020000017066E5E7F4FCE0101960E94B41744E022
:1020100050E0BE016D5F7F4F85E090E00E944D4033
:102020000E94AA276091160670911706625E7F4F84
:10203000CE0101960E94B4178B819C81AD81BE8137
:102040008093120690931306A0931406B09315067E
:102050001FC0892BE9F46DE577E081EC96E00E94E2
:10206000061786EF9FEF90934105809340050E94ED
:102070007153DC01CB01805A9541AF4FBF4F809324
:10208000030690930406A0930506B093060608C0C5
:102090000E94422D81E090E090934105809340059D
:1020A00099E288E10FB6F894A895809360000FBE7E
:1020B00090936000A895C7C060E070E080E090E079
:1020C0000E94B419BCC0A8951E8A0E9403208111E9
:1020D000BAC00091B40A1091B50A0115110509F4AE
:1020E000B2C0C8010E94631F682E712CF2E06F1607
:1020F00071040CF004C2A7C00E9471530091030642
:102100001091040620910506309106060617170760
:102110002807390708F04EC044E150E06CE57DE047
:102120008E010F5F1F4FC8010E94FA6769E574E0D6
:10213000C8010E944F65F80101900020E9F7CF0126
:10214000801B910B08968138910538F50E94032079
:10215000882319F18091E0079091E107019611F42D
:1021600081E090E09093E1078093E0078091E007A1
:102170009091E107909365078093660747E050E0F0
:1021800060E677E0C8010E94711FAC01455051091B
:1021900060E677E082EA0E94921F83E090E09093ED
:1021A0004105809340056FEB76E081EC96E00E945C
:1021B000061749C00E940320811145C082E090E0CB
:1021C0003EC00E94715300910306109104062091B5
:1021D000050630910606061717072807390798F5F0
:1021E00010924105109240052EC00E94715300913B
:1021F0000306109104062091050630910606061785
:10220000170728073907D0F21EC060E070E080E0B1
:1022100090E00E94163B892B89F60E947153DC01E5
:10222000CB0188579C4EAF4FBF4F809303069093CE
:102230000406A0930506B093060686EF9FEF9093E1
:102240004105809340050FB6F894A89580916000F1
:10225000886180936000109260000FBE80914005FD
:1022600090914105181619060CF024C1009116062C
:10227000109117060115110509F41CC10E94715334
:102280004B015C017801BEE3EB0EF11CF70180818C
:102290009181A281B381A5019401281B390B4A0BBE
:1022A0005B0BCA01B901683E33E0730781059105F4
:1022B00008F446C028EE33E040E050E00E94FF6E94
:1022C000861A970AA80AB90AD7018D929D92AD92F3
:1022D000BC921397F80186A597A5A0A9B1A9690199
:1022E0007A01CC0CDD1CEE1CFF1C8C159D05AE0587
:1022F000BF0528F416A617A610AA11AA09C0821BAA
:10230000930BA40BB50BF80186A797A7A0ABB1ABB5
:10231000F80182A993A9A4A9B5A98C159D05AE05BC
:10232000BF0528F412AA13AA14AA15AA09C0821B71
:10233000930BA40BB50BF80182AB93ABA4ABB5AB7D
:10234000F80186A597A5A0A9B1A9892B8A2B8B2B6B
:1023500069F4EE5BFF4F8081833041F484E0808339
:10236000C8010E944B3E01967C0102C0E12CF12C79
:10237000F80182A993A9A4A9B5A9892B8A2B8B2B33
:10238000A1F4EE5BFF4F8081833011F081110DC00D
:102390001082F8013E9684E1DF011D928A95E9F7EB
:1023A000C8010E944B3E03967C01B2E0EB16F1049B
:1023B00029F0E4E0EE16F10409F050C080E590E069
:1023C0000E94AB276091160670911706625F7F4FDF
:1023D000CE0101960E94B417CE0103960E94A32756
:1023E00060911606709117066A5E7F4FCE010196C6
:1023F0000E94B41744E050E0BE016D5F7F4F81E062
:1024000090E00E944D4060911606709117066E5E36
:102410007F4FCE0101960E94B41744E050E0BE0108
:102420006D5F7F4F85E090E00E944D400E94AA279B
:102430006091160670911706625E7F4FCE0101967D
:102440000E94B4178B819C81AD81BE81809312065E
:1024500090931306A0931406B0931506F2E0EF16BE
:10246000F10491F034F4EA94EF2821F56BEA76E078
:1024700010C043E0E416F10451F054E0E516F10415
:10248000C9F469E776E010C06BE976E00DC068E852
:1024900076E081EC96E00E94061786EF9FEF90931E
:1024A00041058093400506C081EC96E00E94061726
:1024B0000E94422D99E288E10FB6F894A895809386
:1024C00060000FBE9093600080914005909141059F
:1024D00066960FB6F894DEBF0FBECDBFDF91CF91E9
:1024E0001F910F91FF90EF90DF90CF90BF90AF9032
:1024F0009F908F907F906F905F904F90089560E0D5
:10250000C8010E94F01BDC011996AD90BC901A978F
:1025100061E0C8010E94F01BFC0181849284F2E01A
:102520006F16710409F4B2C162E0C8010E94F01B89
:10253000DC011996CD90DC901A97B3E06B1671040C
:1025400009F4A8C163E0C8010E94F01BFC01E1840A
:10255000F284F4E06F16710451F064E0C8010E9447
:10256000F01BDC0119960D911C911A9703C08E0186
:102570000A5E1F4F9092F4078092F307D092F607FD
:10258000C092F5076EE377E081EC96E00E94C015FB
:10259000B40181EC96E00E94B2176CE377E081EC25
:1025A00096E00E94C0154AE050E0B60181EC96E04A
:1025B0000E948C1665E377E081EC96E00E94C015DE
:1025C000B70181EC96E00E94B21760E377E081ECFE
:1025D00096E00E94C0150E9403208111E6C0609120
:1025E000F3077091F40780915E0790915F07409127
:1025F000F5075091F607DC01ED91FC91611571052D
:1026000021F00088F189E02D16C00684F785E02DC1
:1026100024E633E03A8329834090EF075090F00797
:102620006090F1077090F2074B825C826D827E822F
:10263000BE016F5F7F4F19958130910509F0AEC0E3
:102640009093E1078093E00787E0E0E5F2E0DE01A8
:10265000119601900D928A95E1F7FE013196A5E65B
:10266000B7E0CE01089621912D93E817F907D9F725
:10267000E114F10429F00115110521F082EC03C0E9
:1026800082E001C082E880936C0710926D078FE0B2
:1026900080936E074FE050E060E677E0C5010E944E
:1026A000711FE114F10479F0AC0160E677E0C70135
:1026B0000E94711F0115110531F0AC0160E677E051
:1026C000C8010E94711FAC014550510960E677E0D6
:1026D00080E10E94921F0E9471536093E207709301
:1026E000E3078093E4079093E5076093E607709310
:1026F000E7078093E8079093E90780915E07909140
:102700005F07DC01ED91FC910084F185E02D1995C6
:10271000892BC1F40E9471530091E6071091E707DD
:102720002091E8073091E907DC01CB01801B910B78
:10273000A20BB30B88399A43A105B105F0F28CEFD7
:102740009FEF1CC0CE0145960E94AB300497D1F498
:1027500080916307811111C00E9471536093E60755
:102760007093E7078093E8079093E9071092EA07D0
:102770001092FA071092F90718C090E09093FA07A8
:102780008093F90780915E0790915F07DC01ED91DE
:10279000FC910488F589E02D19954FC08EEF9FEFCD
:1027A0009093FA078093F90748C062E277E081ECE2
:1027B00096E00E94C015B50181EC96E00E94F416E7
:1027C00044E150E06CE57DE0CE0101960E94FA679D
:1027D00069E574E0CE0101960E944F65CE01019635
:1027E0000E94C93344E150E066E177E0CE010196F2
:1027F0000E94FA6769E574E0CE0101960E944F6578
:10280000CE0101960E94C93384E090E09093410587
:10281000809340050E947153DC01CB0188579C4E88
:10282000AF4FBF4F8093030690930406A093050615
:10283000B093060669EF76E0B8CC6DEE76E081ECF9
:1028400096E00E94C0156091F9077091FA074AE07E
:1028500050E081EC96E00E948C1665ED76E081EC0C
:1028600096E00E9406170E947153DC01CB01885745
:102870009C4EAF4FBF4F8093030690930406A093E6
:102880000506B093060684EF9FEFD9CC8BE5C82EE2
:1028900087E0D82E7E0126E1E20EF11C87016ACE88
:1028A000CF92DF92EF92FF920F931F93CF93DF931C
:1028B0006C017A018B01C0E0D0E0CE15DF0589F014
:1028C000D8016D918D01D601ED91FC910190F081BF
:1028D000E02DC6011995892B11F47E0102C02196C5
:1028E000ECCFC701DF91CF911F910F91FF90EF9037
:1028F000DF90CF900895FC01A089B1898C91A689C1
:10290000B78982FD0FC09C91818D8F5F8F73228D5F
:10291000821749F0218DDF01A20FB11D5D969C93B6
:10292000818F08958C910895FC01538D448D252F3E
:1029300030E0842F90E0821B930B541710F0CF9659
:10294000089501970895FC01918D828D981761F08B
:10295000828DDF01A80FB11D5D968C91928D9F5FD6
:102960009F73928F90E008958FEF9FEF0895FC0181
:10297000918D828D981731F0828DE80FF11D858D34
:1029800090E008958FEF9FEF0895FC01918D228DC7
:10299000892F90E0805C9F4F821B91098F7399274C
:1029A000089584E296E00E94C51421E0892B09F481
:1029B00020E0822F089581EC96E00E94C51421E06A
:1029C000892B09F420E0822F0895FC01848DDF011A
:1029D000A80FB11DA35ABF4F2C91848D90E0019692
:1029E0008F739927848FA689B7892C93A089B18981
:1029F0008C9180648C93938D848D981306C002888B
:102A0000F389E02D80818F7D80830895EF92FF927E
:102A10000F931F93CF93DF93EC0181E0888F9B8D01
:102A20008C8D981305C0E889F989808185FD24C0C3
:102A3000F62E0B8D10E00F5F1F4F0F731127E02E46
:102A40008C8DE8120CC00FB607FCFACFE889F98923
:102A5000808185FFF5CFCE010E94E514F1CF8B8DEB
:102A6000FE01E80FF11DE35AFF4FF0820B8FEA8958
:102A7000FB898081806207C0EE89FF896083E889D5
:102A8000F98980818064808381E090E0DF91CF913B
:102A90001F910F91FF90EF900895CF93DF93EC017A
:102AA000888D8823C9F0EA89FB89808185FD05C06E
:102AB000A889B9898C9186FD0FC00FB607FCF5CFA8
:102AC000808185FFF2CFA889B9898C9185FFEDCFF0
:102AD000CE010E94E514E7CFDF91CF91089580E009
:102AE00090E0892B21F00E94DB14811121C080E04D
:102AF00090E0892B41F080E090E0892B21F00E944A
:102B00000000811118C080E090E0892B21F00E9424
:102B1000D114811113C080E090E0892BA1F080E0F6
:102B200090E0892B81F00E94000081110AC0089575
:102B30000E940000DCCF0E940000E5CF0E94000050
:102B4000EACF0C9400000895A89508950E94FE64B1
:102B5000A8950E94A90E029714F00E9483310C944C
:102B6000345160E08DE00C94CB5261E08DE00C9428
:102B7000CB52DC01ED91FC910190F081E02D199494
:102B8000EF92FF920F931F93CF93DF938C017B0102
:102B9000C0E0D0E0F701EC0FFD1F6491662361F007
:102BA000D801ED91FC910190F081E02DC8011995BB
:102BB000892B11F02196EECFCE01DF91CF911F919D
:102BC0000F91FF90EF9008956115710579F0FB0169
:102BD00001900020E9F73197AF01461B570BDC014C
:102BE000ED91FC910280F381E02D199480E090E05A
:102BF00008954F925F926F927F92EF92FF920F93A0
:102C00001F93CF93DF93CDB7DEB7A1970FB6F8949C
:102C1000DEBF0FBECDBF7C01FA01CB0119A222306D
:102C200008F42AE08E010F5D1F4F422E512C612CBB
:102C3000712CBF01A30192010E94FF6EF901CA012C
:102C4000015011096A3014F4605D01C0695CD8015B
:102C50006C93232B242B252B61F7B801C7010E940D
:102C6000E415A1960FB6F894DEBF0FBECDBFDF917D
:102C7000CF911F910F91FF90EF907F906F905F9099
:102C80004F900895CF92DF92EF92FF920F931F9390
:102C9000CF93DF93EC016A017B012115310579F4B3
:102CA000E881F9810190F081E02D642FDF91CF91CF
:102CB0001F910F91FF90EF90DF90CF9019942A30E1
:102CC0003105E9F477FF1AC06DE20E94B9158C0155
:102CD00044275527BA014C195D096E097F092AE07E
:102CE000CE010E94F915800F911FDF91CF911F91A6
:102CF0000F91FF90EF90DF90CF9008952AE0B701F9
:102D0000A601CE01DF91CF911F910F91FF90EF901F
:102D1000DF90CF900C94F9159A01AB01770F660BF9
:102D2000770B0C9442168F929F92AF92BF92CF92E4
:102D3000DF92EF92FF920F931F93CF93DF937C016B
:102D40008B016C0182E0C80ED11C4701E5E08E0EBC
:102D5000911CC0E0D0E0F60141916F0150E060E0CD
:102D600070E02AE0C8010E94F9155C016EE2C8011A
:102D70000E94B9158A0D9B1DC80FD91FC814D9040C
:102D800051F7F701458150E060E070E02AE0C801AA
:102D90000E94F9158C0F9D1FDF91CF911F910F910C
:102DA000FF90EF90DF90CF90BF90AF909F908F906B
:102DB00008956AEE73E00C94E4150F931F93CF937C
:102DC000DF93EC019A01AB01770F660B770B0E9442
:102DD00042168C01CE010E94D916800F911FDF91FF
:102DE000CF911F910F9108950F931F93CF93DF936E
:102DF000EC010E94E4158C01CE010E94D916800FCF
:102E0000911FDF91CF911F910F9108950F931F9301
:102E1000CF93DF93EC010E94C0158C01CE010E947C
:102E2000D916800F911FDF91CF911F910F910895B7
:102E30000F931F93CF93DF93EB018DE295E09F9368
:102E40008F938CE295E09F938F938BE295E09F9315
:102E50008F938AE295E09F938F9389E295E09F9309
:102E60008F9388E295E09F938F938EE394E09F93F6
:102E70008F938B818F938A818F930E941A662DB7CF
:102E80003EB7205F3F4F0FB6F8943EBF0FBE2DBF39
:102E9000069784F460ED77E081EC96E00E94C0151F
:102EA0006A817B8181EC96E0DF91CF911F910F9138
:102EB0000C94F4160E941D2D08E215E0C0E0D0E04D
:102EC000F80161918F01CE010E94F16E2196C6300A
:102ED000D105B1F762EE77E081EC96E0DF91CF911A
:102EE0001F910F910C940617CF93DF93CDB7DEB7E8
:102EF0002C970FB6F894DEBF0FBECDBF1C821B828D
:102F00001E821D828FEF9FEF98878F838BE792E061
:102F10009A83898386E290E09A8789871C861B863C
:102F200066EB77E081EC96E00E9406176091070659
:102F300070910806CE0101960E947E356FEFCE019A
:102F400001960E94932166EA77E081EC96E00E9468
:102F500006172C960FB6F894DEBF0FBECDBFDF91DB
:102F6000CF9108950C94E41524E633E0FC013183FD
:102F70002083FB014081518162817381FC01428386
:102F800053836483758308951F920F920FB60F9237
:102F900011240BB60F922F933F934F935F936F9330
:102FA0007F938F939F93AF93BF93EF93FF9384E2AD
:102FB00096E00E94E514FF91EF91BF91AF919F9130
:102FC0008F917F916F915F914F913F912F910F90D2
:102FD0000BBE0F900FBE0F901F9018951F920F926F
:102FE0000FB60F9211240BB60F922F933F934F936E
:102FF0005F936F937F938F939F93AF93BF93EF9361
:10300000FF9384E296E00E947B14FF91EF91BF91C1
:10301000AF919F918F917F916F915F914F913F9170
:103020002F910F900BBE0F900FBE0F901F90189511
:103030001F920F920FB60F9211240BB60F922F937F
:103040003F934F935F936F937F938F939F93AF9330
:10305000BF93EF93FF9381EC96E00E94E514FF91FC
:10306000EF91BF91AF919F918F917F916F915F9100
:103070004F913F912F910F900BBE0F900FBE0F906D
:103080001F9018951F920F920FB60F9211240BB636
:103090000F922F933F934F935F936F937F938F93F1
:1030A0009F93AF93BF93EF93FF9381EC96E00E94C1
:1030B0007B14FF91EF91BF91AF919F918F917F9181
:1030C0006F915F914F913F912F910F900BBE0F9099
:1030D0000FBE0F901F901895CF92DF92EF92FF9244
:1030E0001F93CF93DF93EC016A017B01122FE889D4
:1030F000F98982E080834115514E61057105B1F077
:1031000060E079E08DE390E0A70196010E94FF6EF8
:10311000DA01C9010197A109B109B695A79597955B
:103120008795AC01411580E15807A8F0E889F98935
:10313000108260E874E88EE190E0A70196010E9499
:10314000FF6EBA01A90141505109610971097695D3
:10315000679557954795EC85FD855083EE85FF85EE
:103160004083188EEC89FD891083EA89FB89808170
:1031700080618083EA89FB89808188608083EA8915
:10318000FB89808180688083EA89FB8980818F7DCB
:103190008083DF91CF911F91FF90EF90DF90CF90D0
:1031A00008959FE9980F963010F429EA05C09FEB27
:1031B000980F963018F429EC280F05C090ED980F61
:1031C0009A3008F4292F822F08950F931F93CF93DD
:1031D000DF93282FDC01C42FD52F8A2F821B86175F
:1031E000D0F48D01ED91F0E084E0F595E7958A95B6
:1031F000E1F7E753FD4F808188832296CE01019746
:10320000F8013081E32FEF70F0E0E753FD4F30819C
:10321000FC013083E2CFFA01E60FF11DE60FF11D4C
:103220001082DF91CF911F910F910895CF93DF937B
:10323000CDB7DEB769970FB6F894DEBF0FBECDBF2E
:103240008FE290E0A0E0B0E089839A83AB83BC83F7
:10325000FE01359685E1DF011D928A95E9F762E965
:1032600077E081EC96E00E940617AE014E5F5F4F5B
:1032700066E088E295E00E94E5181E8663E574E04A
:10328000CE0101960E944F65BE016F5F7F4F81ECBA
:1032900096E00E94F416CE0101960E94C9331E8664
:1032A0006BE574E0CE0101960E944F65BE016F5F31
:1032B0007F4F81EC96E00E94F41665E674E0CE0143
:1032C00001960E94044B69960FB6F894DEBF0FBEBC
:1032D000CDBFDF91CF9108956BE479E081EC96E06A
:1032E0000E94C01563E479E081EC96E00E94061725
:1032F00067E379E081EC96E00E94061768E279E0E6
:1033000081EC96E00E94C0156CE179E081EC96E0DA
:103310000E94061766E079E081EC96E00E94C015F5
:1033200062EF78E081EC96E00E9406176EED78E09F
:1033300081EC96E00E94061760ED78E081EC96E063
:103340000E94061769EC78E081EC96E00E9406176F
:103350006FEB78E081EC96E00E94061766EB78E070
:1033600081EC96E00C940617AF92BF92CF92DF9259
:10337000EF92FF920F931F93CF93DF93CDB7DEB7FA
:10338000CA56D1090FB6F894DEBF0FBECDBF2CE0F0
:10339000E7E5F2E0DE01999601900D922A95E1F7BA
:1033A000FE01F59624E1DF011D922A95E9F78E01D1
:1033B000075D1F4F1816190644F4FB0162817381E3
:1033C0004FE150E0C8010E94936580912D051F9246
:1033D0008F9380912C051F928F9380912B051F92C4
:1033E0008F9380912A051F928F93809129051F92B8
:1033F0008F93809128051F928F9387E694E09F9387
:103400008F931F9288E28F93CE0101967C019F9348
:103410008F930E94AD6562EA78E081EC96E00E94AD
:10342000C015B80181EC96E00E94B217B70181EC9B
:1034300096E00E94F4160FB6F894A895809160006B
:10344000886180936000109260000FBE6E0199E465
:10345000C90ED11CD60113961C921E92129788EEAB
:1034600093E0A0E0B0E0F60184839583A683B78360
:1034700084E0848781E992E09183808316870587C1
:10348000108A178680E590E0928B818B158A6EE119
:1034900072E28AE993E20E9453688C010FB6F894B5
:1034A000DEBF0FBECDBF892B09F4B2C083E090E030
:1034B0000E944566D8011D969C938E931C97FC0133
:1034C000D182C0821282C6010E943E47882319F031
:1034D000C6010E946247D6011F966D917C9150975C
:1034E00051964D915C91529761157105C1F0CE01D5
:1034F000815A9F4FAA964FAFAA97AB965FAFAB97F3
:103500000E94B417AA964FADAA97AB965FADAB9742
:10351000BE01615A7F4FC6010E94222806C0F601F3
:1035200065857685C6010E9430271816190624F095
:10353000C8010E9478236CC0D6011D96BC901D97CF
:103540001E96AC90FF92EF928BE398E09F938F933F
:103550001F930F930E94DC68FF92EF9286E398E03E
:103560009F938F931F930F930E94DC68D8011C9642
:10357000ED91FC911D9781E08283FF92EF9283E3AE
:1035800098E09F938F931F930F930E94DC68D8015C
:103590001C96ED91FC911D971282AF92BF928DEF18
:1035A00097E09F938F931F930F930E94DC6888E3AB
:1035B00098E09F938F931F930F930E94DC68F6010E
:1035C000148A138AD8011C96ED91FC911D97A08056
:1035D000B1800FB6F894DEBF0FBECDBF83E3E82EF7
:1035E000F12CD501ED91FC910084F185E02DC50110
:1035F000199541970CF09BC0B1E0EB1AF10809F462
:1036000096C064E170E080E090E00E943753E9CF1B
:1036100000E010E0F601E388F48899E288E10FB653
:10362000F894A895809360000FBE909360000115F8
:10363000110509F45DC0F8ECEF16F10409F04AC079
:1036400067E978E081EC96E00E940617A3961FAE2A
:103650001EAEA397A5961FAE1EAEA5978FEF9FEF48
:10366000A7969FAF8EAFA79787EB92E0A1969FAFEB
:103670008EAFA197A9961FAF0EAFA99780910706AD
:10368000909108060E940F4BCE01815A9F4F0E94D5
:103690003A4B9093080680930706C8010E9478234E
:1036A0008091070690910806892B79F461E878E00B
:1036B00081EC96E00E9406170E947153DC01CB0159
:1036C0008856954CAF4FBF4F27C00E94BD3682E051
:1036D00090E067C069E678E081EC96E00E94C01552
:1036E0004AE050E0B70181EC96E00E94DD160CC084
:1036F00067E578E081EC96E00E9406176FE378E0DA
:1037000081EC96E00E9406170E947153DC01CB0108
:1037100088579C4EAF4FBF4F80930306909304068B
:10372000A0930506B093060685EF9FEF3AC07E0191
:10373000FFE5EF0EF11CFF92EF9281EF97E09F9370
:103740008F931F930F930E94F9680F900F900F9023
:103750000F900F900F90019709F05CCFF7018081D7
:103760009181D60154969C938E93539720E080E0EC
:103770008A3021F08D3031F0282F04C02A3009F42E
:1037800049CF2AE0C801AA962FAFAA970E949E6847
:10379000AA962FADAA978F3F59F7C8010E947823A8
:1037A00039CFC659DF4F0FB6F894DEBF0FBECDBF7D
:1037B000DF91CF911F910F91FF90EF90DF90CF900D
:1037C000BF90AF9008950C94B419882319F06AEE55
:1037D00077E002C06DEE77E081EC96E00C9406177E
:1037E000FC0186819781009739F0662329F06150AA
:1037F000FC0182819381F7CF08950F931F93CF939C
:10380000DF938B01FC01C681D781209759F0B80165
:10381000888199810E943C65892B21F00A80DB8197
:10382000C02DF3CFCE01DF91CF911F910F9108955D
:10383000CF93DF939B01672B61F4E091C106F09178
:10384000C2060190F081E02D682F81EC96E0199579
:1038500008C0482F50E060E070E081EC96E00E94E4
:10386000F915EC0181EC96E00E94D9168C0F9D1F92
:10387000DF91CF910895DC011696ED91FC91179799
:1038800061157105A1F0309729F417967C936E931A
:103890001697089582819381009711F0FC01FACF69
:1038A00073836283DB011596FC93EE93149708955E
:1038B000CF92DF92EF92FF920F931F93CF93DF93FC
:1038C0008C017B016A010E946C23EC01892B09F1B8
:1038D00082E08887A601DD0C660B770B49875A8743
:1038E0006B877C8788819981009711F00E94DA6646
:1038F000C7010E94036599838883BE01C801DF91D7
:10390000CF911F910F91FF90EF90DF90CF900C948B
:103910003B1CDF91CF911F910F91FF90EF90DF90B3
:10392000CF9008958F929F92AF92BF92CF92DF92E5
:10393000EF92FF920F931F93CF93DF93CDB7DEB734
:10394000C150D1400FB6F894DEBF0FBECDBF282FB7
:103950008091FD0789832A83213090F0253010F073
:10396000273171F48091FE079091FF079B838C8330
:1039700080910008909101089D838E8396E001C09C
:1039800092E08E010F5F1F4F213120F42F3030F471
:103990008BEF01C08AEE820F823078F4309182087A
:1039A00080918308F801E90FF11D808381E0890F80
:1039B000F801E80FF11D9E5F30832F3021F150F4A4
:1039C000253091F0263009F0B1C030918608809101
:1039D00087080EC0263109F48AC0273109F458C07F
:1039E000203109F0A3C054C030918408809185082B
:1039F000F801E90FF11D808381E0890FF801E80FDC
:103A0000F11D9E5F92C04091840850918508F80195
:103A1000E90FF11D508382E0890F31E0390FF80181
:103A2000E30FF11D4083BA0167707727A3E0569535
:103A30004795AA95E1F7672B19F031E0340F01C0E3
:103A4000342FB3E0B90FF801E80FF11D3083A4E083
:103A5000A90F60E070E04FEF4A0F6317B0F450E039
:103A6000CB0195958795400F511F880F991FFC0139
:103A7000EA57F74F60FD02C0808101C08181FA01E1
:103A800080836F5F7F4FAF5FE6CF9B2F930F4EC05A
:103A90003091840880918508F801E90FF11D808339
:103AA00081E0890FF801E80FF11D308363E0690FB1
:103AB0009E5FF801E90FF11D932F990F9083E6E8BF
:103AC000F8E0862F40E0431780F4708151813296F0
:103AD000D801A80FB11D5C9351E0580FD801A50F74
:103AE000B11D8E5F7C934F5FEECF960F1FC080910C
:103AF000860830918708F801E90FF11D308331E025
:103B0000390FF801E30FF11D80833091880880910F
:103B1000890842E0490FF801E40FF11D808383E03A
:103B2000890FF801E80FF11D9C5F30837801F801DF
:103B30004FEF5FEFD02E8E2F801B8917A0F481915D
:103B4000482768E070E0DA01B695A79540FF06C007
:103B5000AD0131E0432730EA532701C0AD01615088
:103B6000710989F7E8CFF801E90FF11D408332E0D0
:103B7000C32EC90E9F5FF801E90FF11D5083F801B4
:103B8000EC0DF11D10828091FB079091FC07DC0188
:103B9000ED91FC910284F385E02DCF5FDE4F288309
:103BA000C150D1401995CF5FDE4F2881C150D1401F
:103BB000019649F7E0911109F0911209309731F01F
:103BC0001995CF5FDE4F2881C150D140A091FB07EE
:103BD000B091FC079E2D9D199C1588F4F701619109
:103BE0007F01ED91FC9111970190F081E02DCD01C5
:103BF000CF5FDE4F2883C150D1401995E2CFED91C0
:103C0000FC9111970680F781E02DCD01CF5FDE4F4B
:103C10002883C150D1401995E0911309F0911409FE
:103C2000CF5FDE4F2881C150D140309731F01995D8
:103C3000CF5FDE4F2881C150D140CF5FDE4F288358
:103C4000C150D1400E9471534B015C0128E0D22E3B
:103C5000C12CCF5FDE4F2881C150D140E22EF12C24
:103C60008091FB079091FC07DC01ED91FC910084B1
:103C7000F185E02D1995892BC1F08091FB0790917A
:103C8000FC07DC01ED91FC910284F385E02D199590
:103C90009091FD07891711F0CC2099F1F801EC0DF6
:103CA000F11D8083DA94C39407C0E0910F09F0916D
:103CB0001009309709F01995B5E0CB1222C0EA81BE
:103CC0008E2F8F7790E08E159F0509F0A3C0E7FF38
:103CD00004C08B81882349F181C08E2F90E0FC01C4
:103CE0003197E731F10568F48827E755FF4F8F4F8B
:103CF0000C94116193E0D92E04C0DB8002C085E0F2
:103D0000D82E0E947153DC01CB0188199909AA09A8
:103D1000BB09813D9740A105B10508F0D2C0D11083
:103D20009FCFF4E0FC1508F079C0AFEFBFEF40E0A3
:103D3000D12CC6010297242F30E028173907C4F48C
:103D4000200F311FF9012081A22728E030E0BD01BA
:103D500076956795A0FF06C0DB01F1E0AF27F0EA9A
:103D6000BF2701C0DB012150310989F74F5FE3CF45
:103D7000800F911FFC0180818A134EC0F601EC0F69
:103D8000FD1F80818B1348C049C04034D8F4880F90
:103D9000991FFC01E550F84FA5E0B0E0AC0FBD1F46
:103DA000A80FB91F2C9130E0322F2227A4E0B0E0F9
:103DB000AC0FBD1FA80FB91F8C91D901A82BCD0145
:103DC00090878783242F4F5F842F90E08617970773
:103DD000E4F220930E0950FD61C080E010920809C2
:103DE00010920A091092090910920D09CF5FDE4F57
:103DF0000FB6F894DEBF0FBECDBFDF91CF911F91FC
:103E00000F91FF90EF90DF90CF90BF90AF909F9079
:103E10008F90089581EEE2CF83EEE0CF8A818530E6
:103E200028F4833028F4813080F5D7CF8731A9F684
:103E30008B8190E0AC015595479530910E0920E0BB
:103E4000822F90E084179507ECF42034C0F4FC0135
:103E50003296EE0FFF1F880F991FBC016550784FF7
:103E6000CE018E0F9F1FDC018C9190E0982F882748
:103E7000E00FF11F3081832BFB0190878783322F66
:103E80002F5FDECF30930E09A8CF5B81652F70E0E6
:103E90007595679520910E0940E096CF403468F4FF
:103EA000880F991FFC01E550F84FD801A80FB91FE2
:103EB00013968C9190E0908787834F5F40930E0913
:103EC0008CCF82EE8BCFDC011696ED91FC9117978B
:103ED00080E0309729F08F5F0280F381E02DF9CFE9
:103EE0000895CF93DF93DC014E5F5F4FFC019F018C
:103EF0002A1B3B0B9191992339F0EB01C40FD51F7D
:103F000098834F5F5F4FF3CFCA01821B930B680FFB
:103F1000791FFB013297308331962083CA01DF91EC
:103F2000CF910895CF92DF92EF92FF920F931F935C
:103F3000CF93DF9300D01F92CDB7DEB79A01E0E0B8
:103F4000922F9F77220F232F221F330B319521159C
:103F5000310509F0906801E00E0FA1E0B0E0AC0F70
:103F6000BD1FAE0FB11DFD0190832115310511F06C
:103F7000E02FE6CF10E0DB01A01BB10B14968C9371
:103F8000FE0131966F0180E090E08017910764F4A4
:103F9000F601F1906F019C01201B310B260F371F9A
:103FA000F901F5820196F1CF80915E0790915F074C
:103FB0004F5F5F4F040F151FFC0120813181F90114
:103FC00022813381A801BD01F90119957C010E946C
:103FD00071536093E2077093E3078093E407909333
:103FE000E50781E0E016F10609F080E00F900F9000
:103FF0000F900F90DF91CF911F910F91FF90EF9055
:10400000DF90CF90089580915E0790915F070097B1
:1040100059F1DC01ED91FC910688F789E02D1995A5
:10402000811124C08091F9079091FA07892BE1F45E
:104030008DEF9FEF9093FA078093F90780915E07C9
:1040400090915F07DC01ED91FC910680F781E02DF6
:10405000199580915E0790915F07DC01ED91FC91CD
:104060000488F589E02D199580E0089581E0089590
:10407000DF92EF92FF920F931F93CF93DF937C0118
:10408000D62E072FEA01122F0E9403208823E9F180
:10409000F70101900020E9F73197EE19FF09CE01F1
:1040A0000796E80FF91FE138F10578F545E050E093
:1040B00060E677E0C7010E94711FED2DF02F60E0F0
:1040C00070E06C177D0759F02191DB01A80FB91F33
:1040D000A25AB84F12962C936F5F7F4FF2CF655064
:1040E0007109112311F021E301C020E3AB01480F56
:1040F000591F60E677E0822FDF91CF911F910F91DA
:10410000FF90EF90DF900C94921F80E0DF91CF91B1
:104110001F910F91FF90EF90DF900895FB010190A8
:104120000020E9F73197AF01461B570B21E00C94B3
:104130003820FC01A285B3851097A9F08685978564
:10414000029788F0CD010196938782876C938685CC
:1041500097850197978786870284F385E02D1082E3
:1041600081E090E0089580E090E00895FC01868170
:1041700097818F3F2FEF920729F02FEF3FEF378383
:1041800026830895A085B185109789F0248535850B
:104190002115310561F0CD010196918780878C91C1
:1041A0002150310935872487082E000C990B08957A
:1041B000FC0186819781019639F481E0248535855B
:1041C000232B19F480E0089581E00895CF92DF92C7
:1041D000EF92FF920F931F93CF93DF937C016A01BD
:1041E0008B01C0E0D0E0CC15DD0589F0D701ED9161
:1041F000FC910284F385E02DC70119958F3FBFEF35
:104200009B0729F0F80181938F012196ECCFCE0115
:10421000DF91CF911F910F91FF90EF90DF90CF90A2
:104220000895CF93DF931F92CDB7DEB7DC01ED91F8
:10423000FC910088F189E02D69831995DC01ED91ED
:10424000FC910190F081E02D69810F90DF91CF9179
:104250001994CF93DF93FC01268137812F3F3F4F85
:10426000F9F4EC01288539858A859B85820F931F97
:104270008115904198F4E881F9810284F385E02D5D
:10428000CE011995813291056CF3E881F98106849C
:10429000F785E02D682FCE01199502C080E001C09E
:1042A00081E0DF91CF910895062E000C770BFC0181
:1042B000778366830895CF93DF93DC0116962D9163
:1042C0003C9117972F3F3F4F31F5EC01E881F98181
:1042D0000088F189E02DCE011995DC01ED91FC916A
:1042E0000084F185E02D1995892B99F0E881F981F9
:1042F0000284F385E02DCE0119958132910534F3C6
:10430000E881F9810684F785E02D682FCE011995A3
:1043100002C080E001C081E0DF91CF910895FC01EF
:10432000848195810895FC0120853185828593855E
:10433000AC014F5F5F4F53874287820F931F0E94EC
:10434000F16E81E090E00895FC01868197818F3FB6
:104350002FEF920729F02FEF3FEF37832683089541
:104360002085318582859385AC014F5F5F4F5387F0
:104370004287820F931F0E94E96E082E000C990B52
:104380000895FC01868197818F3F2FEF920729F0D6
:104390002FEF3FEF378326830895808591850C9416
:1043A0009E68CF92DF92EF92FF92CF93DF93EC0162
:1043B0008E819F818F3F2FEF920759F02FEF3FEFB4
:1043C0003F832E83DF91CF91FF90EF90DF90CF90CE
:1043D00008950E9471536B017C01A4EFCA0EA1E005
:1043E000DA1EE11CF11CE881F9810088F189E02DD9
:1043F000CE011995DC01ED91FC910084F185E02D51
:104400001995892B39F40E9471536C157D058E0521
:104410009F0548F3E881F9810088F189E02DCE01FC
:104420001995DC01ED91FC910284F385E02DDF917B
:10443000CF91FF90EF90DF90CF901994EF92FF9281
:104440000F931F93CF93DF93009719F48FEF9FEF94
:1044500086C0FC01E484F584D7010D911C91D8013C
:10446000ED91FC910688F789E02DC8011995882304
:1044700069F3D801ED91FC910084F185E02DC8012C
:104480001995D801ED91FC91892B61F30284F38594
:10449000E02DC8011995EC010196C1F2F80185895A
:1044A000882349F04C2F50E060E070E02AE081EC76
:1044B00096E00E94F915D70112968C91882309F491
:1044C0004DC0C532D10509F049C0D801ED91FC912C
:1044D0000084F185E02DC801199502975CF0D801A0
:1044E000ED91FC910688F789E02DC801199581119D
:1044F000ECCFACCFD1E0C0E0D801ED91FC910284CB
:10450000F385E02DC80119958F3FBFEF9B0709F494
:104510009DCF9C01215431092A31310530F09C0195
:10452000215631092A31310538F48D2F8295807F4B
:10453000829FC00D11240AC0C0978A30910530F4C3
:104540009D2F9295907F989FC00D1124DD2311F02F
:10455000D0E0D2CF8C2FCC0F990B01C0CE01DF91D0
:10456000CF911F910F91FF90EF900895EF92FF92DE
:104570000F931F93CF93DF938C017B01DC01ED91AF
:10458000FC910284F385E02D1995829749F584E02A
:10459000F701808786E090E00E944566EC01892B58
:1045A000F9F0E3E8F9E0F983E88380E091E0DF01E6
:1045B0009C011D9221503040E1F79B838A831D822C
:1045C0001C82D801ED91FC910284F385E02DC80195
:1045D00019958F3FBFEF9B0731F4CE010E94DA6639
:1045E0008FEF9FEF72C08232910509F44AC080328A
:1045F00091050CF446C08C35910511F0BE013EC00A
:10460000D801ED91FC910284F385E02DC801199544
:104610008F3FBFEF9B0709F38236910539F15CF4B8
:104620008F32910501F18C359105D1F0829749F6D1
:10463000BE0182E223C08E369105D9F03CF4863665
:10464000910509F0BECFBE018CE018C082379105FC
:1046500099F08437910509F0B4CFBE0189E00EC00E
:10466000BE018CE50BC0BE018FE208C0BE0188E030
:1046700005C0BE018AE002C0BE018DE00E9469351E
:10468000A0CF8C819D81009749F0E881F9818E0F40
:104690009F1FFC0131978081882321F0BE0180E0BB
:1046A0000E9469358C819D810E9445668C0100972E
:1046B00039F063E879E00E946E65CE010E94DA6607
:1046C000F7011287018780E090E0DF91CF911F9181
:1046D0000F91FF90EF9008958DE090E00E94456665
:1046E000009729F02DE0FC0111922A95E9F7089531
:1046F0000F931F93CF93DF930097B9F0EC010C85D4
:104700001D85D8018D919C91DC01ED91FC9104886F
:10471000F589E02D1995C8010E94DA66CE01DF9176
:10472000CF911F910F910C943C68DF91CF911F9115
:104730000F910895AF92BF92CF92DF92EF92FF92C6
:104740000F931F93CF93DF9300D01F92CDB7DEB7A7
:104750006115710509F494C06B01182FDB011C96DB
:10476000AD90BC901D97F501E080F180D701ED91EF
:10477000FC910688F789E02DC7011995811104C0C5
:10478000C6010E9478237CC0F5019281911114C06A
:10479000D701ED91FC910190F081E02D612FC701CF
:1047A0001995F7018589882309F467C0612F81EC89
:1047B00096E00E94B91561C0812F8F7D81548A31A6
:1047C00038F380ED810F8A3018F383ED810F82304A
:1047D000F8F21F35E9F21E37D9F21132B1F086EC4A
:1047E000810F823090F08AED810F873070F01D3399
:1047F00061F0812F8F7E8F3241F08DED810F8230FD
:1048000020F01B3511F01D3511F491FFC1CF198235
:104810001A821B821C82812F012E000C990B9F9300
:104820001F9382E994E09F938F938E010F5F1F4F38
:104830001F930F930E94EA650F900F900F900F90B7
:104840000F900F9083E0D82ED00ED701ED91FC9100
:104850000190F081E02DD8016C91C7011995F70105
:104860008589882331F0D8016C9181EC96E00E9413
:10487000B9150F5F1F4FD012E8CF80E090E002C063
:104880008FEF9FEF0F900F900F900F90DF91CF91D0
:104890001F910F91FF90EF90DF90CF90BF90AF905E
:1048A00008952F923F924F925F926F927F928F92D4
:1048B0009F92AF92BF92CF92DF92EF92FF920F93AF
:1048C0001F93CF93DF93CDB7DEB765970FB6F894FC
:1048D000DEBF0FBECDBF7C016B013A01FB0120E0C2
:1048E00080E090E06AE03191332309F140ED430F1D
:1048F0004A3080F4689FA001699F500D1124CA01BD
:10490000C097830F911D37FD9A958F3F910559F3FD
:1049100050F313C03E3289F4233079F0D301A20F53
:10492000B11D12968C932F5F80E090E0DCCF233096
:1049300021F4F301858381E021C0F7014281538195
:104940006481758180910C0690910D06A0910E06F0
:10495000B0910F06481759076A077B0709F49EC1F3
:104960000E9471538701085F1F4F6F7077277C5F2C
:10497000C8010E940646813019F080E090E0F3C142
:1049800084E693E09A838983F70182819381A481ED
:10499000B5818B839C83AD83BE8345E350E0BE012C
:1049A0006F5F7F4FC8010E94F646892B19F4C12C16
:1049B000D12C6FC10E947153F701778366837627EC
:1049C000672776277A83698342E050E0BE016F5FF4
:1049D0007F4FC8010E94474D81E090E09E878D8700
:1049E00042E050E0BE01635F7F4FC8010E94474D27
:1049F00080E091E09E878D8742E050E0BE01635FDA
:104A00007F4FC8010E94474D1E861D8642E050E040
:104A1000BE01635F7F4FC8010E94474D42E050E0F6
:104A2000BE01635F7F4FC8010E94474D42E050E0E6
:104A3000BE01635F7F4FC8010E94474D5601F501DB
:104A40008081882311F1F6015F018191811115C0E8
:104A500045018C189D081814190494F48F8641E0C0
:104A600050E0BE01615F7F4FC8010E94474DA40125
:104A7000B601C8010E94474D03C08E3229F7E8CF26
:104A80006501FFEFCF1ADF0ADACF1F8641E050E061
:104A9000BE01615F7F4FC8010E94474DC12CDD24DC
:104AA000D394DE86CD8642E050E0BE01635F7F4F47
:104AB000C8010E94474DDE86CD8642E050E0BE012F
:104AC000635F7F4FC8010E94474DC8010E94AD46F9
:104AD000892B09F46CCF63E0A62EB12CF2E06F0EA7
:104AE000711C0E9471531B012C01C8010E943C4E95
:104AF00018161906A4F00E947153DC01CB0182192B
:104B00009309A409B509813A9F40A105B105D0F4E4
:104B100062E370E080E090E00E943753E6CFF70157
:104B20004281538164817581808D918DA28DB38D79
:104B3000481759076A077B0741F4848D958DC597FF
:104B400021F406C02FEF3FEF9AC02EEF3FEF97C042
:104B5000F70181A192A10C970CF4A6C04CE050E0A3
:104B6000BE016F5F7F4FC8010E94F44D8B8190E0C2
:104B7000982F88272C81822B9A8B898B298130E072
:104B8000322F22274A81242BF70146815781421771
:104B9000530709F086C097FF84C08F709270892BED
:104BA00009F0DEC0CF80D12CDC2CCC248885C82A2B
:104BB000C114D10409F4D1C0812C912C8D8190E0D5
:104BC000982F88272E81822B8816990608F46FC0AB
:104BD000812C912C41E050E0BE016D5E7F4FC801F9
:104BE0000E94F44D8B89982F907C09F093C081111D
:104BF00086C08B898111EECF42E050E0BE01615F3B
:104C00007F4FC8010E94F44D42E050E0BE01635F57
:104C10007F4FC8010E94F44DC8010E94134EC80185
:104C20000E94134EC8010E94134EC8010E94134EE9
:104C300042E050E0BE016F5E7F4FC8010E94F44D1C
:104C40008F8598898115914009F069C02D853E8531
:104C50003227232732272130310509F060C08989A6
:104C60009A898115944009F075C044E050E0B30181
:104C7000C8012C8B3D8B0E94F44D2C893D89690124
:104C8000F1E0AF1AB10829F02FEFC216D20609F4ED
:104C900028CFC8010E94F145C60165C08EEF9FEF85
:104CA00062C02CEF3FEFEBCF2DEF3FEFE8CF41E0BD
:104CB00050E0BE01635F7F4FC8010E94F44D8D85B7
:104CC000811113C08D858111F2CFC8010E94134E4E
:104CD000C8010E94134EC8010E94134EC8010E94D1
:104CE000134EFFEF8F1A9F0A69CF8D859FEF980FA4
:104CF0009D87882339F3C8010E94134EF6CF8B8914
:104D00009FEF980F9B8B882309F473CFC8010E94F3
:104D1000134EF5CFC8010E94134E1B8A6ACF412C57
:104D2000512C89899A8998278927982748165906E6
:104D300038F4C8010E94134E8FEF481A580AF1CF79
:104D4000EFEF8E1A9E0A8C149D0409F043CF26EFD4
:104D50003FEF95CF27EF3FEF92CF2AEF3FEF8FCF77
:104D60002BEF3FEF8CCF65960FB6F894DEBF0FBEEA
:104D7000CDBFDF91CF911F910F91FF90EF90DF900A
:104D8000CF90BF90AF909F908F907F906F905F90EB
:104D90004F903F902F90089580E3FB0180833296DF
:104DA000842F82958F7090E1899F401911244A3099
:104DB00014F4405D01C0495C4293482F8111F0CF4B
:104DC0000895CF93DF931F92CDB7DEB76983DC01DF
:104DD000ED91FC910280F381E02D41E050E0BE01B5
:104DE0006F5F7F4F19950F90DF91CF910895DC0190
:104DF000ED91FC91068CF78DE02D199591E08927B6
:104E00000895862F089581E086270895CF93DF9334
:104E10001F92CDB7DEB789832091840A3981E09152
:104E2000850AF091860A822F90E080959095F894FB
:104E30000080082200824BE000C05DE000005A952F
:104E4000E9F7008008220894379508F4022A0082C6
:104E50004A9599F778940F90DF91CF91089508952E
:104E6000CF92DF92EF92FF920F931F93CF93DF9336
:104E7000CDB7DEB7AF970FB6F894DEBF0FBECDBF8C
:104E80007C016A0104E613E01A8309831C861B86F1
:104E900088EE93E0A0E0B0E08D879E87AF87B88B67
:104EA00088E993E09A878987188F0F8B198E1A8E5D
:104EB0001B8E1C8E84E089A31DA30CA31EA21FA21F
:104EC00018A619A68091120690911306A0911406B7
:104ED000B09115068CA79DA7AEA7BFA78B839C8317
:104EE000AD83BE8318861F82AE014C5D5F4FCE013D
:104EF00001960E94512481309105B1F4D701ED91C2
:104F0000FC910684F785E02D1BA70AA78EA19FA11F
:104F1000A8A5B9A58CA79DA7AEA7BFA7A601BE014E
:104F2000665D7F4FC7011995AF960FB6F894DEBF47
:104F30000FBECDBFDF91CF911F910F91FF90EF90EA
:104F4000DF90CF90089544E050E0BC018FE090E006
:104F50000C944D4008958CBD9DBD08958F929F92F5
:104F6000AF92BF92CF92DF92EF92FF920F931F9377
:104F7000CF936C015B017A01FC01C485C43041F41C
:104F800081E090E0F6019383828380E090E04EC060
:104F90008A014130584010F000E018E080E590E0D0
:104FA0000E94AB278C2F0E94AD334C0163E070E070
:104FB0008C2F0E948746873111F08C3121F48016A6
:104FC000910660F302C000E010E080E590E00E94EE
:104FD000AB279801A50160E070E08C2F0E94483358
:104FE00060E270E08C2F0E94D03262E070E08C2F83
:104FF0000E94874684FD10C063E070E08C2F0E9401
:105000008746811104C08C2F0E94954EB9CF80E550
:1050100090E00E94AB27E9CF40E162E070E08C2F86
:105020000E947D46012B09F4ABCFC701CF911F91A0
:105030000F91FF90EF90DF90CF90BF90AF909F9037
:105040008F900895CF92DF92EF92FF920F931F936C
:10505000CF93DF93FC012485243009F07FC06A01DF
:105060008B01EC01F12C8F2D0E94A94E811102C001
:10507000FC8607C08B7F8831D9F3F394F4E0FF12EC
:10508000F2CF8C85843009F469C0209103023091FD
:1050900004022F5F3F4F11F420E030EC3093040204
:1050A00020930302409103025091040220E061E04A
:1050B0000E949F40FC84F80182818F3F51F48381DC
:1050C0008F3F99F484818F3F81F485818F3F69F40C
:1050D00043C081110AC0F8018381811106C0848117
:1050E000811103C085818823B9F1C114D104A1F1D4
:1050F00080E590E00E94AB27B8016E5F7F4F8F2D57
:1051000090E0982F882744E050E0845F9B4F0E94F6
:105110004D40B6018F2D0E94E54664E070E08F2D72
:105120000E94D0320E9471536B017C01F4E9CF0ED2
:10513000F1E1DF1EE11CF11CCE010E9436478731F0
:1051400059F161E070E080E090E00E943753CE01B9
:105150000E943647811105C084E08C8780E090E092
:105160001DC00E947153C616D706E806F90620F73F
:105170008C850E94954EEC85F0E0EE0FFF1FE95DF7
:10518000F44F1182108284E08C8763E17AE081EC35
:1051900096E00E940617E2CF81E090E0DF91CF9188
:1051A0001F910F91FF90EF90DF90CF90089578942A
:1051B0001F920F920FB60F9211240BB60F92CF923F
:1051C000DF92EF92FF920F931F932F933F934F9392
:1051D0005F936F937F938F939F93AF93BF93CF937F
:1051E000DF93EF93FF93809170008E7F8093700028
:1051F0000FE310E08BE1E82EF12C9BE2C92ED12CBD
:10520000C091870AD091880A2097F9F403321105DA
:1052100008F43BC003521109E091850AF091860A17
:1052200090818091840A282F2095922390839BE07F
:10523000D7011197F1F79150D9F79081892B80838D
:10524000C6010197F1F780E00DC00B301105E8F0C1
:105250000B501109E091890AF0918A0AEC0FFD1FA9
:10526000319780810E9406272196D093880AC093A7
:10527000870A80910102909102028C179D0708F025
:10528000BFCF1092880A1092870A809170008160C7
:1052900080937000FF91EF91DF91CF91BF91AF911B
:1052A0009F918F917F916F915F914F913F912F913E
:1052B0001F910F91FF90EF90DF90CF900F900BBE5A
:1052C0000F900FBE0F901F90189581E08093830A76
:1052D00080910002282F30E0F901E353F64FE4916A
:1052E000F0E0EE0FFF1FED54F64F459154915093AF
:1052F000860A4093850AF901E359F64FE491E09359
:10530000840A61E00E94FB5283E08093B100E0E7F1
:10531000F0E08081816080830895CF93DF93181639
:10532000190644F0809170008E7F80937000109277
:10533000830A19C0EC018091890A90918A0A0E941F
:10534000DA66CE01C130D24014F080E092E0909352
:105350000202809301020E94456690938A0A80931C
:10536000890A892B29F4109202021092010208C0C6
:105370008091830A811104C0DF91CF910C9465293B
:10538000DF91CF910895EF92FF921F93CF93DF9318
:105390001F921F92CDB7DEB7162F2091830A2111DD
:1053A00006C089839A830E9465299A8189817C013C
:1053B00021E0E21AF108E114E2E0FE0698F42091FF
:1053C0000102309102022817390710F40E948D293A
:1053D0008091890A90918A0A009721F08E0D9F1D75
:1053E000FC0110830F900F90DF91CF911F91FF90E0
:1053F000EF900895CF93DF93CDB7DEB729970FB61F
:10540000F894DEBF0FBECDBFAE014F5F5F4F0E946D
:105410004741882389F08D818F3361F020F48F31EB
:1054200059F489E00CC08F3519F08F3739F004C07A
:105430008BE005C08AE003C080E001C08CE02996C3
:105440000FB6F894DEBF0FBECDBFDF91CF910895A8
:10545000AF92BF92CF92DF92EF92FF920F931F9382
:10546000CF93DF931F921F92CDB7DEB77C018A01E5
:10547000FC018581968169837A830E944942698112
:105480007A818823D1F1F701858196810E94744346
:1054900040E06EEBF701858196810E948A425801B7
:1054A0006801F9E0CF0ED11CF70105811681C80112
:1054B0000E94CE41C8010E94AB4166E988E196E0B6
:1054C0000E947352C8010E94A841C8010E94CE41A7
:1054D00061EEC8010E94B741C8010E945A41F5011E
:1054E00081935F01EC15FD05F9F6F7018581968141
:1054F0000E94494291E0813009F090E0892F0F909D
:105500000F90DF91CF911F910F91FF90EF90DF905F
:10551000CF90BF90AF900895089580E090E00895F7
:105520004F925F926F927F928F929F92AF92BF92B3
:10553000CF92DF92EF92FF920F931F93CF93DF935F
:10554000CDB7DEB7A9970FB6F894DEBF0FBECDBFBB
:105550004C018B017B01E40EF51ED7011C926DE717
:105560007AE081EC96E00E94C015B40181EC96E0EF
:105570000E94B2176AE77AE081EC96E00E94C015BB
:10558000FE0131965F0120918B0B30918C0B211520
:10559000310511F425E93BE0C501821B930B8A3FDD
:1055A000910514F0680103C065E77AE02BC0CE14C2
:1055B000DF0441F0D6016D916D0181EC96E00E940F
:1055C000B915F5CF81EC96E00E94D916FF24F3942B
:1055D0008091400590914105049709F0F12C45E137
:1055E00050E066E177E0C5010E94FA674BE050E0C9
:1055F000B501C4010E948565FF2049F0892B39F46B
:105600006AE67AE081EC96E00E940617FFC11982F3
:105610001A821B821C82FE01359680E1DF011D92F9
:105620008A95E9F7C8010E94E7506C016FE270E0CB
:10563000C4010E94A265009741F0BC016F5F7F4FDB
:1056400043E150E0C5010E949365B501CE01469645
:105650000E94CD50CE0146960E94F24F882309F455
:10566000D5C18E8D873011F4F110D0C1BFEFCB16AC
:10567000DB0609F064F4EEEFCE16EFEFDE060CF079
:10568000C5C1FDEFCF16FFEFDF06F1F1B4C1C114C4
:10569000D10471F021E0C216D10409F0ACC101E0DF
:1056A0000F2520E030E040E050E061E070E0AAC16A
:1056B0005E013FE1A30EB11CC12CD12C9501011557
:1056C0001105F1F0B3E0CB16D104D1F08FEFC81A79
:1056D000D80AC80128A739A70E94CC674C016CE200
:1056E00070E0C8010E945A658C0128A539A5892B54
:1056F00011F00F5F1F4FD5018D929D925D01DFCF9D
:1057000001E00F25A60174C1CE0185969E01295D99
:105710003F4F3F932F93215031093F932F939F93F6
:105720008F9388E994E09F938F931F930F930E9428
:105730001A660FB6F894DEBF0FBECDBF039709F00F
:1057400065C11DA17EA18FA1E72E171708F4E12ED8
:105750008E1508F4E82E1E19D72EDE18C82ECE1886
:105760009E2D90959F3F39F080E090950E94C65104
:10577000082F009501C00FEF8D2D90E0810F911D36
:105780008C0D911D892B29F4E02EE09400E070E04F
:1057900000C10F3FF1F0011101C001E0802E912CFA
:1057A000A12CB12C6FEF7FEF80E090E0A501940178
:1057B0000E94216FA12FB0E00E94406F172FAD2DE6
:1057C000B0E00E94406FD72EAC2DB0E00E94406F39
:1057D000C72EAD2CB12CA10EB11CAC0CB11CFFEF2F
:1057E000AF16B1040CF5A114B10419F4AA24A394C2
:1057F000B12C2501612C712C6FEF7FEF80E090E0E0
:10580000A30192010E94216FA12FB0E00E94406F7E
:10581000172FAD2DB0E00E94406FD72EAC2DB0E019
:105820000E94406FC72E05C02FEFA216B10409F0E9
:105830006CF43E2D2A2D320F08F43FEF932F3F3F9B
:1058400029F080E00E94C651E82E02C0EE24EA94BE
:10585000812F1D1508F48D2D8C1508F48C2D8113C6
:105860002FC0D1100DC0782F20E8721B08F470E013
:1058700020E6729F070E70E0711D1124705388C0DE
:105880002D2D30E0482F50E0421B530B24173507D5
:1058900044F47D2D20E6729F070E70E0711D1124E7
:1058A00077C076E57D0D781B24E0721B08F470E06C
:1058B00020E6729F070E70E0711D1124705E68C0B3
:1058C0008D113AC0C1101BC02BEA722F711B08F456
:1058D00070E0172F3FE2139F010E10E0111D1124FD
:1058E000382F321B08F430E0732F20E6729F070E2A
:1058F00070E0711D1124710F7695705C49C02C2DDC
:1059000030E090E0821B930B7C2D2817390744F47C
:1059100020E6729F070E70E0711D1124705A38C086
:1059200025E5721B08F470E020E3729F070E70E01B
:10593000711D112470582CC011110DC07C2D20E850
:10594000721B08F470E020E3729F070E70E0711D77
:10595000112478571DC0212F30E08C2D90E0821B40
:10596000930B712F2817390744F420E6729F070E16
:1059700070E0711D112470560BC025E5721B08F4F0
:1059800070E020E6729F070E70E0711D11247054C4
:105990007F5F272F30E0ADE6B1E00E94536F812C8E
:1059A000912C54018A94A50194010E94216F38A37F
:1059B0002F8F202F30E0A4E6B0E00E94536FA501A6
:1059C00094010E94216F3AA329A32E2D30E0A4E672
:1059D000B0E00E94536FA50194010E94216F3CA387
:1059E0002BA301E00F259E01215E3F4F43E050E0D5
:1059F00060E070E007C001E00F2520E030E040E00B
:105A000050E0B601CE0146960E946607A9960FB6F1
:105A1000F894DEBF0FBECDBFDF91CF911F910F91E4
:105A2000FF90EF90DF90CF90BF90AF909F908F90BE
:105A30007F906F905F904F9008951F93CF93DF9367
:105A400064E97AE081EC96E00E94C015C8E2D5E0F6
:105A50001C2F1A5F499150E060E070E020E181EC7A
:105A600096E00E94F91562E97AE081EC96E00E94E6
:105A7000C0151C13EFCF81EC96E0DF91CF911F9101
:105A80000C94D916AF92BF92CF92DF92EF92FF9211
:105A90000F931F93CF93DF9300D000D0CDB7DEB725
:105AA00062E87AE081EC96E00E94C0158E010D5FFD
:105AB0001F4F7E0187E0E80EF11C580184E6C82ED6
:105AC00083E0D82EDA82C9821B821C821D821E824C
:105AD00080E590E00E94AB2744E050E0B5018FE004
:105AE00090E00E941D400E94AA27F80141918F0179
:105AF00050E060E070E02AE081EC96E00E94F91549
:105B000060E87AE081EC96E00E94C0150E151F0552
:105B1000C9F681EC96E00E94D91626960FB6F89445
:105B2000DEBF0FBECDBFDF91CF911F910F91FF90D0
:105B3000EF90DF90CF90BF90AF9008955F926F92FB
:105B40007F928F929F92AF92BF92CF92DF92EF920D
:105B5000FF920F931F93CF93DF93CDB7DEB7E497F8
:105B60000FB6F894DEBF0FBECDBF5C017B016A01AA
:105B7000890119A21AA21BA21CA2FE01B5968CE0F3
:105B8000DF011D928A95E9F761E975E0CE01019682
:105B90000E94F367D5011296ED91FC9113976081F5
:105BA000718140E250E0CE0101960E947565B2E03D
:105BB000EB16F104A1F054F4E114F104B9F0EA9405
:105BC000EF2809F058C067E374E00BC085E0E816E1
:105BD000F10429F099E0E916F10441F04CC06AE3C0
:105BE00074E0CE0181960E946E654EC001151105CC
:105BF00009F44AC0612C712C83EAA82E84E0B82EE7
:105C000094E0592E7E01A1E3EA0EF11C4601B1E0B9
:105C10008B1A91086C147D04BCF5F8018081918188
:105C20000E5F1F4F9F938F93BF92AF921F925F9211
:105C3000FF92EF920E94AD6540E150E0B701CE01C6
:105C400081960E9475650FB6F894DEBF0FBECDBF7A
:105C50006814790461F066EA74E0C7010E946E6519
:105C600040E150E0B701CE0181960E9475659FEF3B
:105C7000691A790ACFCF6DE57AE081EC96E00E944F
:105C800006178FEF9FEF23C067E57AE081EC96E07F
:105C90000E94C015BE016F5F7F4F81EC96E00E94AD
:105CA000B21764E57AE081EC96E00E94C015BE016F
:105CB0006F5D7F4F81EC96E00E94F416BE016F5D30
:105CC0007F4FCE0101960E948E2080E090E0E49606
:105CD0000FB6F894DEBF0FBECDBFDF91CF911F91FD
:105CE0000F91FF90EF90DF90CF90BF90AF909F907B
:105CF0008F907F906F905F900895EF92FF920F9337
:105D00001F93CF93DF9300D000D0CDB7DEB78C01C7
:105D10000E945E5085FF40C0E82EF12CC8010E9411
:105D20000E50A62F372F282FF801408550E04A301B
:105D3000510528F5FA018827E054FF4F8F4F0C9446
:105D40001161A9833A83022E000C330B3C832B8311
:105D5000892F990F990B9E838D839E012F5F3F4F53
:105D600043E050E009C08A2F932F9A8389839E01D4
:105D70002F5F3F4F41E050E060E070E005C020E061
:105D800030E040E050E0B701C8010E949E2DB7010D
:105D90006F7DC8010E94495026960FB6F894DEBF69
:105DA0000FBECDBFDF91CF911F910F91FF90EF906C
:105DB0000895EF92FF920F931F93CF93DF9300D03C
:105DC00000D0CDB7DEB78C017B0162E070E00E94AD
:105DD0003250892B19F4E982FA8205C08F2D880F81
:105DE000880BF9828A83A981BA81BB2724E630E037
:105DF0000E9420612FE330E040E050E00E94216FDC
:105E00003A832983C8012B833C834D835E830E94A0
:105E10005E50E82EF12CC8010E940E502B813C816F
:105E20004D815E81621773078407950779F4672BAC
:105E3000682B692B09F44DC082E0E816F10471F07B
:105E400085E0E816F10409F044C008C0232B242B98
:105E5000252B51F182E0E816F10409F520E030E04D
:105E600040E050E061E070E0C8010E949E2D9E017C
:105E70002F5F3F4F41E050E060E070E0C8010E94BA
:105E80009E2D61E0C8010E94495049815A81052E2A
:105E9000000C660B770BC8010E94FF4F1AC085E00B
:105EA000E816F10421F7DACF85E0E816F10489F06D
:105EB00082E0E816F10469F062E0C8010E944950EE
:105EC00020E030E040E050E062E070E0C8010E9475
:105ED0009E2D80E090E026960FB6F894DEBF0FBEB0
:105EE000CDBFDF91CF911F910F91FF90EF9008955B
:105EF000EF92FF920F931F93CF93DF931F921F9206
:105F0000CDB7DEB77C010E945E50182F86FF1EC001
:105F1000C7010E940E507A83698367E37AE081ECBF
:105F200096E00E940617612F70E0D701ED91FC9179
:105F30006F7B0190F081E02D01E09E012F5F3F4FCC
:105F400041E050E0C701199581E001C080E00F9069
:105F50000F90DF91CF911F910F91FF90EF900895D7
:105F6000FF920F931F93CF93DF93CDB7DEB729979F
:105F70000FB6F894DEBF0FBECDBF8C010E94F24F6A
:105F8000882309F473C0C8010E945E50D801189696
:105F9000FC90B7E0FB1649F0823009F449C0853027
:105FA00009F446C0813009F46AC0C8010E940E504D
:105FB000362F272F4F2D50E04A30510508F041C0B1
:105FC000FA018827E653FF4F8F4F0C941161D801D7
:105FD0001496ED91FC9115978085853091F56BE2D3
:105FE0007AE081EC96E00E940617D8011496ED91B4
:105FF000FC9115970681178101151105C9F0F8016B
:1060000061857285CE0101960E94CD50CE01019628
:106010000E94F24F882331F0CE0101960E94B02FEA
:10602000892B39F5D80112960D911C911397E4CF65
:1060300080E026C0092F990F110B05C0032F122FE6
:1060400002C000E010E061E27AE081EC96E00E949C
:10605000C0154AE050E0B80181EC96E00E94DD16E0
:1060600081E090E0012B69F480E00BC08FEF9FEF9F
:1060700008C064E27AE081EC96E00E94061781E0B5
:1060800090E029960FB6F894DEBF0FBECDBFDF912A
:10609000CF911F910F91FF900895CF93DF93EC0163
:1060A000E881F9810284F385E02DCE0119950196EE
:1060B000B9F7DF91CF9108950F931F93CF93DF939B
:1060C000EC018B0168EA74E00E94B217011511051A
:1060D000B9F1F80161918F01662391F1603220F0EE
:1060E000623211F06C3541F56CE5CE010E94B915B4
:1060F000F801319780818C30D1F044F48930D9F0A7
:106100008A30B9F0883029F762E616C0823259F039
:1061100024F48D30F1F662E70FC08F3231F08C3508
:10612000C1F66CE509C062E207C06FE205C066E631
:1061300003C06EE601C064E7CE010E94B915C9CF65
:1061400062E2CE010E94B91580E090E0DF91CF912C
:106150001F910F9108955F926F927F928F929F92FD
:10616000AF92BF92CF92DF92EF92FF920F931F9365
:10617000CF93DF931F92CDB7DEB74C0180E697E057
:106180000E94664C811126C022C00F5F1F4F89817B
:10619000F801E25AF84F8183282F2F7730E02C9DA9
:1061A000A0012D9D500D3C9D500D1124A40EB51E37
:1061B00037E0CC0CDD1CEE1CFF1C3A95D1F787FFB5
:1061C00015C0CE0101960E94664C8111DECF80E0A1
:1061D00090E088C070906007198201E010E0A12C67
:1061E000B12CC12CD12C7601C394EBCF872D807FAD
:1061F00055245394803309F0512C8FEF800FD40134
:106200008C93552021F1C801805A984F0E94664C0A
:106210008823E9F2C8018F59984F0E94664C882361
:10622000B1F20E5F1F4FD401EC91F0E0E25AF84F4B
:10623000E380F12CFE2CEE248481E80EF11C809189
:10624000600781FF08C0B2E0EB0EF11C04C080E0E3
:10625000E12CF12C01C082E0C82ED12CC01AD10A49
:106260009EEF692E77247A94C601800F911F8A15BC
:106270009B0568F5CE0101960E94664C882309F4BF
:10628000A6CF8091F7079091F8070097A9F05520C5
:1062900099F0F4012081A301421B51099A01200FBA
:1062A000311FE216F30640F4DC01ED91FC91019000
:1062B000F081E02D698119950038110528F4898154
:1062C000F801E25AF84F82830F5F1F4FCDCF8091C4
:1062D000F7079091F807892B21F40138110508F090
:1062E00076CFC8010F90DF91CF911F910F91FF9052
:1062F000EF90DF90CF90BF90AF909F908F907F9066
:106300006F905F9008952F923F924F925F926F929D
:106310007F928F929F92AF92BF92CF92DF92EF9235
:10632000FF920F931F93CF93DF931F92CDB7DEB7EA
:106330000E940320982E882309F41DC10E947153E6
:106340002B013C018091E6079091E707A091E807B7
:10635000B091E907A3019201281B390B4A0B5B0B93
:10636000DA01C90189399A43A105B105A8F48091E0
:10637000E2079091E307A091E407B091E507A3013C
:106380009201281B390B4A0B5B0BDA01C9018939D1
:106390009A43A105B105D0F12091EA0780915E07EB
:1063A00090915F07222379F02CEF3FEF3093FA07AB
:1063B0002093F907DC01ED91FC910488F589E02D2B
:1063C0001995912CD8C020EC20936007109261079A
:1063D000DC01ED91FC910280F381E02D42E050E080
:1063E00060E677E019954092E2075092E3076092E9
:1063F000E4077092E5074092E6075092E707609243
:10640000E8077092E90781E08093EA0780915E07D0
:1064100090915F07DC01ED91FC910084F185E02D06
:106420001995892B09F4A7C0CE0101960E94AB30C3
:106430006C01892B09F49FC04092E6075092E70750
:106440006092E8077092E90780916007807F80334F
:1064500009F076C08091EB079091EC07892B09F445
:106460008AC0E980F12CF701E25AF84F038110E06D
:10647000102F00278481080F111DF701EE59F84FE6
:106480005F01B7016D59784FA801CF010E942A65BD
:1064900098012E0D3F1DF901E25AF84F14828091A8
:1064A00060078670882EA091EB07B091EC0742E060
:1064B000841337C0858190E0982F882746811C017E
:1064C000240E311C4BEF5FEF4E195F09401B510B3F
:1064D0004C0D5D1DB9016B59784FC501FD01199532
:1064E00080E4809360078092610730926207209277
:1064F000630780915E0790915F07DC01ED91FC914D
:106500000280F381E02D44E050E060E677E01995E9
:106510004092E2075092E3076092E4077092E50729
:106520002AC04DEF5FEF4E195F09401B510B4C0D18
:106530005D1DB9016D59784FC501FD0119951BC04D
:10654000803CA9F480ED80936007109261078091F0
:106550005E0790915F07DC01ED91FC910280F38171
:10656000E02D42E050E060E677E0199504C0803D00
:1065700011F41092EA07892D0F90DF91CF911F91AE
:106580000F91FF90EF90DF90CF90BF90AF909F90D2
:106590008F907F906F905F904F903F902F900895D5
:1065A000CF93C82F462F61E070E00E947D4661E0E6
:1065B00070E08C2F0E9487468111F9CFCF9108950A
:1065C0008F929F92AF92BF92CF92DF92EF92FF9203
:1065D0000F931F93CF93DF93B82E4B018A01A22E06
:1065E00068E270E00E948746C82FD0E069E270E060
:1065F0008B2D0E948746DC2FCC27C82B9E0137703D
:10660000CB2CD12CC601880F991FAC014855554F92
:106610006A01FA0180819181820F931FA801420FC4
:10662000531F4130584098F060E078E07B01E21A57
:10663000F30AA701B4010E941D40A8014E195F0989
:10664000B4016E0D7F1DF6018081918102C0A80109
:10665000B4010E941D40A1100EC0C00FD11F4D2FCC
:1066600068E270E08B2D0E947D464C2F69E270E05D
:106670008B2D0E947D46DF91CF911F910F91FF904E
:10668000EF90DF90CF90BF90AF909F908F90089544
:106690009F92AF92BF92CF92DF92EF92FF920F93B1
:1066A0001F93CF93DF93982E8B015A01690164E207
:1066B00070E00E948746E82EF12C65E270E0892D9B
:1066C0000E948746FE2CEE24E82AE701C00FD11F66
:1066D0009E013770E92CF12CC701880F991FAC017E
:1066E0004056554F7A01FA0180819181820F931FA4
:1066F000A9014C0D5D1D4130584090F000E018E0BC
:10670000021B130BA801B5010E944D40A601401BBE
:10671000510BB501600F711FF7018081918102C09B
:10672000A601B5010E944D40CC0DDD1D4D2F64E248
:1067300070E0892D0E947D464C2F65E270E0892D26
:10674000DF91CF911F910F91FF90EF90DF90CF904D
:10675000BF90AF909F900C947D46FF920F931F9334
:10676000CF93DF93F82EC0E0D0E08F2D0E94FE3F44
:106770008C01892B21F08F2D0E94FE3FEC01C01768
:10678000D10799F7CE01DF91CF911F910F91FF9023
:106790000895CF93DF93FC0101900020E9F79F015A
:1067A000281B390B285F3F4F2138310570F5EC016C
:1067B0000E940320882349F18091E0079091E1072E
:1067C000019611F481E090E09093E1078093E00757
:1067D0008091E0079091E1079093650780936607A9
:1067E00047E050E060E677E0CE010E94711FFC01B7
:1067F000E25AF84F1282AC014450510960E677E04A
:1068000082E8DF91CF910C94921F80E0DF91CF91CD
:1068100008951F920F920FB60F9211240BB60F928C
:106820002F933F934F935F938F939F93EF93FF9398
:1068300020919E0A30919F0A80919C0A90919D0A16
:10684000AC014F5F5F4F50939D0A40939C0AF90142
:10685000E80FF91F80818093CE008091060290910D
:10686000070220919C0A30919D0A8217930748F4F1
:106870008FEF9FEF90939D0A80939C0A88E480930A
:10688000C900FF91EF919F918F915F914F913F913F
:106890002F910F900BBE0F900FBE0F901F90189569
:1068A0001F920F920FB60F9211242F933F938F9345
:1068B0009F9320919A0A30919B0A80919C0A909113
:1068C0009D0A21303105A9F48F3F2FEF920789F4FB
:1068D0001092C8001092CD0089E08093CC0086E22F
:1068E0008093CA001092CE0010929D0A10929C0ACA
:1068F00017C0892BA9F41092C8001092CD0083E034
:106900008093CC008EE08093CA0088E28093C90017
:106910001092CE0081E090E090939D0A80939C0AB3
:106920009F918F913F912F910F900FBE0F901F90CD
:1069300018951F920F920FB60F9211240BB60F925B
:106940002F933F934F935F936F937F938F939F9377
:10695000AF93BF93EF93FF932091C8008091CE0037
:106960009091990A24FF08C081E08093990A809150
:106970009E0A90919F0A55C0913099F481110EC0E2
:1069800082E08093990A0E9471536093930A7093F6
:10699000940A8093950A9093960A3EC01092990AA1
:1069A00044C0923009F041C0E091970AF091980AF2
:1069B0009081981721F091E09093050280832091B7
:1069C000970A3091980A8091910A9091920A28171B
:1069D000390711F51092990A809105028823D1F0A8
:1069E00080918F0A9091900A892BA1F01092C90092
:1069F000E0918F0AF091900A199580E98093C9007F
:106A00001092C8001092CD0083E08093CC008EE0FD
:106A10008093CA00109205028091970A9091980A7B
:106A200001969093980A8093970AFF91EF91BF91F6
:106A3000AF919F918F917F916F915F914F913F9116
:106A40002F910F900BBE0F900FBE0F901F901895B7
:106A5000CF92DF92EF92FF920F931F93CF93DF932A
:106A60008C017B0186E090E00E944566EC019093EA
:106A70008E0A80938D0AF80101900020E9F7CF017A
:106A8000801B910B0E9445666C01B8010E946E65E7
:106A9000F80101900020E9F73197E01BF10BEC0DB4
:106AA000FD1D1082D982C882FB82EA8280918B0A06
:106AB00090918C0A9D838C83D0938C0AC0938B0A0F
:106AC000DF91CF911F910F91FF90EF90DF90CF90CA
:106AD0000895FB01248135814281538124173507B4
:106AE00058F440815181DA01A20FB31F8C93848145
:106AF000958101969583848380E008958F929F927B
:106B0000AF92BF92CF92DF92EF92FF920F931F93BB
:106B1000CF93DF936115710509F4FFC0FB01008578
:106B2000002E000C110B220B330B0730110508F05F
:106B3000F4C0DB01EC01F8018827EC52FF4F8F4FC6
:106B40000C9411616AEA74E006C019968C9188234E
:106B500089F06FEA74E0CE01DF91CF911F910F9120
:106B6000FF90EF90DF90CF90BF90AF909F908F906D
:106B70000C94E41564EB74E0EECF19964D915D91A1
:106B80006D917C911C972AE030E0CE01DF91CF918E
:106B90001F910F91FF90EF90DF90CF90BF90AF903B
:106BA0009F908F900C9442161996CD90DD90ED90A9
:106BB000FC901C9720E030E0A901C701B6010E94BB
:106BC000A86187FF09C06AEB74E0CE010E94B2178A
:106BD000F7FAF094F7F8F094C701B6010E94266224
:106BE0004B015C012AE0AB01BC01CE010E94F9150A
:106BF0006CEB74E0CE010E94B217C501B4010E9493
:106C000055629B01AC01C701B6010E943B612DECAE
:106C10003CEC4CE45DE30E943C6120E030E040E26B
:106C200051E40E940C630E942662AB0160E070E0B8
:106C30002AE0CE010E94F91570C019966D917C91E1
:106C40001A97CE01DF91CF911F910F91FF90EF9096
:106C5000DF90CF90BF90AF909F908F900C945C305E
:106C600016960D911C9117976BE5CE010E94B915F0
:106C7000019619F48FEF9FEF52C00115110571F0C5
:106C8000B801CE010E947E350196A1F3F801028180
:106C900013810115110589F36CE2E7CF6DE52FC073
:106CA00016960D911C9117976BE7CE010E94B915AE
:106CB000019601F30115110509F1F8016081718157
:106CC000CE010E945C300196A9F26AE3CE010E94D7
:106CD000B915019679F2B801CE010E947E35019670
:106CE00049F2F801028113810115110519F36CE2D3
:106CF000CE010E94B9150196E9F6BCCF6DE7CE0131
:106D00000E94B91521E030E0019611F020E030E05A
:106D100088279927821B930B02C080E090E0DF91C7
:106D2000CF911F910F91FF90EF90DF90CF90BF9088
:106D3000AF909F908F900895CF93DF93EC01E881FF
:106D4000F9810284F385E02DCE0119958F3F2FEF55
:106D5000920771F0E881F9818132910594F30684FC
:106D6000F785E02D682FCE01199580E090E002C0F4
:106D70008FEF9FEFDF91CF9108956F927F928F9267
:106D80009F92AF92BF92CF92DF92EF92FF920F93BA
:106D90001F93CF93DF93CDB7DEB761970FB6F8940B
:106DA000DEBF0FBECDBF6EEB74E080910706909101
:106DB00008060E94FD1B8C010097D1F10E94631F01
:106DC0008230B1F560E0C8010E94F01B7C0161E0F7
:106DD000C8010E94F01BDC0119960D911C911A97B5
:106DE000F701818521E09091830A992309F454C326
:106DF000909170009E7F909370001092830A109281
:106E00000202109201028093000221110E94652962
:106E1000C8010E948D2963E97BE081EC96E00E9425
:106E2000C0154AE050E0B80181EC96E00E94DD1602
:106E300062EC74E080910706909108060E94FD1BA9
:106E40009093B70A8093B60A009709F49FC00E94F6
:106E5000631F082F10E00115110509F497C0000FFA
:106E6000111F000F111F8091B20A9091B30A892B54
:106E700009F07FC0C8010E9445669093B30A8093D1
:106E8000B20A10929B0A10929A0A1092B90A1092B2
:106E9000B80A1092990A10929D0A10929C0A013029
:106EA00022E012070CF0FAC27801C70101960E9495
:106EB000456690939F0A80939E0A9093980A8093C8
:106EC000970A8E0D9F1D9093920A8093910A0E94BB
:106ED00071536093930A7093940A8093950A9093E8
:106EE000960A80E090E0E0919E0AF0919F0AE80FF8
:106EF000F91F10820196E816F906ACF782E090E0DF
:106F000090939B0A80939A0A80E98093C90010921B
:106F1000C8001092CD0083E08093CC008EE0809377
:106F2000CA00F0920702E092060220919E0A309178
:106F30009F0A8091060290910702820F931F9093FF
:106F4000920A8093910A232B09F4ACC26BEB7AE08E
:106F500081EC96E00E94C0154AE050E0B80181EC57
:106F600096E00E94DD168BE69FE49093900A809352
:106F70008F0A69E77BE081EC96E00E94C0154AE049
:106F800050E0B80181EC96E00E94DD160091070602
:106F90001091080668EC74E0C8010E94FD1B9093F4
:106FA000BB0A8093BA0A6FEC74E0C8010E94FD1B13
:106FB0009093450580934405009791F462ED74E049
:106FC00080910706909108060E94FD1B909343054F
:106FD00080934205DC011696ED90FC901797CFC187
:106FE000209146052111EACFFC01E680F7808091CF
:106FF000300590913105892B09F0D1C064E17BE027
:1070000081EC96E00E94061781E190E00E944566BF
:107010008C0188E1D80111968C93119712961C92DD
:1070200012971C9250961C921E921F971092BF0AA4
:107030001092BE0A1092570B1092790B0E942B45AA
:10704000109331050093300583E190E00E9445667E
:10705000FC018FE297E2928B818B16830583148269
:10706000108289E0818311E012831383F093390544
:10707000E093380580EA90E00E94456690933505DC
:107080008093340588E290E00E94456690932F0536
:1070900080932E051092BF0A1092BE0A1092570BD1
:1070A0001092790B0E942B4580913005909131050B
:1070B0000E94AB4181E00E945B4B811168C061E09E
:1070C0007BE081EC96E00E940617C0903005D090DE
:1070D0003105C6010E94AB4140E060EFC6010E944D
:1070E0008A42C6010E94A841E0913005F091310525
:1070F000108361EE7AE081EC96E00E9406178091A1
:107100003005909131050E944942882331F065EDA8
:107110007AE081EC96E00E94061700913805109104
:1071200039050E9471534B015C01B0E18B0EB7E24F
:107130009B1EA11CB11CD8011596ED91FC911697D0
:107140008FEF83871486DF0113963B961D92AE174F
:10715000BF07E1F7F801148277247394BE01665FDC
:107160007F4FD80115968D919C9116970E94B3423E
:1071700018160CF49EC185EE93E590933305809329
:107180003205E0913805F0913905128208C067ECAC
:107190007AE081EC96E00E94061780E001C081E071
:1071A00080934605109237051092360501E010E0F5
:1071B00078E0D72EE114F10409F400CF8091460560
:1071C000882309F4FBCEF7018085863009F09BC047
:1071D000A080B180CE0101964C01350190E1690E8D
:1071E000711CD5018C910E94D118C82EB2E0AB0E53
:1071F000B11CF501319780810E94D118C29460EFD3
:10720000C6228C29F40181934F01A614B70449F7D3
:107210008091360590913705843191050CF073C04B
:10722000880F991FE0912E05F0912F05E80FF91FA7
:1072300011830083A0913605B091370533E0AA0F82
:10724000BB1F3A95E1F78091340590913505A80F61
:10725000B91FFE0131968D2D01900D928A95E1F7AF
:107260006CE37BE081EC96E00E94C01560913605EE
:10727000709137054AE050E081EC96E00E948C1650
:1072800065E37BE081EC96E00E94C01580913605B5
:107290009091370543E0880F991F4A95E1F72091B7
:1072A000340530913505820F931F0E943A4C81ECD2
:1072B00096E00E94D916609136057091370553E02B
:1072C000660F771F5A95E1F7809134059091350547
:1072D000680F791FDB018C91883261F48091380549
:1072E000909139050E94B84B8091300590913105FD
:1072F0000E947E42809136059091370501969093C9
:10730000370580933605F701E280F38053CFC1142F
:10731000D104D1F1E114F104B9F1D70118968C919F
:107320008530A9F7C7010E94631F182F823078F3B8
:1073300061E0C7010E94F01BFC010185B28414309A
:1073400008F46BC163E0C7010E94F01BFC01C1841B
:10735000D28460E0C7010E94F01BFC018185928508
:10736000A385B4850597A109B1090297A105B105C7
:1073700008F429C1D7011296ED90FC901397C090A4
:107380004205D0904305C3CFF60186819781909343
:107390003D0580933C05009107061091080665ECB9
:1073A00074E0C8010E94FD1B90933F0580933E0549
:1073B00068ED74E0C8010E94FD1B9093B50A8093AC
:1073C000B40A66E67BE081EC96E00E9406176FE562
:1073D0007BE081EC96E00E94C01581E0209142059F
:1073E00030914305232B09F480E00E94E51B67E5FB
:1073F0007BE081EC96E00E94C01581E020913E0583
:1074000030913F05232B09F480E00E94E51B6FE4D7
:107410007BE081EC96E00E94C01581E02091BA0AE1
:107420003091BB0A232B09F480E00E94E51B69E43C
:107430007BE081EC96E00E94C01581E02091B40AC7
:107440003091B50A232B09F480E00E94E51B61E42A
:107450007BE081EC96E00E94C01581E0209144051C
:1074600030914505232B09F480E00E94E51B6196CD
:107470000FB6F894DEBF0FBECDBFDF91CF911F9145
:107480000F91FF90EF90DF90CF90BF90AF909F90C3
:107490008F907F906F90089520E0B5CCE12CE2E0D2
:1074A000FE2E03CD64EA7AE081EC96E00E94061796
:1074B0005ACD0E947153681579058A059B0508F01D
:1074C0005ACE67E0CE010A960E943A419989891303
:1074D00070C065EF73E081EC96E00E94B217D801AE
:1074E0008C9181113AC015968D919C9116970E94AE
:1074F0004942BE01665F7F4FF801858196810E94F7
:10750000744340E064EBD80115968D919C911697D9
:107510000E948A42F801C580D680C6010E94CE41F1
:10752000C6010E94AB4167E888E196E00E94735271
:1075300060E888E196E00E947352C6010E94A8416B
:10754000C6010E94CE41D82ED80115968D919C91EE
:1075500016970E944942D5FE33C0AE014F5F5F4F80
:10756000BE01665F7F4FC8010E94282AF801D180C2
:107570008A85803109F455C0BE01665F7F4FC8011E
:107580000E94FA298D1520F4D80111968C910BC018
:107590008A85803111F48CE006C0BE01665F7F4FA2
:1075A000C8010E94FA29F801818384818F5F848356
:1075B000D5CD6BEF73E081EC96E00E94B217CECD93
:1075C000D8017C92CACF61E0802F0E94FB5211E06B
:1075D000CA94CD2809F010E0612F802F0E94CB5271
:1075E00064E77BE081EC96E00E94C0154AE050E041
:1075F000602F7B2D81EC96E00E948C1662E77BE089
:1076000081EC96E00E94C015612F70E04AE050E0E6
:1076100081EC96E00E94DD16ADCE82E0C82ED12C22
:1076200098CEFCE0FD1508F4AFCFB5CFCF93DF9334
:10763000CDB7DEB72C970FB6F894DEBF0FBECDBF27
:1076400063ED7BE081EC96E00E94061786E290E015
:107650000E94E96E8B37C1F51C821B821E821D823F
:107660008FEF9FEF98878F838BE792E09A838983D0
:1076700086E290E09A8789871C861B8680910706A0
:10768000909108060E940F4BCE0101960E943A4B42
:10769000909308068093070681EC96E00E94D91625
:1076A0008091070690910806892B19F466EB7BE020
:1076B0000DC06FEA7BE081EC96E00E9406170E9405
:1076C000BD3681E090E008C062EC7BE081EC96E0A2
:1076D0000E94061780E090E02C960FB6F894DEBF6B
:1076E0000FBECDBFDF91CF9108950C94163B2F9222
:1076F0003F924F925F926F927F928F929F92AF9242
:10770000BF92CF92DF92EF92FF920F931F93CF938E
:10771000DF93CDB7DEB7E3970FB6F894DEBF0FBEA9
:10772000CDBF7C011A012B0139010E9471534B011D
:107730005C0187010D5B1F4FC8010E943C4E18166B
:107740001906A4F00E947153DC01CB018819990934
:10775000AA09BB09281639064A065B06D8F062E377
:1077600070E080E090E00E943753E6CF42E250E0C4
:10777000BE016F5F7F4FC8010E94F44D8981823046
:1077800011F080E061C1F801848995898334910505
:10779000C1F702C08FEF58C16D817E818F819885BE
:1077A0000E9419614B015C01F30160837183828344
:1077B000938346E050E0B701685F7F4FCE014D965E
:1077C0000E941D65892BE9F6F70180819181A281D4
:1077D000B38188169906AA06BB0698F28481958122
:1077E000A681B78188159905AA05BB0550F289893C
:1077F0009A89AB89BC8986879787A08BB18B8EECE1
:10780000A82EB12CC8010E94134EF1E0AF1AB108A6
:10781000C9F719A6670182E2C80ED11CF701B69616
:10782000FBA7EAA7C7018A969DA78CA73C974F01A3
:1078300089969FA78EA73897F9ABE8AB1701F6E1B9
:107840002F0E311CC5979BAB8AABF801818D928DB1
:10785000181619060CF0F7C0C8010E94134E8333A6
:10786000910509F4CBC0FCF481309105C9F11CF4F9
:10787000892B59F3DCC083309105D1F1069709F0CB
:10788000D6C0C8010E94134E5C0144E050E06AA9D2
:107890007BA9C8010E94F44D412C512CBB24F4E07B
:1078A000AF1AB10840C08A33910509F47BC03CF49B
:1078B0008533910569F0C69709F440C0B8C08B3391
:1078C000910509F485C08F3F910509F4BECFAFC083
:1078D000C8010E94134EC8010E94134E89A7B5CF5C
:1078E000C8010E94134E44E050E068A979A93AC04B
:1078F000C8010E94134E5C0144E050E0B101C80190
:107900000E94F44D412C512CBB2494E0A91AB108DB
:107910004A145B040CF099CFC8010E94134EEFEF9C
:107920004E1A5E0AF5CF4A145B040CF08ECFC801E4
:107930000E94134E8FEF481A580AF5CFC8010E94D3
:10794000134EB82EF701828D811110C0838D8111E5
:107950000DC0848D81110AC0858D811107C044E05E
:1079600050E0B401C8010E94F44D6FCFEEA5FFA511
:107970004080518062807380B401CE0183960E9462
:10798000B4178DA19EA1AFA1B8A584159505A60534
:10799000B70529F3BB2009F458CFC8010E94134E44
:1079A000BA94F8CFC8010E94134E44E050E06AA593
:1079B0007BA5C8010E94F44DF70166A177A180A5BF
:1079C00091A50E94196166A377A380A791A73DCFD7
:1079D000C8010E94134E44E050E06CA57DA5C8018B
:1079E0000E94F44DF70162A573A584A595A50E9498
:1079F000196162A773A784A795A727CFC8010E9422
:107A0000134E44E050E0B601C8010E94F44DF70166
:107A100062A173A184A195A10E94196162A373A3BD
:107A200084A395A366A777A780AB91AB0ECFC801BF
:107A30000E94134EB82EBB2009F407CFC8010E9444
:107A4000134EBA94F8CF89A5E3960FB6F894DEBF2B
:107A50000FBECDBFDF91CF911F910F91FF90EF909F
:107A6000DF90CF90BF90AF909F908F907F906F905E
:107A70005F904F903F902F9008957F928F929F92AA
:107A8000AF92BF92CF92DF92EF92FF920F931F932C
:107A9000CF93DF93CDB7DEB7A6970FB6F894DEBFCE
:107AA0000FBECDBF8C01762E942E852E20E2B22EF5
:107AB000CE0101967C01FC012B2D11922A95E9F74C
:107AC00084E693E09AA389A38FEF8BA38CA38DA365
:107AD0008EA3680183E4C80ED11C43E450E0BE01CC
:107AE0006F5D7F4FC6010E94F646019609F4BFC044
:107AF00081E089838A8386E0A82EAB821C82F8010C
:107B000064817581868197810E9419616D837E836E
:107B10008F83988789869A8680E890E09C878B87F8
:107B20004CE150E0B701C6010E94474DF7012B2DF3
:107B300011922A95E9F7480188E0880E911CF4011A
:107B4000D70101900D92AA94E1F740E150E0B7010E
:107B5000C6010E94474DF7011192BA94E9F796E0E9
:107B6000A92EB12C40E250E0B701C6010E94474D5A
:107B7000F1E0AF1AB108B1F783E6898392E89A83FE
:107B800093E59B838C8385E38D8381E08E837F8265
:107B90009DE3988797E099878A8786E0F401DE0164
:107BA0001B9601900D928A95E1F78CE0898B8A8B68
:107BB0006DED74E0CE0143960E946E65F801438539
:107BC000BE01675E7F4FC8010E94CC26F801448544
:107BD000BE01655E7F4FC8010E94CC26F801458535
:107BE000BE01635E7F4FC8010E94CC264EE150E08B
:107BF000B701C6010E94474DF3E07F121EC082E329
:107C0000898384E08A83F80196859B8397859C838A
:107C100090899D8391899E8396E39F838887828D37
:107C20008987838D8A87848D8B87858D8C874CE0AF
:107C300050E0B701C6010E94474D87E3898386E083
:107C40008A8391E09B8393E09C838D838FE08E8376
:107C50008AE38F838BE388878FEF898749E050E041
:107C6000B701C6010E94474DC6010E94AD46A696C7
:107C70000FB6F894DEBF0FBECDBFDF91CF911F913D
:107C80000F91FF90EF90DF90CF90BF90AF909F90BB
:107C90008F907F9008952F923F924F925F926F92B4
:107CA0007F928F929F92AF92BF92CF92DF92EF928C
:107CB000FF920F931F93CF93DF93CDB7DEB7279734
:107CC0000FB6F894DEBF0FBECDBF8C010E94BF6718
:107CD0002FEC37E040E050E00E94216FDC01CB0147
:107CE0000196A11DB11DF80184839583A683B783F6
:107CF00080839183A283B3835801F3E4AF0EB11C58
:107D0000C5010E94F14564E470E0C5010E94064689
:107D1000882309F43CC10E9471532B013C01812C42
:107D2000912C1D82C8018E5B9F4F9F838E8343E001
:107D3000342E58EEC52E53E0D52EE12CF12C62E006
:107D4000262EAE81BF818C91833009F407C1811149
:107D500020C0F80184819581A681B7810196A11D7B
:107D6000B11D84839583A683B7830E9471536419E0
:107D7000750986099709A70196010E94FF6EA9015E
:107D800061E0C8010E943D3D81E0AE81BF818C93DE
:107D9000C6C08430F9F4F80184819581A681B78149
:107DA0000196A11DB11D84839583A683B7830E948C
:107DB00071536419750986099709A70196010E94F4
:107DC000FF6EA90163E0C8010E943D3DAE81BF8105
:107DD0002C92A5C0813061F5F80142AD53AD64AD80
:107DE00075AD9E012F5F3F4FC8010E94773B8D8389
:107DF000823009F094C089819A81AB81BC81F801FD
:107E000084839583A683B7830E947153641975098F
:107E100086099709A70196010E94FF6EA90163E0F8
:107E2000C8010E943D3DED81AE81BF81EC937EC0D3
:107E3000823009F074C0D801DA964D915D916D9150
:107E40007C91DD979E012F5F3F4FC8010E94773BD9
:107E50008D83853009F05CC0EE81FF813082F801AE
:107E600082A193A1A4A1B5A1892B8A2B8B2B41F4CC
:107E700084E893E0A0E0B0E082A393A3A4A3B5A319
:107E8000F80186A197A1A0A5B1A5892B8A2B8B2BE0
:107E900061F482A193A1A4A1B5A1B695A7959795E8
:107EA000879586A397A3A0A7B1A7F80182A593A55C
:107EB000A4A5B5A5892B8A2B8B2BA9F482A193A10C
:107EC000A4A1B5A1AC01BD0123E0769567955795B6
:107ED00047952A95D1F7841B950BA60BB70B82A764
:107EE00093A7A4A7B5A7F80186A197A1A0A5B1A5BE
:107EF00086A797A7A0ABB1AB82A593A5A4A5B5A56E
:107F000082AB93ABA4ABB5AB88248394912C0EC009
:107F1000FD81F63021F4AE81BF811C9207C0BD8186
:107F2000BF3F21F4EE81FF8110821D82F1E08F16A8
:107F3000910409F406CF0E947153DC01CB0184192E
:107F40009509A609B709F80126A937A940AD51AD91
:107F5000281739074A075B0708F0F3CEC5010E94CE
:107F6000F145F80184819581A681B7810196A11D13
:107F7000B11D84839583A683B7830E947153F80152
:107F8000FE966083718382839383C40102C080E084
:107F900090E027960FB6F894DEBF0FBECDBFDF91FD
:107FA000CF911F910F91FF90EF90DF90CF90BF90F6
:107FB000AF909F908F907F906F905F904F903F9089
:107FC0002F9008952C9A08952C9808951F93CF937D
:107FD000DF93182F66E270E00E948746C82FD0E03A
:107FE00067E270E0812F0E948746DC2FCC279E013C
:107FF000282BC901DF91CF911F9108951F93CF9333
:10800000DF93182F60E270E00E948746C82FD0E00F
:1080100061E270E0812F0E948746DC2FCC279E0111
:10802000282BC901DF91CF911F9108958EBD0000CB
:108030000DB407FEFDCF8EB50895CF92DF92EF927B
:10804000FF920F931F93CF93DF93EC017A018B0183
:108050006C01C40ED51ECC15DD05A9F00E94E43FCD
:108060008FE00E9416408D2F0E9416408C2F0E9498
:108070001640219680E00E941640F80181938F01FE
:108080000E94E23FE8CFC701DF91CF911F910F918E
:10809000FF90EF90DF90CF900895CF92DF92EF9214
:1080A000FF920F931F93CF93DF93EC017A018B0123
:1080B0006C01C40ED51ECC15DD05A1F00E94E43F75
:1080C00080EF0E9416408D2F0E9416408C2F0E9438
:1080D00016402196F80181918F010E9416400E945E
:1080E000E23FE9CFC701DF91CF911F910F91FF9040
:1080F000EF90DF90CF9008951F93CF93DF931F925F
:108100001F92CDB7DEB7182F6A8399830E94E43F90
:1081100080EF0E9416409981892F0E941640812F7E
:108120000E9416406A81862F0E9416400E94E23FFC
:1081300081E00F900F90DF91CF911F910895FF92F2
:108140000F931F93CF93DF931F921F92CDB7DEB78C
:10815000F82E8A012A8369830E94954E80E590E07B
:108160000E94AB272A816981462F422B60E070E094
:108170008F2D0E947D460115110551F40091BC0A16
:108180001091BD0A0F5F1F4F1093BD0A0093BC0AE8
:10819000412F64E070E08F2D0E947D46402F65E006
:1081A00070E08F2D0E947D4661E070E08F2D0E946F
:1081B000D0320E94AA2781E00F900F90DF91CF91DB
:1081C0001F910F91FF9008951F93CF93DF931F92FC
:1081D0001F92CDB7DEB7182F80E590E069837A83D0
:1081E0000E94AB2721E041E050E069817A81812F34
:1081F0000E94E0320E94AA2781E090E00F900F9049
:10820000DF91CF911F91089585ED8093BC008091FF
:10821000BC0084FDFCCF1092550B08950895E091A9
:10822000BF0A8091BE0AE81730F4F0E0E95FF44F2E
:10823000808190E008958FEF9FEF08959091BF0A9D
:108240008091BE0A981750F4E92FF0E0E95FF44FEF
:10825000208130E09F5F9093BF0A02C02FEF3FEF75
:10826000C90108958091BE0A90E02091BF0A821B47
:1082700091090895DC01E0E0615038F08D91E82724
:10828000F0E0EE51F44FE491F7CF8E2F0895CF93A5
:10829000DF93EA010E94282A882339F068E0CE01A2
:1082A0000E943A4191E02885821390E0892FDF9166
:1082B000CF910895FC0181819091550B9111FCCFD4
:1082C00091E09093550B9093540B2FEF2093530B09
:1082D0001092520B1092510B9093300B9091300BE7
:1082E000880F892B8093300B80912F0B813061F4A4
:1082F00010922F0B8091300B8093BB008091BC00BB
:1083000083FDF8CF85EC01C085EE8093BC008091A1
:10831000550B8130E1F38091520B811103C08091A4
:10832000520B01C081E0A1E3BBE027E03BE0F90193
:108330009E2F921B981718F49D919193F9CF10924C
:10834000BF0A8093BE0A88E196E00E941E4108950C
:1083500081E00C945B4BFC01818191E09093560B82
:108360008093780B1092570B1092790B08951F93FE
:10837000CF93DF93EC01162F0E94AB4161EE88E1B1
:1083800096E00E947352612F88E196E00E9473523A
:10839000CE01DF91CF911F910C94A841AF92BF9273
:1083A000CF92DF92EF92FF921F93CF93DF93EC0176
:1083B0000E9471536B017C0128EEC20E23E0D21E95
:1083C000E11CF11C8BE4A82EB12C0E9471536C159A
:1083D0007D058E059F0598F460EFCE010E94B741A0
:1083E000CE010E945A41182F80FF11C0EF85F889F5
:1083F000309709F01995C5010197F1F7E6CF81E0B3
:108400008A8364EE74E081EC96E00E94F416812F7A
:10841000DF91CF911F91FF90EF90DF90CF90BF90B1
:10842000AF9008951F93CF93DF93EC01162F0E9416
:10843000CE41CE010E94AB4162ED88E196E00E9400
:108440007352212F30E02095309584E0220F331FA6
:108450008A95E1F7612F622B88E196E00E947352C2
:10846000CE010E94A841CE010E945A41811711F00D
:1084700084E08A83DF91CF911F910895CF93DF939A
:10848000EC0163EC0E94B741CE01DF91CF910C94D7
:108490005A411F93CF93DF93EC010E94CE41CE014E
:1084A0000E943E4260E0CE010E941242CE010E9434
:1084B000CE41CE010E94AB4164EB88E196E00E9480
:1084C0007352CE010E94A841CE010E94CE41182FC6
:1084D00082FF02C082E08A838881882341F0CE0136
:1084E0000E943E42682F6160CE010E94124211FB41
:1084F000882780F9DF91CF911F910895CF93DF9363
:10850000EC010E943E42682F6460CE01DF91CF9162
:108510000C941242EF92FF921F93CF93DF931F921E
:10852000CDB7DEB77C01162F49830E94CE41498129
:10853000442319F0C7010E947E42C7010E94AB414B
:1085400065EA88E196E00E947352612F88E196E027
:108550000E947352C7010F90DF91CF911F91FF903E
:10856000EF900C94A8416F927F928F929F92AF925E
:10857000BF92CF92DF92EF92FF920F931F93CF9310
:10858000DF93FC01248521119FC0872E762EEC01FC
:108590000E944942811108C06FEE74E081EC96E0C0
:1085A0000E94F4168FEF91C0CE010E94CE4140E0B0
:1085B00060EFCE010E948A42E12CF12C66246A947D
:1085C000CC24C394D12C0E2D06950695069510E06B
:1085D0008E2D8770560101C0AA0C8A95EAF78B850B
:1085E000082E000C990BE816F90634F4FE01E00F92
:1085F000F11F93809A2006C099249394E816F906F7
:1086000009F0912CCE010E94CE41CE010E94AB41D7
:1086100068E788E196E00E947352911002C060E022
:1086200001C060E888E196E00E947352CE010E948A
:10863000A841CE010E94CE41282F2074982F907817
:1086400085FF13C02223B9F0482F50E060E070E0AE
:1086500022E081EC96E00E94F9156BEF74E081EC6A
:1086600096E00E94F4168EEF30C0211104C09111E3
:1086700004C06E2C08C0992331F0FE01E00FF11FF9
:108680008381A82A06C0FE01E00FF11FA094838118
:10869000A822A382FFEFEF1AFF0A80E4E816F10494
:1086A00009F091CF6B86EFEF6E1202C081E08C87EC
:1086B000DE011396E72DF82D2B968D918193AC1743
:1086C000BD07D9F781E001C080E0DF91CF911F9114
:1086D0000F91FF90EF90DF90CF90BF90AF909F9061
:1086E0008F907F906F900895CF92DF92EF92FF92DC
:1086F0000F931F93CF93DF931F92CDB7DEB78C01FB
:10870000F62E40E065E579830E948A42CF2C79817C
:10871000D72E760188E0E80EF11CF60161916F0119
:1087200040E0C8010E948A42CE14DF04B1F70F90E6
:10873000DF91CF911F910F91FF90EF90DF90CF903D
:1087400008951F920F920FB60F9211240BB60F923D
:108750002F933F934F935F936F937F938F939F9349
:10876000AF93BF93EF93FF938091B900887F8036DA
:1087700009F49CC068F5883209F45BC090F480313C
:1087800009F454C038F4882309F4F6C0883009F499
:108790004DC0F6C0883109F44CC0803209F45DC088
:1087A000EFC0803409F468C048F4803309F455C040
:1087B000883309F0E5C08093530BD8C0803509F4A5
:1087C0004FC0883509F45DC0883409F0D9C0D6C0DF
:1087D000883909F4C7C0A8F4883709F467C038F4A9
:1087E000883609F463C0803709F460C0C9C088388E
:1087F00009F4B8C0803909F45FC0803809F0C0C0FE
:108800005BC0803B09F486C038F4803A09F466C046
:10881000883A09F47FC0B4C0803C09F4A7C0883C02
:1088200009F4A4C0883B09F48AC0AAC08091300B27
:1088300010C09091520B8091510B981770F5E091F8
:10884000520B81E08E0F8093520BF0E0EF5CF44FFF
:1088500080818093BB0085EC86C08093530B8EC0D3
:10886000E091520B81E08E0F8093520B8091BB0000
:10887000F0E0EF5CF44F80839091520B8091510BAC
:108880006EC0E091520B81E08E0F8093520B80916D
:10889000BB00F0E0EF5CF44F80838091540B8111BA
:1088A0006DC081E080932F0B84EA61C083E08093E8
:1088B000550B1092060BCFCF8091060B803208F03B
:1088C00051C0E091060B81E08E0F8093060B8091E2
:1088D000BB00F0E0EA51F54F8083BDCF85EC80937B
:1088E000BC001092550B8091060B803230F4E09161
:1088F000060BF0E0EA51F54F10826091060B70E034
:10890000E091E40AF091E50A86EE9AE0199510925A
:10891000060B36C084E08093550B1092E30A109248
:10892000E20AE091E00AF091E10A19958091E20AE9
:10893000811105C081E08093E20A1092C00AE091A3
:10894000E30A81E08E0F8093E30AF0E0E054F54FF4
:1089500080818093BB009091E30A8091E20A98178E
:1089600008F479CF85E88093BC000AC085EC809339
:10897000BC001092550B04C01092530B0E9404418E
:10898000FF91EF91BF91AF919F918F917F916F91E7
:108990005F914F913F912F910F900BBE0F900FBEA3
:1089A0000F901F9018954091E20A262F30E0240F77
:1089B000311D21323105DCF42091550B2430C9F4EE
:1089C000FC0180E090E0861758F43091E20A219192
:1089D000DC01A054B54FA30FB11D2C930196F3CF2A
:1089E0008091E20A680F6093E20A80E0089581E0D6
:1089F000089582E00895CF92DF92EF92FF920F9355
:108A00001F93CF93DF937C01262F972F8A018091AC
:108A1000560B882391F0C62FD72F6E01C40ED51E9A
:108A2000CC15DD0571F06991D701ED91FC910190B4
:108A3000F081E02DC7011995F3CF642F822F0E949A
:108A4000D344C801DF91CF911F910F91FF90EF9018
:108A5000DF90CF9008951092550B81E08093540BD6
:108A600010922F0B61E084E10E94CB5261E085E11E
:108A70000E94CB52E9EBF0E080818E7F8083808181
:108A80008D7F808388E48093B80085E48093BC0068
:108A90000895FC01818D928D0895FC01848995894A
:108AA000089524E633E0FC0131832083FB014089F3
:108AB000518962897389FC0142835383648375837E
:108AC0000895DC01ED91FC91048CF58DE02D199455
:108AD00080E00895FC019485FB018485981303C010
:108AE00081E0943009F480E0089521E0FC01848560
:108AF000843009F420E0822F08950895CF92DF9208
:108B0000EF92FF920F931F93CF93DF93CDB7DEB712
:108B1000AF970FB6F894DEBF0FBECDBF7C016A01E0
:108B200004E613E01A8309831C861B8688EE93E013
:108B3000A0E0B0E08D879E87AF87B88B88E993E08F
:108B40009A878987188F0F8B198E1A8E1B8E1C8E11
:108B500084E089A31DA30CA31EA21FA218A619A618
:108B60008091120690911306A0911406B0911506FB
:108B70008CA79DA7AEA7BFA78B839C83AD83BE8325
:108B800018861F82AE014C5D5F4FCE0101960E9498
:108B9000512481309105B1F4D701ED91FC91048805
:108BA000F589E02D1BA70AA78EA19FA1A8A5B9A5AD
:108BB0008CA79DA7AEA7BFA7A601BE01665D7F4F8C
:108BC000C7011995AF960FB6F894DEBF0FBECDBFA3
:108BD000DF91CF911F910F91FF90EF90DF90CF9099
:108BE0000895CF93DF93EC01888D843061F00E946B
:108BF000954EE88DF0E0EE0FFF1FE95DF44F118216
:108C0000108284E0888FDF91CF910895EF92FF92D8
:108C10001F93CF93DF93FC01208D243011F080E06F
:108C20001CC07B01EC0110E0812F0E94A94E811134
:108C300002C0188F05C08831E1F31F5F1430A1F71F
:108C4000888D843061F3FD86EC861A8E198E20E0C3
:108C5000A70162E00E949F4081E0DF91CF911F91C8
:108C6000FF90EF9008950F931F93CF93DF931F9280
:108C7000CDB7DEB78C01DC01ED91FC910084F1856C
:108C8000E02D1995892B51F0BE016F5F7F4FF801E0
:108C900084850E94E440898190E002C08FEF9FEFBD
:108CA0000F90DF91CF911F910F910895FC01848562
:108CB0000C94A14DCF93DF931F92CDB7DEB741E067
:108CC00050E0BE016F5F7F4FFC0184850E94A14D83
:108CD000181619061CF4898190E002C08FEF9FEFEF
:108CE0000F90DF91CF910895FC018485843011F0BD
:108CF0000C947F4D80E090E008959B0190E00496F5
:108D0000982F8827642F820F931F0C947C400F9319
:108D10001F93CF93DF931F92CDB7DEB790E00496F9
:108D2000982F88278C01060F171F0E94E43F8FE0C1
:108D30000E941640812F0E941640802F0E941640EC
:108D400080E00E94164089830E94E23F89810F9053
:108D5000DF91CF911F910F910895CF93FC01C08DAA
:108D600080E590E00E94AB2760E270E08C2F0E94CB
:108D7000D03262E070E08C2F0E94874684FD19C0DB
:108D800062E070E08C2F0E94874683FF0BC048E1B1
:108D900062E070E08C2F0E947D460E94AA2780E04E
:108DA00090E011C00E94AA2780E590E00E94AB27C6
:108DB000E0CF40E162E070E08C2F0E947D460E948F
:108DC000AA2781E090E0CF910895CF93DF93C82F39
:108DD000D62F472F60E170E00E947D464D2F61E164
:108DE00070E08C2FDF91CF910C947D46FF920F9312
:108DF0001F93CF93DF93FB01DC0157961C921E92C9
:108E000056975896FC908281811109C08381811107
:108E100006C08481811103C085818823F9F0411542
:108E20005105E1F08A01EF0180E590E00E94AB2757
:108E3000BE016E5F7F4F2F2D30E0922F882744E0D8
:108E400050E0845F9B4F0E944D40B8018F2D0E94DF
:108E5000E5460E94AA2781E090E002C080E090E011
:108E6000DF91CF911F910F91FF900895FC018485B0
:108E7000843011F00C94A94E80E00895CF93DF93D5
:108E8000FC0124852430D1F0EC010E943647843166
:108E900081F0882371F0883161F08C3161F4E881D0
:108EA000F9810084F185E02DCE01199521E0892B0F
:108EB00019F420E001C021E0822F01C080E0DF91A1
:108EC000CF910895CF92DF92EF92FF921F93CF93AD
:108ED000DF93FC0114851430A9F1EC0180E590E0EA
:108EE0000E94AB2768E070E0812F0E94D0320E9480
:108EF000AA270E9471536B017C01CE010E94364764
:108F00008823B1F061E070E080E090E00E94375388
:108F10000E947153DC01CB018C199D09AE09BF0978
:108F2000883E9340A105B10540F38C850E94954E83
:108F3000EC85F0E0EE0FFF1FE95DF44F1182108227
:108F400084E08C87DF91CF911F91FF90EF90DF90AD
:108F5000CF9008952F923F924F925F926F927F929F
:108F60008F929F92AF92BF92CF92DF92EF92FF9239
:108F70000F931F93CF93DF93CDB7DEB72B970FB629
:108F8000F894DEBF0FBECDBF8C012B010E949C3632
:108F9000019609F4D3C2D801ED91FC910284F385C6
:108FA000E02DC80119957C018F3FBFEF9B0709F4A5
:108FB000C5C2D801ED91FC910684F785E02D682F9C
:108FC000C8011995B2E2EB16F10429F4B201C80107
:108FD0000E94B622B5C2EDE2EE16F10429F0C701F7
:108FE000C0970A9708F045C1D801ED91FC91028421
:108FF000F385E02DC80119951C018F3FBFEF9B073A
:1090000009F49CC28D9781F4D801ED91FC91028402
:10901000F385E02DC80119951C01019609F48EC253
:1090200088248A94982C03C088248394912CC101AD
:10903000C097C12CD12C0A97C8F48AE0F82EFC9C6A
:10904000C001FD9C900D1124B101605371096C01A8
:10905000C60ED71ED801ED91FC910284F385E02D58
:10906000C80119951C01C0970A9748F3BEE22B1658
:109070003104C1F0C1018F7D8534910599F0C89C00
:10908000C001C99C900DD89C900D1124092E000C94
:10909000AA0BBB0BF20181879287A387B48782E07A
:1090A0008087DDC0B601DD0C880B990B0E945762EA
:1090B0006B017C01FEE22F163104B1F5D801ED9170
:1090C000FC910284F385E02DC80119951C01A12CA7
:1090D000B12C20E030E040E251E4C701B6010E942B
:1090E0000C636B017C01B10160537109072E000C08
:1090F000880B990B0E9457629B01AC01C701B60116
:109100000E943C616B017C01B1E0AB1AB108D8014F
:10911000ED91FC910284F385E02DC80119951C01A5
:10912000C0970A97B0F202C0A12CB12CC1018F7D6B
:109130008534910509F043C0D801ED91FC9102847A
:10914000F385E02DC80119951C018B32910559F466
:10915000D801ED91FC910284F385E02DC8011995A9
:109160001C01B1E00CC08D9761F4D801ED91FC9128
:109170000284F385E02DC80119951C01BFEFBE8361
:1091800002C0E1E0EE83612C712C4AE0C101C0977E
:109190008A309105C0F4469D9001479D300D112401
:1091A0003901680E791ED801ED91FC910284F38596
:1091B000E02DC8014B8719951C014B85E7CFB1E025
:1091C000BE83612C712CB401990C880B990B0E9401
:1091D0005762A70196010E940C636B017C01B501E7
:1091E000BB0C880B990B0E9457624B015C01B301C9
:1091F000770C880B990B0E9457626F837887898759
:109200009A87EE816E2FEE0F770B880B990B0E94D9
:1092100057629B01AC016F81788589859A850E9490
:109220000C639B01AC01C501B4010E943C619B0130
:10923000AC0160E070E080E291E40E9479639B0100
:10924000AC01C701B6010E940C63D20119966D935F
:109250007D938D939C931C9783E018968C93D801F3
:10926000ED91FC910684F785E02D622DC8011995DA
:1092700022C0BBE5EB16F10409F060C0D801ED9106
:10928000FC910284F385E02DC80119958B35910579
:1092900009F054C185E0F2018087C8010E949C3624
:1092A000D801ED91FC910284F385E02DC801199558
:1092B0008D35910519F480E090E042C1D801ED911F
:1092C000FC910684F785E02D682FC8011995DD24EF
:1092D000DA940E946C237C01009709F42FC1DD20F1
:1092E00021F0F2019783868308C0D50113969C93E1
:1092F0008E931297FC01B582A482C8010E949C360D
:10930000B701C8010E94AA47892B09F017C1C801FB
:109310000E949C36D801ED91FC910284F385E02DEA
:10932000C8011995D12C57018C32910591F221E099
:1093300030E08D35910509F089C086C0BBE7EB169A
:10934000F10409F088C0D801ED91FC910284F38505
:10935000E02DC80119958B37910509F0EFC086E023
:10936000F2018087C8010E949C36D801ED91FC91E2
:109370000284F385E02DC80119958D37910509F414
:109380009ACFD801ED91FC910684F785E02D682FE6
:10939000C8011995BB24BA940E946C237C010097E4
:1093A00009F4CCC0BB2021F0F2019783868308C06A
:1093B000D60113969C938E931297FC01D582C4829A
:1093C000C8010E949C36B701C8010E94B6220196CE
:1093D00009F4B4C0C8010E949C36D70119968D913A
:1093E0009C911A9711969C938E931A961C921E929A
:1093F0001997D801ED91FC910284F385E02DC80105
:109400001995CA9709F09AC0C8010E949C36B70105
:10941000C8010E94AA47019609F490C0C8010E94A1
:109420009C36D801ED91FC910284F385E02DC801B2
:109430001995B12C67018C32910509F4ADCF21E06B
:1094400030E08D37910511F420E030E0882799272E
:10945000821B930B75C0BEE6EB16F10411F5198261
:109460001A821B821C82D801ED91FC910484F5853F
:10947000E02D44E050E0BE016F5F7F4FC8011995B9
:10948000049709F05BC044E050E06AEA74E0CE0162
:1094900001960E948565009709F050C0F201108680
:1094A0004FC0F6E6EF16F10419F5CE0101967C01E6
:1094B00085E0D7011D928A95E9F7D801ED91FC91DD
:1094C0000484F585E02D45E050E0B701C801199509
:1094D0000597A1F545E050E064EB74E0C7010E94F8
:1094E0008565009759F521E0F2012087118628C093
:1094F000F4E7EF16F10411F519821A821B821C821F
:10950000D801ED91FC910484F585E02D44E050E014
:10951000BE016F5F7F4FC8011995049779F444E04D
:1095200050E06FEA74E0CE0101960E9485650097D5
:1095300029F421E0F2012087218702C08FEF9FEFFD
:109540002B960FB6F894DEBF0FBECDBFDF91CF9143
:109550001F910F91FF90EF90DF90CF90BF90AF9051
:109560009F908F907F906F905F904F903F902F9043
:109570000895CF92DF92EF92FF920F931F93CF93B4
:10958000DF9300D01F92CDB7DEB78C017B0129831A
:109590003A834B835C830E946C236C0129813A815E
:1095A0004B815C81892B19F183E0F601808721874B
:1095B00032874387548780819181009711F00E9400
:1095C000DA66C7010E940365F60191838083B601C4
:1095D000C8010F900F900F900F90DF91CF911F91C6
:1095E0000F91FF90EF90DF90CF900C943B1C0F9069
:1095F0000F900F900F90DF91CF911F910F91FF90DF
:10960000EF90DF90CF900895FB0101900020E9F7E3
:109610003197AF01461B570B20E00C9438200F9375
:109620001F93CF93DF93EC012097F9F00A811B8100
:10963000888587FD06C08E819F81009711F00E946A
:109640000F4B8885843031F489859A85009711F015
:109650000E94DA6688819981009711F00E94DA668B
:10966000CE010E94DA66E801DFCFDF91CF911F9132
:109670000F9108950F931F93CF93DF93009791F06D
:109680008C010E946C23EC01892B61F0C8010E94BF
:109690009C36BE01C8010E94AA47019631F4CE0152
:1096A0000E940F4B80E090E001C0CE01DF91CF918E
:1096B0001F910F910895382F2091790B9091780B7D
:1096C000213208F049C08091550B8111FCCF42E056
:1096D0004093550B3093540B3FEF3093530B109244
:1096E000520B2093510BA8E5BBE041E35BE0FA018C
:1096F0003E2F341B321718F43D913193F9CF10925D
:10970000300B2091300B990F922B9093300B90914E
:109710002F0B913061F410922F0B9091300B90939E
:10972000BB009091BC0093FDF8CF95EC01C095EE85
:109730009093BC009091550B9230E1F39091530BB4
:109740009F3F79F08091530B803241F08091530B11
:10975000803331F084E005C081E003C082E001C0C5
:1097600083E01092570B1092790B1092560B0895CC
:10977000DF92EF92FF920F931F93CF93DF93CDB7BA
:10978000DEB729970FB6F894DEBF0FBECDBF8C01B0
:109790007B01AE014F5F5F4F0E944741D82E882367
:1097A00009F459C0F7018081803109F454C08FE178
:1097B0008D83F801858196810E944942B701F801A5
:1097C000858196810E94744340E06EE4F8018581B2
:1097D00096810E948A4240E06B81F80185819681E2
:1097E0000E948A4240E06C81F801858196810E9446
:1097F0008A42F7018081803139F040E06D81F801C3
:10980000858196810E948A42F801858196810E9415
:109810004942B701F801858196810E947443F8019D
:10982000408168E4858196810E948A4264E170E00B
:1098300080E090E00E943753F8018081882331F066
:109840006AE070E080E090E00E943753F801858183
:1098500096810E9449428D2D29960FB6F894DEBF5D
:109860000FBECDBFDF91CF911F910F91FF90EF9071
:10987000DF900895EF92FF920F931F93CF93DF93A2
:10988000EC018C01085F1F4F7E01699170E084E05C
:10989000759567958A95E1F740E150E081EC96E097
:1098A0000E948C16F70160816F7070E040E150E01B
:1098B00081EC96E00E948C16C017D10729F7DF9142
:1098C000CF911F910F91FF90EF900895CF92DF926B
:1098D000EF92FF92CF93DF93EC010E9471536B01E3
:1098E0007C0180915E0790915F07DC01ED91FC9116
:1098F0000084F185E02D1995892B79F40E9471532C
:10990000AB01BC014C195D096E097F0948395A4306
:109910006105710530F380E00DC080915E07909184
:109920005F07DC01ED91FC910284F385E02D199530
:10993000888381E0DF91CF91FF90EF90DF90CF900F
:1099400008950895CF93DF931F92CDB7DEB7698353
:10995000DC01ED91FC910280F381E02D41E050E0CB
:10996000BE016F5F7F4F19950F90DF91CF910895E2
:10997000BF92CF92DF92EF92FF920F931F93CF93FC
:10998000DF9300D000D0CDB7DEB7FC01208D2430AE
:1099900009F053C06A017B018C01B12C63E070E0D7
:1099A0008B2D0E948746811103C0F801B08E06C03E
:1099B0008831D9F3B394F4E0BF12F0CFF801808D71
:1099C0008430D9F196E0ECEBF3E0DE0111960190E2
:1099D0000D929A95E1F7F70193819F779C8394818B
:1099E0009D8395819E83B7016E5F7F4F90E0982F96
:1099F000882744E050E0845F9B4F0E944D40B601B1
:109A0000F801808D0E94E546F801808D90E0982F46
:109A1000882746E050E0BE016F5F7F4F8A5F9B4F13
:109A20000E944D40F801128E118E20E8A60162E0DE
:109A3000808D0E949F4081E001C080E026960FB695
:109A4000F894DEBF0FBECDBFDF91CF911F910F9174
:109A5000FF90EF90DF90CF90BF900895CF93DF936A
:109A60001F92CDB7DEB7FC01218D328D232B49F03B
:109A7000BE016F5F7F4F808D0E94E440898190E03E
:109A800002C08FEF9FEF0F90DF91CF910895AF92BB
:109A9000BF92CF92DF92FF920F931F93CF93DF93EA
:109AA0008C015B01EA01FC01C688D788F08C80E557
:109AB00090E00E94AB278F2D0E94AD338C179D073D
:109AC00020F48F2D0E94AD33EC019E01A501B6015B
:109AD0008F2D0E9448330E94AA27F8018689978912
:109AE0008C0F9D1F978B868BCE01DF91CF911F919D
:109AF0000F91FF90DF90CF90BF90AF900895FF92AD
:109B00000F931F93CF93DF93F82E80E590E00E9490
:109B1000AB27C0E0D0E08F2D0E94E63F8C01892B5F
:109B200021F08F2D0E94E63FEC01C017D10799F775
:109B30000E94AA27CE01DF91CF911F910F91FF9034
:109B40000895AF92BF92CF92DF92EF92FF921F9350
:109B5000CF93DF93182F5B017A0180E590E00E949C
:109B6000AB27C0E0D0E0812F0E94E63F6C01892B3B
:109B700021F0812F0E94E63FEC01CC15DD0599F71D
:109B8000209799F463E070E0812F0E94874684312A
:109B9000F1F08823E1F0C1E0D0E08C3111F4C0E0B5
:109BA000D0E0D195C195D10912C0EC16FD060CF498
:109BB000E7011C161D065CF420E0AE01B501812F03
:109BC0000E94E03260E470E0812F0E94D0320E9457
:109BD000AA27CE01DF91CF911F91FF90EF90DF90E8
:109BE000CF90BF90AF900895CF93DF93FC01218D6C
:109BF000328D2115310519F48FEF9FEF11C0EC0163
:109C00004217530708F0A901888D0E94A14D18162C
:109C1000190694F7298D3A8D281B390B3A8F298F15
:109C2000DF91CF9108950F931F93CF93DF931F92EE
:109C3000CDB7DEB7FC01218D328D232B61F08C0175
:109C400041E050E0BE016F5F7F4F808D0E94A14DCB
:109C5000181619061CF08FEF9FEF08C0F801818DD0
:109C6000928D0197928F818F898190E00F90DF9183
:109C7000CF911F910F9108950F931F93CF93DF936F
:109C8000CDB7DEB728970FB6F894DEBF0FBECDBFB5
:109C90008C01F801818D928D892B49F0D801ED91CD
:109CA000FC910284F385E02DC8011995F2CF808DD7
:109CB0000E947F4D181619065CF548E050E0BE0181
:109CC0006F5F7F4FD80158968C910E94A14D9C01E7
:109CD00018161906DCF489819A81AB81BC81F801E0
:109CE000808B918BA28BB38B8D8190E0982F8827EE
:109CF0002E81820F911D958B848B2F8130E0322F26
:109D000022278885280F311D328F218FC90102C07B
:109D100080E090E028960FB6F894DEBF0FBECDBF6E
:109D2000DF91CF911F910F910895CF93C82F80E5B8
:109D300090E00E94AB2760E170E08C2F0E94D0324F
:109D40004FEF62E070E08C2F0E947D46CF910C9423
:109D5000AA271F93CF93DF931F92CDB7DEB7182F9B
:109D600080E590E00E94AB2763E070E0812F0E94C5
:109D7000874689830E94AA2789810F90DF91CF911E
:109D80001F9108958F929F92AF92BF92CF92DF92D0
:109D9000EF92FF920F931F93CF93DF93E62EB72E90
:109DA000D42EA52EC22E932EF02E812EBC01809192
:109DB0004205909143050E94FD1BEC01892B09F49B
:109DC00054C08885853009F050C060E0CE010E9403
:109DD000F01B8C0161E0CE010E94F01BDC011996A2
:109DE000CD91DC911A97D8011996ED91FC911A97B3
:109DF000E130F10561F02CF4EF2BB9F56F2DCE01B8
:109E000017C0E230F10541F03797A9F02EC06F2D51
:109E1000CE0103960E94C3296E2DCE010E94C32954
:109E20006D2DCE0101960E94C3296C2DCE010296A4
:109E30000E94C3291AC00097C1F0FC0180858530BB
:109E4000A1F4C681D781209781F00F2D182D2C2DDC
:109E5000392D4D2D5A2D6E2D7B2D89859A850E9489
:109E6000C24E0A80DB81C02DEECFDF91CF911F91D2
:109E70000F91FF90EF90DF90CF90BF90AF909F90A9
:109E80008F900895CF92DF92EF92FF920F931F93DE
:109E9000CF93DF93E091B60AF091B70A309791F033
:109EA0009085953079F469017A01EB01682FCF0133
:109EB0000E94F01B9601A701BE01FC0181859285DD
:109EC0000E94C24EDF91CF911F910F91FF90EF90B2
:109ED000DF90CF900895AF92BF92CF92DF92EF9232
:109EE000FF920F931F93CF93DF93E1E0F0E0C0E088
:109EF000D0E0CC24C394D12C40917E0B50917F0BA9
:109F0000B6010C2E02C0660F771F0A94E2F77F019C
:109F100084E0E80EF11CCF01B12C9C01A091060257
:109F2000B0910702A817B90720F4209106023091DA
:109F30000702A0919E0AB0919F0AA20FB31FAC9096
:109F4000A091B20AB091B30A9C0121503109A20F2D
:109F5000B31F0A2D10E02C9130E00217130729F0EF
:109F6000462B572BAC92BB24B39401968E159F05BC
:109F7000A1F650937F0B40937E0BBB2011F1809193
:109F8000B20A9091B30AE80FF91F028110E0218113
:109F900030E0408150E03197608170E0CE010E9456
:109FA000424F0E947153DC01CB01845D9E4FAF4F45
:109FB000BF4F80937A0B90937B0BA0937C0BB09355
:109FC0007D0B2196F701C430D10509F095CFDF91C3
:109FD000CF911F910F91FF90EF90DF90CF90BF90A6
:109FE000AF900895DC011296ED91FC911397309794
:109FF00021F081E09085953009F080E00895DC0142
:10A000001696ED91FC911797309739F08085823044
:10A0100021F441875287638774870895FC01868104
:10A020009781009789F0FC012085223041F025308E
:10A0300079F460E00E94F01B009779F0FC016185E3
:10A0400072858385948508956FEF7FEFCB01089526
:10A050006EEF7FEF8FEF9FEF08956DEF7FEF8FEF44
:10A060009FEF0895FC0184819581009761F0FC01C8
:10A070002085223029F0253049F40E94F01BFC0194
:10A080008185928508958FEF9FEF08958EEF9FEF62
:10A090000895CF93C62F63E0FC01828193810E94D3
:10A0A000F01B009749F04C2F50E060E070E0FC019D
:10A0B0004187528763877487CF91089563E0FC01DD
:10A0C000828193810E94F01B009719F0FC01818529
:10A0D00008958FEF08958F929F92BF92CF92DF9253
:10A0E000EF92FF920F931F93CF93DF93EC010E94A7
:10A0F000F24F882309F445C08A819B810E94631F27
:10A10000082F10E06801CC0CDD1CE12CF12C92E052
:10A11000B92E0430110504F5F701EC0DFD1DEE53C9
:10A12000FC4F808091800E946C23009751F0FC01CD
:10A13000B086A401990C660B770B41875287638721
:10A140007487BC018A819B810E943B1C0F5F1F4F5B
:10A15000F2E0EF0EF11CDDCF0A811B8160E0C80147
:10A160000E94F01BFC018185888761E0C8010E9484
:10A17000F01B9D838C8362E0C8010E94F01B9F83CB
:10A180008E83DF91CF911F910F91FF90EF90DF9021
:10A19000CF90BF909F908F900895CF93DF93EC0165
:10A1A00082E292E0998388836115710549F080917C
:10A1B0004205909143050E94FD1B9B838A8302C048
:10A1C0001B821A82CE01DF91CF910C946B50CF93FA
:10A1D000DF93EC0167E374E00E946565892B51F120
:10A1E0006AE374E0CE010E946565892B31F165E078
:10A1F00075E0CE010E946565892B11F16AE075E07A
:10A20000CE010E946565892BF1F061E175E0CE0118
:10A210000E946565892BD1F088818D32D1F090ED57
:10A22000980F9A30B0F08B37B9F08332C1F48DEFCC
:10A230009FEF17C081E090E014C082E090E011C071
:10A2400083E090E00EC084E090E00BC085E090E0F9
:10A2500008C080E090E005C08EEF9FEF02C08FEF56
:10A260009FEFDF91CF910895EF92FF920F931F938D
:10A27000CF93DF9380917E0B90917F0BC4E0D0E071
:10A2800021E030E0A90148235923452B29F0A901F9
:10A290004095509584239523220F331F219791F7E2
:10A2A00090937F0B80937E0B0E94715300917A0BE9
:10A2B00010917B0B20917C0B30917D0B6017710707
:10A2C0008207930708F45BC0012B022B032B09F4D0
:10A2D00056C010927A0B10927B0B10927C0B10924E
:10A2E0007D0BE12CF12CE091B20AF091B30AEC0F56
:10A2F000FD1F038110E0228130E0418150E0608148
:10A3000070E0C7010E94424F8FEFE81AF80A2496C6
:10A3100084E0E816F10439F7C1E0D0E0809106024C
:10A32000909107028C179D0728F480910602909166
:10A33000070201C0CE0120919E0A30919F0AF901C7
:10A34000E80FF91F408150E060E070E02AE081EC06
:10A3500096E00E94F91566E175E081EC96E00E94B6
:10A36000B2172196C131D105C9F681EC96E0DF9193
:10A37000CF911F910F91FF90EF900C94D916DF9120
:10A38000CF911F910F91FF90EF900895BC01823003
:10A39000910508F40895613E8EE1780748F49B0129
:10A3A00095E0369527959A95E1F748E0420F01C070
:10A3B0004FEF91E0242F30E0290F311D359527957F
:10A3C000229FF001239FF00DF00D11246E177F07DF
:10A3D00018F44FEF420F05C02F3F310539F091E0DF
:10A3E000920F491738F78FEF890F08958FEF08956F
:10A3F00090E0FC013197E231F10508F04EC088276A
:10A40000E552FF4F8F4F0C941161809180008F7740
:10A4100003C0809180008F7D80938000089580919B
:10A420008000877FF9CF84B58F7702C084B58F7D98
:10A4300084BD08958091B0008F7703C08091B000F3
:10A440008F7D8093B0000895809190008F7707C032
:10A45000809190008F7D03C080919000877F8093D2
:10A46000900008958091A0008F7707C08091A00090
:10A470008F7D03C08091A000877F8093A000089506
:10A48000809120018F7707C0809120018F7D03C0CC
:10A4900080912001877F8093200108953FB7F89431
:10A4A0008091850B9091860BA091870BB091880BC2
:10A4B00026B5A89B05C02F3F19F00196A11DB11D1F
:10A4C0003FBFBA2FA92F982F8827820F911DA11D5A
:10A4D000B11DBC01CD0142E0660F771F881F991F97
:10A4E0004A95D1F70895CF93DF931F92CDB7DEB78A
:10A4F00069832091560B2223D1F02091790B2032D1
:10A5000040F021E030E0FC013383228380E090E0E2
:10A5100015C08091570BE82FF0E0E85AF44F99816D
:10A5200090838F5F8093570B8093790B05C061E018
:10A53000CE0101960E94D34481E090E00F90DF911C
:10A54000CF910895CF93DF93282F30E0F901EA5E91
:10A55000F24F8491F901E359F64FD491F901E35395
:10A56000F64FC491CC2391F081110E94F851EC2F49
:10A57000F0E0EE0FFF1FE450F34FA591B491EC9182
:10A58000ED2381E090E021F480E002C080E090E0E3
:10A59000DF91CF9108951F93CF93DF93282F30E061
:10A5A000F901EA5EF24F8491F901E359F64FD49133
:10A5B000F901E353F64FC491CC23C9F0162F811152
:10A5C0000E94F851EC2FF0E0EE0FFF1FED54F64F14
:10A5D000A591B4918FB7F894111105C09C91ED2FFE
:10A5E000E095E92302C0EC91ED2BEC938FBFDF9156
:10A5F000CF911F910895CF93DF9390E0FC01E35931
:10A60000F64F2491FC01E353F64F8491882361F1C6
:10A6100090E0880F991FFC01EE51F34FC591D49142
:10A62000FC01ED54F64FA591B491611109C09FB79B
:10A63000F8948881209582238883EC912E230BC087
:10A64000623061F49FB7F8943881822F809583231C
:10A650008883EC912E2B2C939FBF06C08FB7F89464
:10A66000E8812E2B28838FBFDF91CF9108958F92A1
:10A670009F92AF92BF92CF92DF92EF92FF926B01C7
:10A680007C010E944E524B015C01C114D104E104D3
:10A69000F104F1F00E944E52DC01CB0188199909B6
:10A6A000AA09BB09883E9340A105B10570F321E0DA
:10A6B000C21AD108E108F10888EE880E83E0981EDE
:10A6C000A11CB11CC114D104E104F10419F7DDCFC0
:10A6D000FF90EF90DF90CF90BF90AF909F908F90C2
:10A6E00008952FB7F8946091810B7091820B80913F
:10A6F000830B9091840B2FBF08951F920F920FB67A
:10A700000F9211242F933F938F939F93AF93BF93F7
:10A710008091810B9091820BA091830BB091840B5F
:10A720003091800B23E0230F2D3720F40196A11DDB
:10A73000B11D05C026E8230F0296A11DB11D20936F
:10A74000800B8093810B9093820BA093830BB0932B
:10A75000840B8091850B9091860BA091870BB09113
:10A76000880B0196A11DB11D8093850B9093860BDC
:10A77000A093870BB093880BBF91AF919F918F915E
:10A780003F912F910F900FBE0F901F901895CF9370
:10A79000DF93C1E1D0E068EE73E080E090E00E94DA
:10A7A00037534AE050E0BE0181EC96E00E94DD168E
:10A7B000219789F7DF91CF9108950E946C1966E780
:10A7C0007DE081EC96E00C940617AF92BF92CF9299
:10A7D000DF92EF92FF920F931F93CF93DF93CDB74A
:10A7E000DEB7C154D1090FB6F894DEBF0FBECDBF9E
:10A7F000CB018A014EE459E46CE470E049835A834A
:10A800006B837C83FE0135962CE1DF011D922A9536
:10A81000E9F74AAB5BAB6CAB7DABF1962CE0DF01AB
:10A820001D922A95E9F7AE014F5D5F4F68E00E94E7
:10A83000E5181AAABE016F5D7F4F80914405909183
:10A8400045050E94FD1B7C01009771F162E374E0F5
:10A850000E94FD1BFC01C184D284C114D104C9F043
:10A8600041E150E0B601CE0181960E949365B601A8
:10A8700081EC96E00E94B21764E77DE081EC96E0FF
:10A880000E94C0154AE050E0B80181EC96E00E94B9
:10A89000DD1663E274E0C7010E94FD1BDC0119961E
:10A8A000ED90FC901A9708C06BE67DE081EC96E095
:10A8B0000E940617E12CF12C0138BFEF1B0709F4A9
:10A8C000C7C00535110509F4C3C00115110509F408
:10A8D000BFC06CE57DE0CE0101960E94F36740E2C7
:10A8E00050E0BE016F5D7F4FCE0101960E947565FD
:10A8F0001F930F9383EA94E09F938F936E01E2E39B
:10A90000CE0ED11CDF92CF920E94EA65B601CE0135
:10A9100001960E94044B0F900F900F900F900F9094
:10A920000F90E114F10409F493C0809142059091D5
:10A930004305009709F48CC0B7010E94FD1B7C0100
:10A94000009709F485C0DC0118968C91853009F0D8
:10A950007FC060E0C7010E94F01BFC0181859285E9
:10A96000A385B4850597A105B10509F071C0C7019C
:10A970000E94631F843008F46BC08430B1F50E94DC
:10A980006C236C01892B21F085E0D60118968C93FD
:10A990000E946C235C01892B59F082E0F5018087CD
:10A9A000012E000C220B330B01871287238734877B
:10A9B0000E946C238C01892B59F082E0F80180877A
:10A9C00088EC90E0A0E0B0E081879287A387B4870D
:10A9D000B501C6010E943B1CB801C6010E943B1C88
:10A9E000B601C7010E943B1C33C064E0C7010E944E
:10A9F000F01B6C01009761F161E00E94F01B5C01AB
:10AA000060E0C6010E94F01B012E000C220B330BEC
:10AA1000DC0119960D931D932D933C931C97F50122
:10AA200081859285A385B485892B8A2B8B2B39F45C
:10AA3000D7016D917C9188E195E00E94044B88ECF0
:10AA400090E0A0E0B0E0F50181879287A387B4870A
:10AA5000CF5BDF4F0FB6F894DEBF0FBECDBFDF91E7
:10AA6000CF911F910F91FF90EF90DF90CF90BF900B
:10AA7000AF900895CF93DF93CDB7DEB7CB57D10911
:10AA80000FB6F894DEBF0FBECDBF789484B5826058
:10AA900084BD84B5816084BD85B5826085BD85B582
:10AAA000816085BD80916E00816080936E00109200
:10AAB000810080918100826080938100809181007B
:10AAC000816080938100809180008160809380000C
:10AAD0008091B10084608093B1008091B00081606A
:10AAE0008093B0008091910082608093910080916A
:10AAF00091008160809391008091900081608093AB
:10AB000090008091A10082608093A1008091A100BB
:10AB100081608093A1008091A00081608093A0005B
:10AB200080912101826080932101809121018160C7
:10AB30008093210180912001816080932001809188
:10AB40007A00846080937A0080917A00826080939A
:10AB50007A0080917A00816080937A0080917A00F7
:10AB6000806880937A001092C10087E495E090930A
:10AB700084058093830510928C0A10928B0A26E03C
:10AB800040E052EC61E070E081EC96E00E946C18CD
:10AB90006DED73E58AEC93E00E94283564E777E178
:10ABA0008FEC93E00E94283565E77BE384ED93E02A
:10ABB0000E94283563EE7BE189ED93E00E94283501
:10ABC00068E177E18DED93E00E94283567EC73E54D
:10ABD00081EE93E00E94283566E179E186EE93E00C
:10ABE0000E9428350E946C1986E0E2E1F2E0DE0165
:10ABF000119601900D928A95E1F748E2C42E45E046
:10AC0000D42EF12C00E010E0C8010E94E96ED601BC
:10AC10008D936D0181508E3F10F4FF24F3940F5FEC
:10AC20001F4F0630110581F7F1100FC064EC74E07E
:10AC300081EC96E00E94061786E0FE013196A8E2BC
:10AC4000B5E001900D928A95E1F70E941D2D60E01C
:10AC500070E080E090E00E94163B61E08DE00E9491
:10AC6000FB5226E040E855E260E070E084E296E0C6
:10AC70000E946C1888EA95E19093100980930F095F
:10AC800085EB95E1909312098093110981EB95E191
:10AC9000909314098093130964E170E080E090E0E0
:10ACA0000E94375310924605E0913005F09131052E
:10ACB000309721F084EA95E1908B878780E99AE2CA
:10ACC0009093EC078093EB07A89581EC96E00E94A7
:10ACD000C514892B09F493C081EC96E00E94A3145B
:10ACE000182F8A3031F08D3021F0883009F076C08D
:10ACF00060C0E0918305F091840510826AEE73E0F4
:10AD000081EC96E00E94B2176DEE73E087E495E067
:10AD10000E9409689A838983FE0133967F0101E0CE
:10AD200010E0D02EC12E6DEE73E080E090E00E9426
:10AD30000968D7018D939D937D010E31110539F47A
:10AD400000918D0A10918E0AE980FA8008C00F5F89
:10AD50001F4F892B31F7F4CFF801048115810115BC
:10AD60001105A1F0F80160817181C7010E9465653C
:10AD7000892B91F7D8011296ED91FC911397BE01A2
:10AD80006F5F7F4F8D2D9C2D199506C064EE74E08A
:10AD900081EC96E00E94061781EC96E00E94D9169D
:10ADA00064EF74E081EC96E00E94C01587E495E0C2
:10ADB00010C068E081EC96E00E94B915809183058F
:10ADC00090918405F5E087349F0709F008F47DCF62
:10ADD0000197909384058093830577CF682F81EC4A
:10ADE00096E00E94B915E0918305F0918405CF01AA
:10ADF00001969093840580938305108366CF0E940B
:10AE0000A90E029714F00E94833180914605882391
:10AE100009F48BC28091440590914505892B09F472
:10AE200084C20E947153009187051091880520917A
:10AE3000890530918A05601771078207930708F426
:10AE400074C20E9471532B013C018091380590918E
:10AE50003905009709F457C2209185053091860580
:10AE60006091360570913705261737070CF42BC112
:10AE70000E9471539B01AC0128573C4E4F4F5F4FCE
:10AE8000EC962CAF3DAF4EAF5FAFEC9761E275E053
:10AE900081EC96E00E940617E0913005F0913105B3
:10AEA000309739F4E0912E05F0912F0580E090E085
:10AEB0000BC08FEF83871486DF0113963B961D929C
:10AEC000AE17BF07E1F7EECF209136053091370579
:10AED000821793070CF081C0208131812E7F21934E
:10AEE00031930196F1CF6091360570913705F3E00B
:10AEF000660F771FFA95E1F72091340530913505FB
:10AF0000620F731F0E94B34218160CF0E5C6C09082
:10AF10003605D0903705B4E1CB16D1040CF0DCC671
:10AF20000E947153EC962CAD3DAD4EAD5FADEC97EC
:10AF3000621773078407950708F0CEC6A090340502
:10AF4000B0903505760133E0EE0CFF1C3A95E1F741
:10AF5000EA0CFB1C67E0C7010E943A41D701179633
:10AF60009C9189133AC000E010E00C151D05ECF52A
:10AF700048E050E0B701C5010E941D65B8E0AB0E86
:10AF8000B11C892BC9F5000F111FE0912E05F0911E
:10AF90002F05E00FF11F8081918181609183808373
:10AFA0006AE175E081EC96E00E94C015809136055B
:10AFB0009091370523E0880F991F2A95E1F720919A
:10AFC000340530913505820F931F0E943A4C63E19E
:10AFD00075E081EC96E00E94061780913005909113
:10AFE0003105009709F07FCF77C6809138059091A1
:10AFF0003905892B21F4F1CF0F5F1F4FB6CFE091B8
:10B000003605F0913705EE0FFF1F80912E059091C8
:10B010002F05E80FF91F21E030E0318320836EE037
:10B0200075E081EC96E00E94C01560913605709144
:10B0300037054AE050E081EC96E00E948C1667E00C
:10B0400075E081EC96E00E94C015809136059091E4
:10B050003705B3E0880F991FBA95E1F720913405C1
:10B0600030913505820F931F0E943A4C81EC96E097
:10B070000E94D916609136057091370513E0660F6E
:10B08000771F1A95E1F78091340590913505680F87
:10B09000791FDB018C91883261F4809138059091A1
:10B0A00039050E94B84B80913005909131050E947E
:10B0B0007E42809136059091370501969093370531
:10B0C000809336058ACF0091340510913505A9018A
:10B0D000E3E0440F551FEA95E1F7040F151FD8016F
:10B0E0004C91483209F004C1AE01435C5F4FB80196
:10B0F0000E944741882381F16DADB8E06B9FB0019C
:10B1000011248EAD282F30E0322F2227330F330F3A
:10B11000330F262B372BF8018081803101F52596DE
:10B120006FAD259770E024968FAD2497AB01481B37
:10B130005109CA019695982F8827979587950E945F
:10B14000FD6060517109207F13E0220F331F1A95B3
:10B15000E1F7620F731F04C060E874EE01C0B9012B
:10B16000613854EE75076CF0072E000C880B990BB4
:10B170000E94576220E030E040E05CE30E940C63F4
:10B1800004C060E070E08EEF92EC0E941F62E091DC
:10B190003205F09133053097A1F0009185051091AB
:10B1A00086059801A3E0220F331FAA95E1F7A0912D
:10B1B0003405B09135052A0F3B1FAB01B901C80119
:10B1C0001995009185051091860553E0000F111F18
:10B1D0005A95E1F78091340590913505080F191FB4
:10B1E000E0903805F0903905D8018C91803149F014
:10B1F000B801C7010E94FA29D82E882309F46CC02F
:10B2000002C04CE0D42EF701858196810E9449420C
:10B21000882309F461C0B801D70115968D919C91DE
:10B2200016970E947443F701408164E485819681FA
:10B230000E948A42D70112968C91882309F44CC04F
:10B24000E7EFED0DE33040F4F0E0EE0FFF1FE85EB6
:10B25000FD4FC080D18004C02EEEC22E22E0D22E3F
:10B260000115110599F1F7018381882379F1808116
:10B2700081112CC00E9471534B015C019601DD0CC1
:10B28000440B550BEC962CAF3DAF4EAF5FAFEC9738
:10B29000AE01435C5F4FB801C7010E94282A8DAD03
:10B2A00081111AC00E947153DC01CB01EC962CADC8
:10B2B0003DAD4EAD5FADEC97821B930BA40BB50B70
:10B2C00088159905AA05BB0518F306C0B601DD0C63
:10B2D000880B990B0E9437538091850590918605C4
:10B2E0000196909386058093850564EC79E00DC006
:10B2F0002F5F3F4F309386052093850580ED97E0C3
:10B300000E94FD6002C06FEF7FEFCB01770FAA0BA9
:10B31000BB0B480E591E6A1E7B1E40928705509239
:10B3200088056092890570928A050E943451809147
:10B33000420590914305892B09F42BC48091400567
:10B3400090914105049709F493C30E9471530091B1
:10B350008B0510918C0520918D0530918E05061777
:10B3600017072807390708F083C380E092E2292EE7
:10B3700092E0392EE0913C05F0913D05309709F4BB
:10B3800077C3811175C39085953009F05AC3AF9684
:10B390003FAE2EAEAF97E196FFAFEEAFE197CE0195
:10B3A00083599F4F0E946B500E9471532B013C01A7
:10B3B000E6968FADE697843061F008F42AC38830B2
:10B3C00009F427C3893009F4DDC0853009F026C3AC
:10B3D00020C380913A0590913B05892B09F0CAC0A2
:10B3E000CE0183599F4F0E94782F8111C3C041E045
:10B3F00050E050933B0540933A0560E070E0CE0189
:10B4000083599F4F0E9432506C0161E070E0CE0181
:10B4100083599F4F0E9432507C0126E240E855E25A
:10B4200060E070E084E296E00E946C18C092FD0734
:10B4300084E296E09093FC078093FB071092080942
:10B4400010920A0910920909F092FF07E092FE0794
:10B4500081E090E0909301088093000883E00E94CF
:10B46000921C182F811128C0009102081091030826
:10B4700068E475E081EC96E00E94C015E196EEADBF
:10B48000FFADE1976081718181EC96E00E94B21777
:10B4900061E475E081EC96E00E94C01540E150E067
:10B4A000B80181EC96E00E94DD16B801CE01835907
:10B4B0009F4F0E94D92E0DC06BE275E081EC96E0A3
:10B4C0000E94C01560E170E0812F0E94181C00E00E
:10B4D00010E010923B0510923A05A0903C05B09008
:10B4E0003D05D50112968D919C9113973EAE2DAEE0
:10B4F00021969FAF8EAF2197CE01CD960E946B50C3
:10B50000AB28C1F1CE01CD960E94F24F882391F174
:10B5100026968FAD2697843069F560E070E0CE0105
:10B52000CD960E9432508C159D0521F561E070E0AA
:10B53000CE01CD960E9432508E159F05D9F4B801E8
:10B54000CE01CD960E94D92EE0913C05F0913D05AB
:10B550008281938190933D0580933C05892B51F422
:10B56000E0914205F09143058681978190933D05D6
:10B5700080933C05CE0183599F4F0E947D2E80ED24
:10B5800097E04EC280913A0590913B05892B91F747
:10B59000CE0183599F4F0E94782F8111EBCFE1E0BC
:10B5A000F0E0F0933B05E0933A050E946C237C01A8
:10B5B000892B21F086E0D70118968C9361E975E01C
:10B5C000CE01CD960E94F367E196EEADFFADE19717
:10B5D000608171814FE150E0CE01CD960E9475658A
:10B5E0006FEE73E0CE01CD960E944F6526E040E8F5
:10B5F00055E260E070E084E296E00E946C1860E042
:10B6000070E0CE0183599F4F0E9432508093FD0716
:10B6100084E296E09093FC078093FB071092080960
:10B6200010920A0910920909E4E3F8E0F093FF0789
:10B63000E093FE072AE030E03093010820930008F1
:10B6400083E00E94921C182F8111ACC067E875E05E
:10B6500081EC96E00E94C01502E018E0D8016D91DF
:10B660007D918D0140E150E081EC96E00E948C16C6
:10B6700065E875E081EC96E00E94C015B8E00631FF
:10B680001B0761F76091060870910708072E000CF0
:10B69000880B990B0E94576220E030E048EC52E49E
:10B6A0000E94AD619B01AC0165EF73E0C7010E9490
:10B6B000B94A00910A0810910B08A80167EF73E0DE
:10B6C000C7010E94581C60910C0870910D08072E4C
:10B6D000000C880B990B0E94576220E030E048EC88
:10B6E00052E40E94AD619B01AC016BEF73E0C701B6
:10B6F0000E94B94A60910E0870910F08072E000C45
:10B70000880B990B0E94576220E030E040E251E440
:10B710000E94AD619B01AC0169EF73E0C7010E941B
:10B72000B94A40910208509103086DEF73E0C701D8
:10B730000E94581C012B89F1E3968EAD9FADE397D3
:10B74000FC012085253049F561E00E94F01B00973F
:10B7500021F124E630E0E8963FAF2EAFE897DC0118
:10B7600019966D917C911A97CE01835A9F4F0E9432
:10B77000CD50CE01835A9F4F0E94F24F882369F02B
:10B7800001E09E012A583F4F41E050E060E070E048
:10B79000CE01835A9F4F0E94660781EC96E00E947B
:10B7A000D9160BC06FE675E081EC96E00E94C015DB
:10B7B00060E170E0812F0E94181C8091020883FFD5
:10B7C00016C08EE398E09093FF078093FE07E1E0B8
:10B7D000F0E0F0930108E093000883E00E94921CDF
:10B7E00081110CC0409102085091030802C040E052
:10B7F00050E060E074E0C7010E94581C62E370E012
:10B8000080E090E00E94375383E190E09093FF073F
:10B810008093FE0784E090E09093010880930008F5
:10B8200083E00E94921C182F8111A5C065E675E087
:10B8300081EC96E00E94C01502E018E0D8016D91FD
:10B840007D918D014AE050E081EC96E00E948C16DB
:10B8500063E675E081EC96E00E94C015B8E00A301E
:10B860001B0761F7009102081091030801151105EB
:10B87000D1F0B801012E000C880B990B0E94576281
:10B880002DEE3EE94CE35EE30E940C6322E538EBCB
:10B8900042E152E40E943B619B01AC016DED73E01B
:10B8A000C7010E94B94A6091040870910508072EEB
:10B8B000000C880B990B0E9457622DEE3EE94CE379
:10B8C0005EE30E940C6322E538EB42E152E40E9401
:10B8D0003B614B015C019B01AC0163EF73E0C7016D
:10B8E0000E94B94A60910808709109081616170657
:10B8F000A4F4072E000C880B990B0E94576220E0DD
:10B9000030E040E251E40E94AD619B01AC0164E093
:10B9100074E0C7010E94B94A07C040E050E064E00B
:10B9200074E0C7010E94581C20E030E040E252E47D
:10B93000C501B4010E9407631816C4F4012BB1F0CD
:10B94000E196EEADFFADE1976081718188E094E012
:10B950000E94044B01E020E030E040E050E062E073
:10B9600070E0CE0183599F4F0E94660781EC96E0FC
:10B970000E94D9160BC06DE475E081EC96E00E9440
:10B98000C01560E170E0812F0E94181C80E091E0FA
:10B990000E9445668C01892B61F1A1961FAE1EAEF7
:10B9A000A197A3961FAE1EAEA3978FEF9FEFA5960C
:10B9B0009FAF8EAFA59788E292E06F969FAF8EAF54
:10B9C0006F97A7961FAE1EAEA797A9961FAF0EAF93
:10B9D000A99780E091E0AD969FAF8EAFAD97AB9603
:10B9E0001FAE1EAEAB97B701CE01835A9F4F0E9488
:10B9F0007E35B801CE01CD960E94044BC8010E944D
:10BA0000DA66C7010E940F4B10923B0510923A056F
:10BA1000B1CDCE0183599F4F0E947D2E84E690E0E8
:10BA2000092E000CAA0BBB0B480E591E6A1E7B1E6A
:10BA300040928B0550928C0560928D0570928E0518
:10BA400081E0E0913C05F0913D0522813381309306
:10BA50003D0520933C05232B09F08CCCE091420559
:10BA6000F09143058681978190933D0580933C0535
:10BA70000E94715300918F051091900520919105BE
:10BA800030919205601771078207930708F481C00F
:10BA9000E0914205F091430506811781812C011543
:10BAA000110509F43FC0F80180858530A9F560E0F3
:10BAB000C8010E94F01BFC0181859285A385B48595
:10BAC0000597A105B10541F5C8010E94631F8530A6
:10BAD00018F161E0C8010E94F01BFC01918462E052
:10BAE000C8010E94F01BDC011996CD90DC901A97DA
:10BAF00063E0C8010E94F01BFC01A184B28464E0F1
:10BB0000C8010E94F01B7C01892B31F0C7010E9403
:10BB1000631F823008F0F7C0D80112960D911C9176
:10BB20001397BDCF0E947153DC01CB0188579C4E07
:10BB3000AF4FBF4F80938F0590939005A0939105D1
:10BB4000B0939205882019F062EA75E002C060EABD
:10BB500075E081EC96E00E94C015AE01435C5F4F3A
:10BB600080918B0B90918C0B009711F485E99BE0F1
:10BB7000481B590B052E000C660B770B2AE081EC55
:10BB800096E00E94F9156DEE73E081EC96E00E945C
:10BB9000B21700913E0510913F050115110509F4FA
:10BBA00097C00E947153C0909305D0909405E09087
:10BBB0009505F0909605C616D706E806F90608F032
:10BBC00087C0F801E680F78083E0282EE114F104B5
:10BBD00009F46FC0D70118968C91863009F063C0C4
:10BBE00064E175E0C7010E94FD1B009719F0FC019C
:10BBF000018501C000E0D7018D919C910E94CC6726
:10BC0000182F61E274E0C7010E94FD1B6C01892BB3
:10BC100049F56EED75E081EC96E00E94C015412F6C
:10BC200050E060E070E02AE081EC96E00E94F915B7
:10BC30006CED75E081EC96E00E94C0156AE070E062
:10BC4000802F0E94181C40E050E061E274E0C701C0
:10BC50000E94581C61E274E0C7010E94FD1B6C0148
:10BC6000892B09F11123F9F007FF01C160E0812F51
:10BC70000E94FB52812F0E94A252332433940197D9
:10BC800009F001C1432C512CF6018485082E000CCB
:10BC9000990B4816590609F489C18385882309F44C
:10BCA000F4C081508387D7011296ED90FC901397D2
:10BCB0008DCF0E947153DC01CB01C296A11DB11D35
:10BCC0008093930590939405A0939505B093960562
:10BCD0000E946F150C94645668EF74E081EC96E056
:10BCE0000E94C01560913605709137054AE050E01A
:10BCF00081EC96E00E94DD16109286051092850573
:10BD000060E47FE102CB60E0C7010E94F01BDC0130
:10BD100019962D903D904D905C901C9761E0C70165
:10BD20000E94F01BFC012185328543855485D80192
:10BD30006D917C91211531054105510559F481EC36
:10BD400096E00E94B21761ED75E081EC96E00E94EA
:10BD5000061713C02150310941095109DC01199618
:10BD60002D933D934D935C931C97232B242B252BD4
:10BD700021F485E194E00E94044B3101B7E22B16D7
:10BD800031043CF0F8016081718188E094E00E9408
:10BD9000044BD8016D917C9181EC96E00E94B21722
:10BDA0006BEC75E081EC96E00E94C0154AE050E033
:10BDB000B60181EC96E00E948C1661EC75E081EC96
:10BDC00096E00E94C0154AE050E0B10181EC96E097
:10BDD0000E948C166BEB75E081EC96E00E94C0151A
:10BDE0004AE050E0B50181EC96E00E948C1661E0DB
:10BDF000892D0E94FB52B2E0AB16B10489F0E5E058
:10BE0000AE16B10469F061E0C7010E94F01BFC01AD
:10BE100081859285A385B485892B8A2B8B2B69F428
:10BE200060E0892D0E94CB5266EB75E081EC96E0D4
:10BE30000E940617882483946FCEB2E02B0E311C2B
:10BE40002C143D043CF461E0892D0E94CB5262EB3E
:10BE500075E0ECCF6C147D043CF060E0892D0E940D
:10BE6000CB526DEA75E0E2CF69EA75E0DFCF62E0C0
:10BE7000812F0E94FB52812F0E94A25233243394BF
:10BE8000892B09F4FFCE312CFDCE412F50E060E02C
:10BE900070E02AE081EC96E00E94F9156AED75E009
:10BEA00081EC96E00E94C0154AE050E0B20181ECBE
:10BEB00096E00E94DD1663E274E0C7010E94FD1B5C
:10BEC0003C0168E274E0C7010E94FD1B5C016DE269
:10BED00074E0C7010E94FD1B8C0162E374E0C7019E
:10BEE0000E94FD1BFC01892BF1F04114510441F02B
:10BEF000A114B10419F467E374E011C0D50107C0BF
:10BF00000115110519F46AE374E009C0D801199606
:10BF10006D917C911A97DB018C91882321F08185AA
:10BF200092850E948E2061147104E1F1F301618514
:10BF30007285CE01CD960E94CD50CE01CD960E9445
:10BF4000F24F882379F1452869F0A114B10441F436
:10BF500001E020E030E040E050E061E070E01EC031
:10BF6000D5010CC00115110541F401E020E030E0DD
:10BF700040E050E062E070E011C0D80119968D9168
:10BF80009C911A97FC012081222361F00E94E750C6
:10BF900001E020E030E040E050E0BC01CE01CD9671
:10BFA0000E946607D6011C963C927DCEF601238640
:10BFB0007ACEE5E1F9E084E693E091838083128212
:10BFC000138214821582EBE1F9E09183808312825F
:10BFD000138214821582E1E2F9E091838083128258
:10BFE000138214821582EAE0F6E091838083128244
:10BFF000138214821582E7E2F9E091838083128232
:10C00000138214821582EDE2F9E09183808312821B
:10C01000138214821582E3E3F9E091838083128214
:10C02000138214821582E9E3F9E0918380831282FE
:10C03000138214821582E0E1F6E0918380831282FC
:10C04000138214821582E8E1F6E01382128248EE30
:10C0500053E060E070E044835583668377832EED80
:10C0600032E031832083EFE3F9E091838083128211
:10C07000138214821582E4E2F6E013821282448372
:10C0800055836683778320EF32E031832083A5EDEB
:10C09000B0E0B587A487A4EDB0E0B787A687A0ED90
:10C0A000B0E0B18BA08BA1EDB0E0B38BA28BA2ED81
:10C0B000B0E0B58BA48BA6EDB0E0B78BA68B118E4C
:10C0C000128E138E148EE1ECF6E0138212824483FA
:10C0D0005583668377833183208325EC30E0358771
:10C0E000248724EC30E03787268720EC30E0318B42
:10C0F000208B21EC30E0338B228B22EC30E0358B2F
:10C10000248B26EC30E0378B268B118E128E138E0B
:10C11000148EE5E4F9E09183808312821382148205
:10C120001582E8E5F9E091838083128213821482FC
:10C130001582EBE4F9E0138212824483558366830F
:10C1400077832EE333E03183208324E02487109229
:10C15000100910920F0910921209109211091092F1
:10C160001409109213099093EE078093ED07109233
:10C17000EF071092F0071092F1071092F2072FEFDD
:10C180003FEF3093FA072093F907F0935F07E093AE
:10C190005E071092F8071092F707EEE5F9E0918339
:10C1A00080831282138214821582E4E6F9E091837F
:10C1B00080831282138214821582EAE6F9E0918369
:10C1C00080831282138214821582E0E7F9E0918362
:10C1D00080831282138214821582E6E7F9E08FEFE2
:10C1E000808312821182148613868FEF9FEFDC0109
:10C1F00087839087A187B287089597FB072E16F44F
:10C20000009407D077FD09D00E94276107FC05D074
:10C210003EF4909581959F4F0895709561957F4F5D
:10C220000895EE0FFF1F881F8BBF0790F691E02D3A
:10C2300019946927962769277827872778270895EB
:10C240000E94536FB7FF0895821B930B0895AA1B9A
:10C25000BB1B51E107C0AA1FBB1FA617B70710F0F1
:10C26000A61BB70B881F991F5A95A9F78095909523
:10C27000BC01CD0108955058BB27AA270E945361E5
:10C280000C94CD620E94BF6238F00E94C66220F01A
:10C2900039F49F3F19F426F40C94BC620EF4E09537
:10C2A000E7FB0C94B662E92F0E94DE6258F3BA17DE
:10C2B000620773078407950720F079F4A6F50C94BC
:10C2C00000630EF4E0950B2EBA2FA02D0B01B901DF
:10C2D00090010C01CA01A0011124FF27591B99F0FC
:10C2E000593F50F4503E68F11A16F040A22F232F08
:10C2F000342F4427585FF3CF469537952795A79558
:10C30000F0405395C9F77EF41F16BA0B620B730BFE
:10C31000840BBAF09150A1F0FF0FBB1F661F771F6F
:10C32000881FC2F70EC0BA0F621F731F841F48F424
:10C33000879577956795B795F7959E3F08F0B0CFAD
:10C340009395880F08F09927EE0F97958795089594
:10C350000E94926208F481E008950E94C1610C94E9
:10C36000CD620E94C66258F00E94BF6240F029F47C
:10C370005F3F29F00C94B66251110C9401630C9448
:10C38000BC620E94DE6268F39923B1F3552391F3F6
:10C39000951B550BBB27AA2762177307840738F034
:10C3A0009F5F5F4F220F331F441FAA1FA9F335D091
:10C3B0000E2E3AF0E0E832D091505040E695001C45
:10C3C000CAF72BD0FE2F29D0660F771F881FBB1FFF
:10C3D000261737074807AB07B0E809F0BB0B802DDD
:10C3E000BF01FF2793585F4F3AF09E3F510578F009
:10C3F0000C94B6620C9401635F3FE4F3983ED4F36F
:10C40000869577956795B795F7959F5FC9F7880FDC
:10C41000911D9695879597F90895E1E0660F771F2E
:10C42000881FBB1F621773078407BA0720F0621BBF
:10C43000730B840BBA0BEE1F88F7E09508950E94EA
:10C4400026626894B1110C94016308950E94E6621B
:10C4500088F09F5798F0B92F9927B751B0F0E1F0C5
:10C46000660F771F881F991F1AF0BA95C9F714C075
:10C47000B13091F00E940063B1E008950C94006324
:10C48000672F782F8827B85F39F0B93FCCF38695AE
:10C4900077956795B395D9F73EF49095809570950B
:10C4A00061957F4F8F4F9F4F0895E89409C097FB88
:10C4B0003EF490958095709561957F4F8F4F9F4F7B
:10C4C0009923A9F0F92F96E9BB279395F6958795BF
:10C4D00077956795B795F111F8CFFAF4BB0F11F482
:10C4E00060FF1BC06F5F7F4F8F4F9F4F16C0882329
:10C4F00011F096E911C0772321F09EE8872F762F5F
:10C5000005C0662371F096E8862F70E060E02AF09F
:10C510009A95660F771F881FDAF7880F969587958B
:10C5200097F90895990F0008550FAA0BE0E8FEEF60
:10C5300016161706E807F907C0F012161306E407E7
:10C54000F50798F0621B730B840B950B39F40A26E0
:10C5500061F0232B242B252B21F408950A2609F4BE
:10C56000A140A6958FEF811D811D089597F99F67C2
:10C5700080E870E060E008959FEF80EC089500246B
:10C580000A941616170618060906089500240A9438
:10C5900012161306140605060895092E0394000CBE
:10C5A00011F4882352F0BB0F40F4BF2B11F460FF4D
:10C5B00004C06F5F7F4F8F4F9F4F089557FD905876
:10C5C000440F551F59F05F3F71F04795880F97FB57
:10C5D000991F61F09F3F79F0879508951216130611
:10C5E0001406551FF2CF4695F1DF08C01616170640
:10C5F0001806991FF1CF8695710561050894089575
:10C60000E894BB2766277727CB0197F908950E9406
:10C61000926208F48FEF08950E941F630C94CD621C
:10C620000E94BF6238F00E94C66220F0952311F08C
:10C630000C94B6620C94BC6211240C9401630E94A9
:10C64000DE6270F3959FC1F3950F50E0551F629F16
:10C65000F001729FBB27F00DB11D639FAA27F00D5B
:10C66000B11DAA1F649F6627B00DA11D661F829F82
:10C670002227B00DA11D621F739FB00DA11D621F67
:10C68000839FA00D611D221F749F3327A00D611D84
:10C69000231F849F600D211D822F762F6A2F112466
:10C6A0009F5750409AF0F1F088234AF0EE0FFF1F99
:10C6B000BB1F661F771F881F91505040A9F79E3FF0
:10C6C000510580F00C94B6620C9401635F3FE4F373
:10C6D000983ED4F3869577956795B795F795E79546
:10C6E0009F5FC1F7FE2B880F911D9695879597F94F
:10C6F0000895FA01EE0FFF1F309621053105A1F1D3
:10C700006115710561F48038BFE39B0749F16894B6
:10C710009038810561F08038BFEF9B0741F0992385
:10C720004AF5FF3FE1053105210519F1E894089428
:10C73000E795D901AA2329F4AB2FBE2FF85FD0F3D8
:10C7400010C0FF5F70F4A695E0F7F73950F019F0CC
:10C75000FF3A38F49F779F930DD00F9007FC9058C5
:10C76000089546F00C94BC6260E070E080E89FE3BE
:10C7700008954FE79F775F934F933F932F930E94C6
:10C7800074642F913F914F915F910E940C630C94C0
:10C79000D16329F416F00C94B6620C9400630C94E7
:10C7A000BC620E94E662A8F39638A0F707F80F92E1
:10C7B000E8942BE33AEA48EB5FE70E9422630F928A
:10C7C0000F920F924DB75EB70F920E94BC64EAEDD4
:10C7D000F1E00E9403644F915F91EF91FF91E59525
:10C7E000EE1FFF1F49F0FE57E0684427EE0F441F7D
:10C7F000FA95E1F74195550B0E9436640F9007FEBC
:10C800000C942A640895DF93CF931F930F93FF92A4
:10C81000EF92DF927B018C01689406C0DA2EEF0163
:10C820000E941F63FE01E894A591259135914591E1
:10C830005591A6F3EF010E945361FE019701A801F3
:10C84000DA9469F7DF90EF90FF900F911F91CF91ED
:10C85000DF9108959B01AC0160E070E080E89FE308
:10C860000C94AD610C94B6620C94F0640E94E66284
:10C87000D8F39923C9F3940F511DA3F3915050405D
:10C8800094F059F0882332F0660F771F881F91507B
:10C890005040C1F79E3F51052CF7880F911D96958A
:10C8A000879597F908955F3FACF0983E9CF0BB27C1
:10C8B000869577956795B79508F4B1609395C1F71C
:10C8C000BB0F58F711F460FFE8CF6F5F7F4F8F4FBA
:10C8D0009F4FE3CF0C94016316F00C94F0640C941A
:10C8E000BC6268940C94B6620E94E662A8F3992335
:10C8F000C1F3AEF3DF93CF931F930F93FF92C92F32
:10C90000DD2788232AF02197660F771F881FDAF723
:10C9100020E030E040E85FEB9FE3883920F0803E84
:10C9200038F021968F770E943C61E2E0F2E004C08B
:10C930000E943C61EFE2F2E00E9403648B01BE01C1
:10C94000EC01FB2E6F5771097595771F880B990BBA
:10C950000E94576228E132E741E35FE30E941F63D0
:10C96000AF2D9801AE01FF900F911F91CF91DF91F4
:10C970000E9453610C94CD62FA01DC01AA0FBB1F27
:10C980009B01AC01BF5728F4222733274427507856
:10C9900020C0B75190F4AB2F0024469537952795CA
:10C9A000011CA395D2F3002071F0220F331F441F06
:10C9B000B395DAF30ED00C943B6161307105A0E8B9
:10C9C0008A07B94630F49B01AC0166277727882790
:10C9D0009078309621F020833183428353830895E9
:10C9E0009F3F31F0915020F4879577956795B795E3
:10C9F000880F911D9695879597F9089581E090E0AD
:10CA0000F8940C94626F0F931F93CF93DF938C0174
:10CA1000FC0101900020E9F7CF01801B910B0E94DF
:10CA20004566EC01009719F0B8010E946E65CE01D1
:10CA3000DF91CF911F910F910895FB01DC0104C09C
:10CA40008D910190801921F441505040C8F7881B06
:10CA5000990B08956817790768F4FB01DC01E40F6E
:10CA6000F51FA40FB51F02C002900E924150504016
:10CA7000D8F708950C943C66FB01DC018D9181345C
:10CA80001CF08B350CF4805E619161341CF06B35C9
:10CA90000CF4605E861B611189F3990B0895FB010C
:10CAA000DC010D900020E9F7119701900D92002014
:10CAB000E1F70895FC018191861721F08823D9F7C9
:10CAC000992708953197CF010895FB01DC018D91DD
:10CAD000019080190110D9F3990B0895FB01DC0135
:10CAE00001900D920020E1F70895FB01DC010D900B
:10CAF0000020E9F711974150504028F001900020A4
:10CB00000D92C9F708951C920895FB01DC01415074
:10CB1000504030F08D910190801919F40020B9F740
:10CB2000881B990B0895FB01DC014150504048F0EF
:10CB300001900D920020C9F701C01D924150504054
:10CB4000E0F70895FC0181E090E00190061609F4F9
:10CB5000CF010020D1F7019708950F931F93CF9332
:10CB6000DF93CDB7DEB72E970FB6F894DEBF0FBEBA
:10CB7000CDBF0E891F89888D998D26E02C831A835D
:10CB8000098397FF02C080E090E801979E838D8320
:10CB9000AE01445E5F4F6A8D7B8DCE0101960E948F
:10CBA00016694D815E8157FD0AC02F813885421775
:10CBB00053070CF49A01F801E20FF31F10822E962E
:10CBC0000FB6F894DEBF0FBECDBFDF91CF911F919E
:10CBD0000F9108950F931F93CF93DF93CDB7DEB7D7
:10CBE0002E970FB6F894DEBF0FBECDBF0E891F89FA
:10CBF00086E08C831A8309838FEF9FE79E838D8362
:10CC0000AE01465E5F4F688D798DCE0101960E9420
:10CC100016692F813885F801E20FF31F10822E96D6
:10CC20000FB6F894DEBF0FBECDBFDF91CF911F913D
:10CC30000F910895CF93DF93CDB7DEB72E970FB640
:10CC4000F894DEBF0FBECDBF85E08C838C899D89B3
:10CC50009A838983AE01485E5F4F6E897F89CE01DA
:10CC600001960E94C56C2E960FB6F894DEBF0FBEDB
:10CC7000CDBFDF91CF910895FB01DC0102C001908F
:10CC80000D9241505040D8F70895CF93DF938230F2
:10CC9000910510F482E090E0E0918D0BF0918E0B05
:10CCA00020E030E0C0E0D0E0309711F140815181C8
:10CCB00048175907C0F04817590761F482819381DA
:10CCC000209719F09B838A832BC090938E0B8093BF
:10CCD0008D0B26C02115310519F04217530718F4A2
:10CCE0009A01BE01DF01EF010280F381E02DDCCF6C
:10CCF0002115310509F1281B390B2430310590F439
:10CD000012968D919C9113976115710521F0FB018D
:10CD10009383828304C090938E0B80938D0BFD01CF
:10CD2000329644C0FD01E20FF31F8193919322508C
:10CD300031092D933C933AC020918B0B30918C0B91
:10CD4000232B41F420910A0230910B0230938C0B7B
:10CD500020938B0B20910802309109022115310597
:10CD600041F42DB73EB740910C0250910D02241BA7
:10CD7000350BE0918B0BF0918C0BE217F307A0F4CD
:10CD80002E1B3F0B2817390778F0AC014E5F5F4F21
:10CD90002417350748F04E0F5F1F50938C0B4093BC
:10CDA0008B0B8193919302C0E0E0F0E0CF01DF9123
:10CDB000CF9108950F931F93CF93DF93009709F4BA
:10CDC0008CC0FC0132971382128200918D0B10915E
:10CDD0008E0B0115110581F420813181820F931F83
:10CDE00020918B0B30918C0B2817390779F5F09334
:10CDF0008C0BE0938B0B71C0D80140E050E0AE1774
:10CE0000BF0750F412962D913C911397AD01211557
:10CE1000310509F1D901F3CF9D01DA013383228372
:10CE200060817181860F971F8217930769F4EC0167
:10CE300028813981260F371F2E5F3F4F3183208392
:10CE40008A819B8193838283452B29F4F0938E0BF7
:10CE5000E0938D0B42C01396FC93EE931297ED0175
:10CE6000499159919E01240F351FE217F30771F480
:10CE700080819181840F951F029611969C938E93C9
:10CE80008281938113969C938E931297E0E0F0E059
:10CE9000D80112968D919C911397009719F0F80183
:10CEA0008C01F6CF8D919C9198012E5F3F4F820FA0
:10CEB000931F20918B0B30918C0B2817390769F445
:10CEC000309729F410928E0B10928D0B02C01382B2
:10CED000128210938C0B00938B0BDF91CF911F91DB
:10CEE0000F9108958F929F92AF92BF92CF92DF924F
:10CEF000EF92FF92CF93DF93EC01688179818A8171
:10CF00009B81611571058105910521F464E279ED3C
:10CF10008BE597E02DE133EF41E050E00E94216F77
:10CF200049015A019B01AC01A7EAB1E40E94406F9C
:10CF30006B017C01ACEEB4EFA50194010E944E6F31
:10CF4000DC01CB018C0D9D1DAE1DBF1DB7FF03C0C5
:10CF50000197A109B04888839983AA83BB83BC0148
:10CF6000CD019F77DF91CF91FF90EF90DF90CF9031
:10CF7000BF90AF909F908F9008950C9472678EE051
:10CF800092E00C94726760930E0270930F0280938C
:10CF90001002909311020895FC0188279927E894C4
:10CFA00021912032E9F3293010F02E30C8F32B32D2
:10CFB00041F02D3239F4689404C00E943468820F25
:10CFC000911D219120532A30C0F31EF49095819534
:10CFD0009F4F089591110C940F6E803219F0895073
:10CFE0008550C8F70895FB01DC0105900D920020E3
:10CFF000E1F70895FB01DC014150504048F00590F5
:10D000000D920020C9F701C01D9241505040E0F739
:10D01000089549E85BE00C940D68FA01A191B08194
:10D02000009719F41097E1F0CD01DC01CD010D90CE
:10D03000002011F4C00113C0FB012191222319F03B
:10D040002015D9F7F3CFFB012191201519F41E9279
:10D05000119606C02223C1F70D900020A1F7D00140
:10D06000FA01A193B08308957AE0979F902D879F4E
:10D07000802D910D11240895FC01238127FF10C0FC
:10D08000EFE8FBE0208131812817390711F4118284
:10D09000108232962BE0E539F207A1F70E94DA669A
:10D0A00080E090E008950F931F93CF93DF93009754
:10D0B00031F46115710519F480E090E03AC08B01FC
:10D0C000EC016EE070E081E090E00E94F36DFC0105
:10D0D000892B91F380E883830115110571F0138783
:10D0E000028781E8838380918F0B9091900B892B2D
:10D0F00021F4F093900BE0938F0B2097C9F0D18728
:10D10000C0878381826083838091910B9091920B81
:10D11000892B71F4F093920BE093910B8091930B18
:10D120009091940B892B21F4F093940BE093930B43
:10D13000CF01DF91CF911F910F910895CF93DF938E
:10D14000EC012B8120FF33C026FF0AC02F7B2B83ED
:10D150008E819F8101969F838E838A8190E029C072
:10D1600022FF0FC0E881F9818081082E000C990B05
:10D17000009719F420622B831AC03196F983E88353
:10D180000EC0EA85FB85199597FF09C02B81019692
:10D1900011F080E201C080E1822B8B8308C02E81D8
:10D1A0003F812F5F3F4F3F832E83992702C08FEF30
:10D1B0009FEFDF91CF9108950F931F93CF93DF934C
:10D1C000CDB7DEB708851985F80183818860838330
:10D1D000AE01445F5F4F6A857B85C8010E94166976
:10D1E000F8012381277F2383DF91CF911F910F9136
:10D1F00008950F931F93CF93DF93CDB7DEB70885C4
:10D200001985F801838188608383AE01445F5F4F95
:10D210006A857B85C8010E94C56CF8012381277F40
:10D220002383DF91CF911F910F9108952F923F9209
:10D230004F925F926F927F928F929F92AF92BF9226
:10D24000CF92DF92EF92FF920F931F93CF93DF93D2
:10D25000CDB7DEB72C970FB6F894DEBF0FBECDBFAB
:10D260007C016B018A01FC0117821682838181FF98
:10D27000BDC1CE0101964C01F7019381F60193FDEA
:10D28000859193FF81916F01882309F4ABC18532A9
:10D2900039F493FD859193FF81916F01853229F4D3
:10D2A000B70190E00E943A6EE7CF512C312C20E07C
:10D2B0002032A0F48B3269F030F4803259F083329E
:10D2C00069F420612CC08D3239F0803339F421604B
:10D2D00026C02260246023C0286021C027FD27C00B
:10D2E00030ED380F3A3078F426FF06C0FAE05F9E42
:10D2F000300D1124532E13C08AE0389E300D1124B6
:10D30000332E20620CC08E3221F426FD6BC12064C6
:10D3100006C08C3611F4206802C0883641F4F6014C
:10D3200093FD859193FF81916F018111C1CF982F5A
:10D330009F7D9554933028F40C5F1F4FFFE3F983D2
:10D340000DC0833631F0833771F0833509F05BC04F
:10D3500022C0F801808189830E5F1F4F44244394CB
:10D36000512C540115C03801F2E06F0E711CF80108
:10D37000A080B18026FF03C0652D70E002C06FEF72
:10D380007FEFC5012C870E942F6E2C0183012C8515
:10D390002F77222E17C03801F2E06F0E711CF801B2
:10D3A000A080B18026FF03C0652D70E002C06FEF42
:10D3B0007FEFC5012C870E941D6E2C012C852068F3
:10D3C000222E830123FC1BC0832D90E048165906B2
:10D3D000B0F4B70180E290E00E943A6E3A94F4CF44
:10D3E000F50127FC859127FE81915F01B70190E04F
:10D3F0000E943A6E31103A94F1E04F1A51084114EC
:10D40000510471F7E5C0843611F0893639F5F80119
:10D4100027FF07C060817181828193810C5F1F4F5C
:10D4200008C060817181072E000C880B990B0E5F7C
:10D430001F4F2F76722E97FF09C09095809570959B
:10D4400061957F4F8F4F9F4F2068722E2AE030E00A
:10D45000A4010E948B6EA82EA81844C0853729F419
:10D460002F7EB22E2AE030E025C0F22FF97FBF2EAA
:10D470008F36C1F018F4883579F0B4C0803719F0D0
:10D48000883721F0AFC02F2F2061B22EB4FE0DC01F
:10D490008B2D8460B82E09C024FF0AC09F2F966090
:10D4A000B92E06C028E030E005C020E130E002C01F
:10D4B00020E132E0F801B7FE07C06081718182810E
:10D4C00093810C5F1F4F06C06081718180E090E006
:10D4D0000E5F1F4FA4010E948B6EA82EA818FB2D73
:10D4E000FF777F2E76FE0BC0372D3E7FA51450F4BC
:10D4F00074FE0AC072FC08C0372D3E7E05C0BA2CEF
:10D50000372D03C0BA2C01C0B52C34FF0DC0FE016D
:10D51000EA0DF11D8081803311F4397E09C032FF9C
:10D5200006C0B394B39404C0832F867809F0B394F3
:10D5300033FD13C030FF06C05A2CB31418F4530C3B
:10D540005B18B32CB31468F4B70180E290E03C8719
:10D550000E943A6EB3943C85F5CFB31410F43B1897
:10D5600001C0312C34FF12C0B70180E390E03C874A
:10D570000E943A6E3C8532FF17C031FD03C088E738
:10D5800090E002C088E590E0B7010CC0832F867858
:10D5900059F031FF02C08BE201C080E237FD8DE21D
:10D5A000B70190E00E943A6EA51438F4B70180E309
:10D5B00090E00E943A6E5A94F7CFAA94F401EA0DD3
:10D5C000F11D8081B70190E00E943A6EA110F5CF65
:10D5D000332009F451CEB70180E290E00E943A6E08
:10D5E0003A94F6CFF7018681978102C08FEF9FEFC3
:10D5F0002C960FB6F894DEBF0FBECDBFDF91CF9152
:10D600001F910F91FF90EF90DF90CF90BF90AF9060
:10D610009F908F907F906F905F904F903F902F9052
:10D62000089520FD09C0FC0123FD05C022FF02C0B2
:10D630007383628351834083089544FD10C046FD87
:10D6400010C0DB01FC01AA0FBB1FEE1FFF1F1094CF
:10D65000D1F76A0F7B1F8E1F9F1F31E003C033E09D
:10D6600001C034E0660F771F881F991F3150D1F732
:10D67000620F711D811D911D08950F931F93CF930C
:10D68000DF938C01C8010E949E68EC0197FD08C0E1
:10D690000E94EA67892BB1F7B801CE010E94726E31
:10D6A000CE01DF91CF911F910F9108958F929F929C
:10D6B000AF92BF92CF92DF92EF92FF920F931F93A0
:10D6C000CF93DF931F92CDB7DEB78C01C62E7A01C0
:10D6D00029830E949E68AC01552729814B32510550
:10D6E00021F04D32510569F42068CA94C11002C07E
:10D6F00080E076C0C80129830E949E68298197FD39
:10D70000F7CF322F3D7FD32E322F307349F5803340
:10D7100039F5BB24BA94BC0C09F44EC0C801298366
:10D720000E949E68298197FD47C0382F3F7D38357C
:10D7300069F48D2D8264D82ECA94CA94CC20E1F16C
:10D74000C8010E949E6897FF0BC036C026FF04C028
:10D750002D2D2260D22E03C03D2D3261D32ECB2C35
:10D76000812C912C540120ED280F283080F0D4FE1C
:10D7700004C0B8010E94726E1CC02A3040F0D6FE70
:10D78000F8CF2F7D3FEE320F363098F727504D2DD2
:10D79000C501B4010E941D6B4B015C018D2D82609F
:10D7A000D82ECA94CC2059F0C8010E949E6897FFD9
:10D7B000DACFD1FC04C09CCF812C912C5401D7FE30
:10D7C00008C0B094A09490948094811C911CA11CDA
:10D7D000B11C2D2DB501A401C7010E94116B81E080
:10D7E0000F90DF91CF911F910F91FF90EF90DF90FD
:10D7F000CF90BF90AF909F908F9008956F927F923F
:10D800008F929F92AF92BF92CF92DF92EF92FF9250
:10D810000F931F93CF93DF93CDB7DEB7A1970FB6CA
:10D82000F894DEBF0FBECDBF5C017A01CE01019638
:10D830006C0180E2F60111928A95E9F7F501838087
:10D8400040E050E0912C712C70E0A1E0B0E0F901D3
:10D8500083FC859183FE81918F01982F9F01811117
:10D8600003C080E090E07CC08E3519F4411551056D
:10D8700049F1E72FF0E0E417F5073CF48D3559F155
:10D880008D3219F4772001F103C0711001C0982E78
:10D89000892F8695869586958601080F111D892FFB
:10D8A00087703D0101C0660C8A95EAF7F801808116
:10D8B00086298083991559F0991510F49F5FE8CF58
:10D8C0009150E6CF71E004C07724739401C0712CAD
:10D8D0004F5F5F4FBCCF772019F08E8180628E83BF
:10D8E000711103C09924939416C0F6019E012F5D17
:10D8F0003F4F808180958193E217F307D1F7F2CFF4
:10D90000E114F10429F0F7018083C70101967C013D
:10D910006150912CF9F0C50169A30E949E6869A12C
:10D9200097FD16C0282F269526952695F601E20F1D
:10D93000F11D208130E0AC014770552702C03595BC
:10D9400027954A95E2F720FDDBCFB5010E94726E64
:10D95000911087CFE114F10411F0F7011082C80192
:10D96000A1960FB6F894DEBF0FBECDBFDF91CF9169
:10D970001F910F91FF90EF90DF90CF90BF90AF90ED
:10D980009F908F907F906F9008954F925F927F92BB
:10D990008F929F92AF92BF92CF92DF92EF92FF92BF
:10D9A0000F931F93CF93DF931F92CDB7DEB76C0118
:10D9B0002B015A01FC0117821682712CF601F380AB
:10D9C000F201F3FC8591F3FE8191382F2F0188231A
:10D9D00009F4F3C090E039830E94EA673981892B0A
:10D9E00021F0C6010E943D6BE9CF353241F4F201CE
:10D9F000F3FC3591F3FE31912F01353269F4C60104
:10DA000039830E949E68398197FDD5C03817B1F2DD
:10DA1000B6010E94726ED1C03A3239F4F3FC3591EE
:10DA2000F3FE31912F0151E001C050E0420110E0BE
:10DA300020ED230F2A3090F45260612F70E080E0D7
:10DA400090E040E259830E941D6B162FF401F3FC15
:10DA50003591F3FE31914F015981EACF052F232FE4
:10DA6000240151FF03C0111102C0A7C01FEF3836B7
:10DA700019F03C3659F011C0F401F3FC2591F3FE86
:10DA800021912F01283649F4052F08600460F20126
:10DA9000F3FC2591F3FE21912F01222309F48DC07F
:10DAA000622F70E087E59EE029830E94126E298133
:10DAB000892B09F482C000FD07C0F501E080F180E8
:10DAC000C50102965C0102C0E12CF12C2E3651F406
:10DAD000F6014681578160E070E0202FC7010E9467
:10DAE000116B6CCF233691F401FF11E0C6010E9447
:10DAF0009E6897FD60C0E114F10429F0F70180836E
:10DB0000C70101967C01115089F751C02B3559F49A
:10DB10009201A701612FC6010E94FE6B2C01892B87
:10DB200009F045C03FC0C60129830E943D6B298191
:10DB300097FD41C02F3659F128F4243631F12936AA
:10DB400049F127C0233769F02537F9F022C0E114E5
:10DB5000F10429F0F7018082C70101967C01115080
:10DB600071F0C6010E949E684C0197FD08C00E949A
:10DB7000EA67892B61F3B601C4010E94726EE11459
:10DB8000F104A9F0F701108212C0006203C0006125
:10DB900001C00064202FA701612FC6010E94566BAF
:10DBA000811105C0F6018381807329F406C000FD50
:10DBB00005CF739403CF772019F0872D90E002C032
:10DBC0008FEF9FEF0F90DF91CF911F910F91FF90FB
:10DBD000EF90DF90CF90BF90AF909F908F907F900D
:10DBE0005F904F9008950F931F93CF93DF93869F7D
:10DBF0008001879F100D969F100D1124C8010E946F
:10DC00004566EC01009729F0A80160E070E00E94F1
:10DC1000286ECE01DF91CF911F910F910895992722
:10DC200088270895FC010590061621F00020D9F7F9
:10DC3000C00108953197CF010895FC01059061500E
:10DC400070400110D8F7809590958E0F9F1F089512
:10DC5000DC0101C06D9341505040E0F70895FC0194
:10DC60006150704001900110D8F7809590958E0F0B
:10DC70009F1F08950F931F93CF93DF93FB01238181
:10DC800021FD03C08FEF9FEF28C022FF16C0468101
:10DC90005781248135814217530744F4A081B18113
:10DCA0009D012F5F3F4F318320838C9326813781E5
:10DCB0002F5F3F4F3783268310C0EB01092F182FAA
:10DCC0000084F185E02D1995892BE1F68E819F81E5
:10DCD00001969F838E83812F902FDF91CF911F918B
:10DCE0000F910895FB01238120FF12C026FD10C073
:10DCF0008F3F3FEF930761F082832F7D2064238362
:10DD00002681378121503109378326839927089549
:10DD10008FEF9FEF0895FA01AA27283051F12031A3
:10DD200081F1E8946F936E7F6E5F7F4F8F4F9F4FAF
:10DD3000AF4FB1E03ED0B4E03CD0670F781F891FF1
:10DD40009A1FA11D680F791F8A1F911DA11D6A0FBF
:10DD5000711D811D911DA11D20D009F468943F9172
:10DD60002AE0269F11243019305D3193DEF6CF0171
:10DD70000895462F4770405D4193B3E00FD0C9F737
:10DD8000F6CF462F4F70405D4A3318F0495D31FDA4
:10DD90004052419302D0A9F7EACFB4E0A6959795F7
:10DDA000879577956795BA95C9F7009761057105CD
:10DDB00008959B01AC010A2E069457954795379517
:10DDC0002795BA95C9F7620F731F841F951FA01D71
:10DDD0000895F999FECF92BD81BDF89A992780B533
:10DDE0000895262FF999FECF1FBA92BD81BD20BD9F
:10DDF0000FB6F894FA9AF99A0FBE01960895A1E227
:10DE00001A2EAA1BBB1BFD010DC0AA1FBB1FEE1FB4
:10DE1000FF1FA217B307E407F50720F0A21BB30BFF
:10DE2000E40BF50B661F771F881F991F1A9469F77B
:10DE300060957095809590959B01AC01BD01CF01D7
:10DE40000895052E97FB1EF400940E94386F57FD2D
:10DE500007D00E94FF6E07FC03D04EF40C94386F7D
:10DE600050954095309521953F4F4F4F5F4F089506
:10DE700090958095709561957F4F8F4F9F4F089536
:10DE80000E94536FA59F900DB49F900DA49F800D8D
:10DE9000911D11240895B7FF0C94406F0E94406FAC
:10DEA000821B930B0895A29FB001B39FC001A39F53
:10DEB000700D811D1124911DB29F700D811D1124C3
:08DEC000911D0895F894FFCFB5
:10DEC80003100000C00120000000950B8000010035
:10DED8000000DEADBEEFFE005E00BC007701000072
:10DEE8000000660700000000992050148D2A4D306C
:10DEF800D820B620E62054218F21000000001121EF
:10DF080050148D2A4D305B21D121E62054218F21D8
:10DF180000044D515454046C617A79686F6D652E14
:10DF28007275000000000000000000000000000002
:10DF38000000000000000000000000932150148D34
:10DF48002A4D302921A421E62054218F21000000E8
:10DF580000E126AE278D2A7D4574465A463346226F
:10DF6800283027564662473E477545032701276AEA
:10DF780045F72600000000112150148D2A4D305B12
:10DF880021C121E62054218F2130313233343536F6
:10DF98003738394142434445460000000000735277
:10DFA800FB448D2A0E4132411E410F410000000002
:10DFB8000615501494144D15C514A314B714000075
:10DFC8000000A615A6158D2AA615A615A615A61530
:10DFD800A615A615A615A615A615A61500000000D7
:10DFE800A61550148D2A8C2AA615A615A61500006C
:10DFF8000000A61550148D2A8C2A00000000E12686
:10E00800AE278D2A7D4574465A4633462228302746
:10E01800564662473E477545032701276A45F72656
:10E0280000000000931600000000A6150000000084
:10E03800A615A6158D2AA615A615A615A615A61504
:10E048006845A615A615A615A615A615A615A615FE
:10E05800A615A61500000000A24C474D8D2AA14C1C
:10E068004945134E2E4D0646B84CF145F6467E45B9
:10E07800AD463C4EF44D614551454D4501005E00AD
:10E088000000000000000000000068656C7000736C
:10E09800617665006C6F6164006765740073657410
:10E0A800006B696C6C00726571000D0A0020005FDE
:10E0B8007374617400560052504D00490073770024
:10E0C800666C7400707772002F616C61726D2F6FCF
:10E0D80076726874002F616C61726D2F736E737243
:10E0E8000053006974656D0073636D640072636D3D
:10E0F8006400656D6974004F4E004F4646002578F0
:10E108003A25783A25783A25783A25783A257825AF
:10E11800D181002F726573702F23002F7265712FC4
:10E12800636F6E660031002F253032782D2530322E
:10E13800782D253032782D253032782D25303278DB
:10E148002D253032782E636F6E6669672E6A736F7D
:10E158006E0025252532780023253258253258258A
:10E168003258002564002C0022006E756C6C007417
:10E178007275650066616C7365002D002E00646D14
:10E188007800646D78696E006D6F64627573006FF6
:10E1980077006974656D73006D7174740057495A1E
:10E1A8006E65740031772054696D656F757400521F
:10E1B80065736574206572726F720020636F6D708D
:10E1C8005F696421005245535400544F47474C45FA
:10E1D8000048414C54003B002F616C61726D6F66C2
:08E1E800662F736E73720000D4
:00000001FF
